:020000040800F2
:1080000008C10020A1810008A9810008A9A90008D1
:10801000AD810008AF810008B181000800000000B8
:10802000000000000000000000000000B381000814
:10803000B581000800000000B7810008B981000880
:10804000BB810008BB810008BB810008BB81000820
:10805000BB810008BB810008BB810008BB81000810
:10806000BB810008BB810008BB810008BB81000800
:10807000BB810008BB8100082397000827970008F0
:10808000BB8100082B970008BB810008BB8100085A
:10809000BB810008BB810008BB810008BB810008D0
:1080A000BB810008BB810008BB810008BB810008C0
:1080B000658C0108BB810008BB810008BB810008FA
:1080C000BB810008BB810008BB810008BB810008A0
:1080D000BB810008B9940108BD940108C19401084E
:1080E000DF9A0008BB810008BB810008BB81000843
:1080F000BB810008BB810008BB8100082F970008E6
:10810000BB810008BB810008BB810008BB8100085F
:10811000B1940108B5940108BB810008BB81000837
:10812000BB810008BB810008BB810008BB8100083F
:10813000BB810008BB810008BB810008BB8100082F
:10814000BB810008BB810008BB810008BB8100081F
:10815000BB8100083397000837970008C5940108D1
:10816000BB810008BB810008BB810008BB810008FF
:10817000BB810008BB810008BB810008BB810008EF
:10818000BB810008BB810008DFF810D000F00EFCB6
:1081900000480047E1B10108AFF3008008C10020AA
:1081A0000648804706480047FEE7FEE7FEE7FEE791
:1081B000FEE7FEE7FEE7FEE7FEE7FEE7098C0108C3
:1081C000898100082DE9F0410024061B254671F144
:1081D000000605DA01240027D0EB070067EB010158
:1081E000161E73F1000605DA0027D2EB07020125FF
:1081F00067EB030300F077FA86460E4617469C4667
:10820000AC4204D00025D0EB050E65EB010624B18D
:108210000020D2EB000760EB030C704631463A4673
:108220006346BDE8F081202A06DBCB17203A41FAED
:1082300002F043EAE07306E041FA02F3D040C2F1F3
:108240002002914008431946704740EA01039B070A
:1082500003D009E008C9121F08C0042AFAD203E0BB
:1082600011F8013B00F8013B521EF9D27047421E43
:1082700012F8013F002BFBD111F8013B02F8013B42
:10828000002BF9D17047421C10F8011B0029FBD1CB
:10829000801A704730B505460020034600E05B1C9D
:1082A000934205D2EC5CC85C201A01D1002CF6D1B7
:1082B00030BD2DE9FE4F804681EA0300C00F0C4619
:1082C000009021F0004123F00045B8EB0200A941E5
:1082D00005D24046214690461C460B46024623F0F6
:1082E0000040104347D0270DC7F30A00C3F30A51DB
:1082F0000290401A019040286BDAC3F3130040F457
:10830000801B0098924620B10023D2EB030A63EB56
:108310000B0B01985946C0F14002504600F014FA88
:1083200006460D4650465946019AFFF77CFF10EB72
:1083300008006141002487EA115284EAE7731A4376
:1083400040D0009A62B3019A012A4FEA075215DC25
:10835000001B61EB02014FF0004202EA0752CDE937
:108360000042001C41F5801132462B4600F0A0FA75
:1083700003B0BDE8F08F40462146F9E7001B61EBF2
:108380000201001C41F5801300185B412018A2F582
:10839000001747EB030140EAD570B6196D4111E0B3
:1083A0006D084FEA360645EAC0754FEA0752001BD2
:1083B00061EB0201001C41F5801149084FEA3000D1
:1083C0000019514132462B4603B0BDE8F04F00F092
:1083D00060BA0098012240000023D0EB020263EB58
:1083E000E073009821464FEAE074B8EB000061EBBF
:1083F0000401E9E783F000435BE781F0004158E7BF
:108400002DE9FE4F81EA030404F0004421F000410D
:1084100000944FF0000B23F0004350EA01045ED0BB
:1084200052EA03045BD0C3F30A54C1F30A552C4447
:10843000A4F2F3340194A0FB0254C1F3130141F4FC
:108440008011C3F3130343F4801301FB024400FBC8
:10845000034E840A970A44EA815447EA8357A4FBEF
:10846000076802958D0A05FB07854FEA932C04FBEC
:108470000C542705029D4FEA065847EA1637B5EB1C
:1084800008056EEB070C870E920E47EA811742EA49
:108490008312A7FB0201B6EB0B0164EB00042B0D6A
:1084A00043EA0C335E1844EB1C50DA465146E7FBB6
:1084B0000201C5F313044FEA0B3343EA14534FEAA6
:1084C0000432019C43EA0603A4F10C040294009CCC
:1084D000CDE900B400F0ECF903B0BDE8F08F002066
:1084E0000146F9E72DE9F04D81EA030404F0004B61
:1084F00021F0004514464FF0000A23F0004150EAF5
:10850000050220D054EA01021DD0C5F30A570246E5
:10851000C5F31303C1F31300C1F30A5640F48015E9
:1085200043F48013A7EB0608101BD64608F2FD386B
:1085300073EB050002D308F1010801E092185B41DA
:10854000B8F1000F03DA00200146BDE8F08D0020ED
:108550004FF48011064684460EE0171B73EB0507A7
:1085600005D3121B63EB050306434CEA010C4908D3
:108570004FEA300092185B4150EA0107EDD152EA10
:10858000030012D082EA040083EA0501084305D003
:10859000101BAB4106D20122002306E000224FF05F
:1085A000004302E06FF0010253101AEB06004CEB9F
:1085B000085110EB0A0041EB0B01BDE8F04D00F053
:1085C00068B90EB5C10F80EAE0700844CA070021FF
:1085D00040F233438DE80E000A460B4600F068F97E
:1085E00003B000BD0EB540F2334102910021CDE948
:1085F00000110A460B4600F05BF903B000BD3EB522
:10860000CA17CB0F002450405140C0186141DA070F
:1086100040F233430094CDE901232246234600F083
:1086200047F903B030BD70B5C1F30A5201F00045FF
:108630000024C1F3130140F2FF3341F480119A4248
:1086400001DA002070BD40F233439A42A2F2334275
:1086500003DC524200F087F800E090402C43F1D058
:10866000404270BD70B5C1F30A5201F000450024CC
:10867000C1F3130140F2FF3341F480119A4202DA50
:108680000020014670BD40F233439A42A2F23342C9
:1086900003DC524200F067F801E000F055F82C438B
:1086A000F0D00023D0EB030063EB010170BD01F0BB
:1086B000004330B421F0004150EA010206D00A0D17
:1086C000A2F56072C1F31301002A02DC30BC002065
:1086D0007047440F44EAC104C100E01830BC00EB0D
:1086E000C25000F09FB82DE9F05F05460020924689
:1086F0009B4688460646814640241BE02846414664
:108700004746224600F02FF853465A46C01A914178
:1087100010D311461846224600F016F82D1A67EBC2
:1087200001084F4622460120002100F00DF817EB0A
:1087300000094E41201EA4F10104DFDC4846314609
:108740002A464346BDE8F09F202A04DB203A00FA7F
:1087500002F1002070479140C2F1200320FA03F398
:10876000194390407047202A04DB203A21FA02F096
:108770000021704721FA02F3D040C2F1200291405B
:1087800008431946704700000FB4002300B589B0B4
:108790000CA900910B996FF00042CB601E4B069321
:1087A0001E4B07930423CDE901321D4A089202466D
:1087B0006B46002000F0A6F909B05DF814FB70B517
:1087C00086B006464FF0FF300091CDE90101002050
:1087D00015460C4604903246694604A8FFF7D4FFBC
:1087E00002460498211825B108B1084600E0204649
:1087F0002860049800280DD0002A02DD00988842E5
:1088000008D0081B0094CDE901043246694604A84B
:10881000FFF7BAFF06B070BD3D8D00085B8D000804
:10882000D18900080029A8BF7047401C490008BF33
:1088300020F00100704710B4B0FA80FC00FA0CF090
:1088400050EA010404BF10BC704749B1CCF12004C8
:1088500021FA04F411FA0CF118BF01212143084355
:10886000A3EB0C01CB1D4FEA00614FEA102042BF81
:10887000002010BC704700EBC35010440029A4BF77
:1088800010BC7047401C490008BF20F0010010BC1C
:10889000704710B5141E73F1000408DA401C41F152
:1088A000000192185B411A4301D120F0010010BD74
:1088B0002DE9F04D92469B4611B1B1FA81F202E0EA
:1088C000B0FA80F220329046FFF73EFF04460F4692
:1088D00040EA0A0041EA0B0153465A46084313D0C6
:1088E000114653EA010019D0C8F140025046FFF783
:1088F0003AFF05460E46504659464246FFF724FFCA
:10890000084305D0012004E020463946BDE8F08D3B
:108910000020054346EAE0762C4337430A98630576
:10892000E40AA0EB08000022FD0A44EA47540A309A
:1089300002D500200146E9E7010510196941DDE98A
:10894000084500196941BDE8F04DA2E770B521F076
:10895000004303430CD0C1F30A550024D5EB0405B2
:1089600064EB0403D617AD1AB34102DB00200146C5
:1089700070BD201841EB025170BD000030B5041EDF
:1089800071F1000404DB4FF00044404264EB01014C
:10899000141E73F1000405DB1C464FF000435242E5
:1089A00063EB0403994208BF904230BD064C074D6B
:1089B00006E0E06840F0010394E8070098471034AF
:1089C000AC42F6D3FFF7E4FBD0DF0108F0DF01088B
:1089D000C0B24FF4F05100F03BBA00002DE9FF4F58
:1089E000087883B09946FF2805D0491C2D2804D06B
:1089F0000024002008E000200BE00124F9E700EB50
:108A0000800003EB4000491C0B78FF2BF7D104B129
:108A1000404200230293147819461D462D2C01D0A4
:108A20002B2C04D1521C2D2C13D000240294AA46C6
:108A30001478FF2C0FD00A25A3FB057801FB0581D4
:108A40004FF0000C03FB0C11521CE3194AEB01011F
:108A5000EEE70124EAE7814453EA010002D019F568
:108A6000C87F06DA03980021C0E9001107B0BDE80D
:108A7000F08F0025AE4E2F46DFF8B882184600F082
:108A8000FBF9CDE90001B9F1000002DAC9F10004F7
:108A900000E004460023A74A1AEB030B42EB045AFA
:108AA00012E0E00707D02A46334638464146FFF732
:108AB000A7FC074688462A46334610461946FFF764
:108AC0009FFC05460E466410002CEAD1DDE900014A
:108AD000B9F1000F5A46534606DAFFF703FD3A464E
:108AE0004346FFF7FFFC05E0FFF78AFC3A464346A2
:108AF000FFF786FC029A0AB181F00041039AC2E9AD
:108B00000001B3E72DE9FF4F1F468DB0D7E90146BD
:108B10004FF0FF382E2045464FF000090B90B96901
:108B20006D1C0E988847396A824688470028F6D11E
:108B3000BAF1FF3F0AD024F4D064002E11DDBAF15F
:108B40002B0F08D0BAF12D0F0BD102E0404611B027
:108B50008DE744F48064B9696D1C0E98884782469D
:108B6000761E6946600501D52D2000E02B208DF88A
:108B7000000001F1010B0DF1200809E0B9696D1C3D
:108B80000E98884782460F9844F40074761E05605C
:108B9000002E02DDBAF1300FF0D00B998A453ED19C
:108BA00044F0800406E00F99681CA9F1010944F41F
:108BB00000740860B9696D1C761E0E98884782465D
:108BC0003028F0D02BE00B998A4505D1200603D43C
:108BD00044F08004761E18E0504611F059FF08B3A7
:108BE0000DF11301761E44F400748B4508D2AAF1EE
:108BF00030000BF8010B200607D5A9F1010003E0B6
:108C0000200602D409F101008146A00502D50F9982
:108C1000681C0860B9696D1C0E9888478246002E52
:108C2000D1DC53E0002E51DDBAF1650F02D0BAF16C
:108C3000450F4BD1A00549D5B9696D1C24F440748A
:108C4000761E0E9888478246002E0CDD2B2804D015
:108C5000BAF12D0F07D144F48074B9696D1C0E98D8
:108C600088478246761EE00501D52D2100E02B21A4
:108C700008F8011BCDF82C8021E00DF12901761EAA
:108C800044F4007488450CD2AAF1300010F0FF00C3
:108C900088F8000002D10B99884509D908F101082C
:108CA00006E0E00501D5244801E042F20F7081465C
:108CB000B9696D1C0E98884782460F980560002E92
:108CC00004DD504611F0E4FE0028D6D1F9690E9873
:108CD0008847FF208BF8000088F8000000200690ED
:108CE00007904B466A4608A906A8FFF777FEA0053D
:108CF00002D46FF001002AE714F0240F0AD0E00735
:108D000014D1DDE906123868031D3B600068C0E934
:108D100000120BE0DDE90601FFF7C9FC0146E007A0
:108D200004D13868021D3A600068016028460EE7E9
:108D3000000014400000F03FF1D8FFFF426842B14C
:108D4000016811F8013B23B1521EC0E90012184618
:108D500070470121C160881E704742685AB1C368DC
:108D6000016843B983688B4205D0491E521CC0E993
:108D70000012002070474FF0FF3070472DE9F04D92
:108D800000231A461B1A8A4103DB00200146BDE876
:108D9000F08DC1F30A52C1F3130141F480154FF075
:108DA000000BD10702D100186D41521E0027044666
:108DB00040F2FF11384601EB620A3E468046024609
:108DC00000204FF48011FFF7CEFCC2197141BB188F
:108DD00046EB0100B4EB030C75EB000C04D3E41A72
:108DE00065EB000517460E46241908F101006D4198
:108DF00080463428E3DDF91946EB0600091BA8413B
:108E000003D24FF0FF32134601E0002213461BEB62
:108E1000070046EB0A51BDE8F04DFFF73ABD0000F0
:108E200030B5041E71F1000404DB4FF000444042F1
:108E300064EB0101141E73F1000405DB1C464FF0C6
:108E40000043524263EB04038B4208BF824230BDB1
:108E50007F2801D9002208E0064A02EB5002C00731
:108E6000127800D1120902F00F0201209040084050
:108E70007047000090DF01080EB540F233420292C5
:108E80000022CDE900221346FFF712FD03B000BD1A
:108E900070B58C1810F8015B15F0070301D110F8BC
:108EA000013B2A1106D110F8012B03E010F8016BE9
:108EB00001F8016B5B1EF9D12B0705D40023521E6C
:108EC0000DD401F8013BFAE710F8013BCB1A921CD4
:108ED00003E013F8015B01F8015B521EF9D5A142D2
:108EE000D8D3002070BD027803E010F8013B1A448B
:108EF000D2B2491E89B2F8D21046704770B5ADF5AE
:108F0000287D00260D46ADF89462ADF8986200EB1E
:108F100040012D4800EBC104608AA84251D9ADF848
:108F200098624AE0A089228A284481B2274800F04A
:108F3000B1F8ADF894626A46208A0BE0BDF894322D
:108F40006168C95CBDF89432D154BDF89412491CD3
:108F5000ADF89412BDF894128842EFD8401E81B249
:108F60001046FFF7C0FF1A498870228A0DF1FF31C1
:108F7000515C814219D1ADF894620CE0BDF89412B5
:108F80006068BDF89422405CA1688854BDF89402E2
:108F9000401CADF89402208ABDF89412401E88420D
:108FA000ECDC01200DF5287D70BD642011F0A8FFD8
:108FB000BDF89802401CADF89802BDF8980206284A
:108FC000B0D30020EEE7000080BD0108707A0020D9
:108FD00022120020F0B50D46064600EB46011C4863
:108FE000002200EBC104ADF5257D608AA8422BD993
:108FF000694606E0A0686368805C98548854521CF7
:1090000092B2208A401E9042F4DC208A401E81B237
:109010006846FFF768FF228A0DF1FF3100275054A0
:10902000A089228A284481B2684600F02FF9294697
:109030003046FFF763FF012807D0642011F060FF7E
:109040007F1CBFB2062FEBD300200DF5257DF0BDB0
:1090500080BD010838B50025ADF800500DF004FFC3
:109060000A4C207000F088F821780948242907D09C
:10907000272908D0282902D1022180F8A51138BD5E
:1090800080F8A55138BD0121F7E700002212002029
:10909000D42200202DE9F041064615460C46012059
:1090A00080F31088254F0020B8800DF0BDFE00062B
:1090B00009D4012011F024FFB888401C80B2B88088
:1090C000C828F2D335E0B888C82832D21C4F102106
:1090D000384601F0BCF90821384601F0BAF9E82019
:1090E00000F030F8C4F3871000F02CF8A006000E52
:1090F00000F028F8002000F025F80024002000F0FF
:1091000021F8641CA4B2042CF8D3002405E0FF204D
:1091100000F018F83055641CA4B2AC42F7D310210B
:10912000384601F096F9002080F310880120BDE850
:10913000F081002080F31088F9E70000221200205F
:109140000000024070B50B4C0546022120460DF090
:1091500085FF0028F9D0294620460DF088FF01211F
:1091600020460DF07BFF0028F9D020460DF07DFF52
:10917000C0B270BD0030014010B5012080F31088EE
:109180001A4C0020A0800DF04FFE000609D40120EB
:1091900011F0B6FEA088401C80B2A080C828F2D38F
:1091A00020E0A088C8281DD2114C1021204601F0D3
:1091B0004EF90821204601F04CF93D20FFF7C2FF8F
:1091C0002A20FFF7BFFF8020FFF7BCFFA720FFF793
:1091D000B9FF1021204601F03CF9002080F31088EF
:1091E000012010BD002080F3108810BD2212002045
:1091F000000002402DE9F04106460D46012080F3B3
:109200001088204C0020A0800DF00EFE000609D42E
:10921000012011F075FEA088401C82B2A280C82AED
:10922000F2D32AE0A088C82827D2174F1021384649
:1092300001F00DF90821384601F00BF98420FFF701
:1092400081FF0020FFF77EFF0020FFF77BFF00205B
:10925000FFF778FF002404E0305DFFF773FF641C24
:10926000A4B2AC42F8D31021384601F0F2F8002045
:1092700080F310880120BDE8F081002080F3108881
:10928000F9E70000221200200000024070B50D46F0
:10929000012181F310881146FFF7ACFF002832D07E
:1092A0001B4C0020A0800DF0BFFD000609D401205A
:1092B00011F026FEA088401C80B2A080C828F2D3FE
:1092C00022E0A088C8281FD2124C1021204601F0AD
:1092D000BEF80821204601F0BCF88320FFF732FFDA
:1092E000C5F38710FFF72EFFA806000EFFF72AFF31
:1092F0000020FFF727FF1021204601F0AAF80020E8
:1093000080F31088012070BD002080F3108870BDAC
:10931000221200200000024010B500231A4604E08B
:1093200010F8014B6340521CD2B28A42F8D318465F
:1093300010BD000010B50446392011F0E1FFE0B285
:1093400011F0FEFFC4F3072011F0FAFFC4F3074049
:1093500011F0F6FF200E11F0F3FF4FF48051034897
:1093600001F077F8BDE8104010F09EB9000402400B
:109370002DE9F041054614460E463A2011F0C0FF93
:10938000F0B211F0DDFF300A11F0DAFF104F4FF4A8
:1093900080563146384601F05CF8B0463E4610F043
:1093A00083F91D2811D1284600F0A4F807463B2078
:1093B00011F0A6FF4146304601F04BF83D44002C29
:1093C000EDD0208838442080E9E7BDE8F081000036
:1093D000000402402DE9F041054614460E463C20AB
:1093E00011F08EFFF0B211F0ABFF300A11F0A8FFC0
:1093F000114F4FF480563146384601F02AF80CB12F
:1094000000202080B0463E4610F04EF91E2811D1B3
:10941000284600F017F907463D2011F071FF41463C
:10942000304601F016F83D44002CEDD02088384439
:109430002080E9E7BDE8F0810004024010B50DF09E
:109440003BFC08B100F028F8BDE81040302000F0E7
:109450009FB80146362000F089B810B508B100F079
:10946000A5F8BDE81040342000F092B810B50446CD
:1094700000F09CF820785C2801D02F2803D100212F
:10948000642000F0FBF8BDE81040322000F080B806
:10949000682000F04BB8000010B5222011F030FF1A
:1094A00011F024FF04464FF48051024800F0D1FF30
:1094B000204610BD000402402DE9F04111F016FFD6
:1094C000064611F013FF054611F010FF044611F097
:1094D0000DFF07464FF48051054800F0BAFF46EAF9
:1094E000052040EA044040EA0760BDE8F081000042
:1094F0000004024070B50546272011F001FF11F06D
:10950000F5FE0446260007D011F0F0FE641E05F8B3
:10951000010B14F0FF04F7D14FF48051024800F022
:1095200098FF304670BD00000004024010B50446AC
:109530000C2011F0E5FE204611F002FFBDE81040BE
:10954000FFF7BABF10B504460A2011F0D9FE204635
:1095500011F0F6FE11F0CAFE04464FF480510248A5
:1095600000F077FF204610BD0004024010B50C4605
:1095700011F0C6FE204611F0E3FE4FF4805103487F
:1095800000F067FFBDE8104010F08EB80004024004
:1095900010B511F0B5FE4FF48051034800F059FFAB
:1095A000BDE8104010F080B80004024070B50546D8
:1095B000012011F0A5FE11F099FE432828D22B209E
:1095C000FFF7C0FF102823D22F2011F099FE0020B2
:1095D00011F0B6FE3220FFF7DBFF142818D1CF20A0
:1095E000FFF7B0FF040013D04C20FFF79FFF00EB04
:1095F00004214C2000F042F85020FFF797FF00EBC9
:109600000421502000F03AF80021702000F036F8D4
:109610002F2011F075FE2C7806E015F8014F5C2C18
:1096200001D02F2C00D10024204611F089FE002CFF
:10963000F3D1BDE870404FF48051014800F009BFFC
:109640000004024070B505462D2011F059FE11F0BE
:109650004DFE0446260007D0287811F071FE641EE6
:109660006D1C14F0FF04F7D14FF48051024800F054
:10967000F0FE304670BD00000004024070B50546A3
:109680000C460D2011F03CFE284611F059FEE0B2C8
:1096900011F056FEC4F3072011F052FEC4F3074048
:1096A00011F04EFE200E11F04BFEBDE870404FF45D
:1096B0008051014800F0CDBE0004024070B5094D54
:1096C000FF22134605F5807605E010F8014B544063
:1096D0002A5D5A40335D491E89B2F6D242EA032020
:1096E00070BD00000DBB010870B500221346154681
:1096F00005E010F8014BA2186B41491E89B2002900
:10970000F7D1100C40EA034092B2801845EB1341A8
:109710004FEA014242EA104108186FEA000080B2A5
:1097200070BD08F047BD08F0E5BC08F0B3BC08F018
:1097300011BD00F0D1BF0CF091BF0000074A90426C
:1097400001D2074801E005481038064A8B0001EABB
:10975000020101D5C160704781607047106402400A
:10976000006002407D0F7D0F0029016802D041F0AA
:10977000010101E021F00101016070472DE9F04392
:10978000016821F0010101600021016041608160F8
:10979000C1600161212141613C493C4A3D251039AC
:1097A000904202D18D60BDE8F083384A4FF4746670
:1097B0001832904201D18E60F5E7344A4FF47417A5
:1097C0003032904201D18F60EDE7304A4FF0746C37
:1097D0004832904202D1C1F808C0E4E72B4B2C4A32
:1097E0006033984201D1CA60DDE7284C294B7834B8
:1097F000A04201D1CB60D6E7DFF89080264C08F17B
:109800009008404501D1CC60CDE7DFF880804FF073
:109810003D5908F1A808404502D1C1F80C90C2E7B3
:109820001E49DFF878800839404501D10D60BAE75C
:109830001A4D1835A84201D10E60B4E7174D3035E6
:10984000A84201D10F60AEE7144D4835A84202D1BD
:10985000C1F800C0A7E7114D10496035091FA842A3
:1098600001D10A609FE70D4A7832904201D10B6026
:1098700099E70A4A9032904201D10C6093E7074A77
:10988000A83290428FD1C1F800908CE7106002405E
:109890003D000020400F002000003D2010640240E9
:1098A0000B0607D5436912B143F0800301E023F0B2
:1098B00080034361802908D0002A026801F01E015C
:1098C00001D00A4300E08A430260704730B5036864
:1098D000124ACC6813400A682243D1E905452C435B
:1098E0002243CC6922430C6A22434C6A22438C6A8D
:1098F00022434C6B22438C6B22431A430260426921
:1099000022F00703D1E90B2422431A4342610A697A
:1099100042604A6882608968C16030BD3F801CF047
:109920002DE9FC41012120200DF0CEF901268DF812
:10993000046000258DF8065003208DF805001B4CAF
:10994000302700978DF807506946204600F02CFD1F
:109950003021204600F07DFD154C84F8305684F807
:10996000325684F8316684F833664FF4FA70C4F8DE
:10997000380600F01FF894F8A803802814D1A4F545
:1099800080504565232084F8AD03052084F8AC039E
:1099900084F8AB73142084F8AA03202084F8A90368
:1099A00084F8A85300F042F8BDE8FC81001402409E
:1099B000D42200207CB511F077FBD02011F044FBBD
:1099C00011F0A6FB002011F03FFB11F0A1FB11F0FC
:1099D0006BFBD12011F038FB11F09AFB00246D468F
:1099E00001E0062C01D2012000E0002011F0FCFA79
:1099F0002855641CE4B2072CF3D311F06FFB0A481E
:109A00009DF8061041719DF8051001719DF8041034
:109A1000C1709DF8021081709DF8011041709DF891
:109A2000001001707CBD00007C2600207CB5184829
:109A3000002401788DF8001041788DF801108178AC
:109A40008DF8021001218DF80310C1788DF80410F3
:109A500001798DF8051040798DF8060011F024FB8E
:109A6000D02011F0F1FA11F053FB002011F0ECFAC4
:109A700011F04EFB6D46285D11F0E6FA11F048FB3F
:109A8000641CE4B2072CF6D311F028FB7CBD000067
:109A90007C26002070B5094D0022134605F580761E
:109AA00005E010F8014B54402A5D5A40335D491ED1
:109AB00089B2F6D242EA032070BD00000DBB010856
:109AC000072A00D9072240EA002021B1012901D14B
:109AD000D040C0B270479040C0F307207047704735
:109AE000072A00D9072240EA002029B1012902D122
:109AF0009040C0F307207047D040C0B270470000CC
:109B000070B5ADF5327D00260D46ADF8BC62ADF8FE
:109B1000C06200EB4001324800EBC104608AA842F9
:109B20005CD9ADF8C06255E0012264212D4800F0F7
:109B3000BFF92C4800788DF80000382842D1228ADD
:109B4000E06802FB0501274800F0B2F9ADF8BC62FD
:109B50006A46208A0BE0BDF8BC326168C95CBDF87A
:109B6000BC32D154BDF8BC12491CADF8BC12BDF8D2
:109B7000BC128842EFD8401E81B2104600F05AFA5B
:109B8000228A0DF1FF31515C81421BD1ADF8BC62DC
:109B90000EE0BDF8BC226168895CA26800FB05206C
:109BA000BDF8BC221154BDF8BC02401CADF8BC028B
:109BB000208ABDF8BC12401E8842EADC01200DF567
:109BC000327D70BD642011F09BF9BDF8C002401CCD
:109BD000ADF8C002BDF8C0020628A5D30020EEE70C
:109BE00000B8010894550020F0B50E46074600EB7A
:109BF00047012648ADF5317D002500EBC1048DF805
:109C0000BC52608AB0423DD900210846FFF778FF78
:109C1000012837D1694609E0A268401E00FB0620F2
:109C20006268285C505548556D1CADB2208AA84228
:109C3000F2D80025208AE16800FB0611401E82B29E
:109C4000134800F0B3F9208A401E81B2684600F044
:109C5000F1F98DF8BC02208AE168012201447043C9
:109C6000401E0144AFA800F0A1F931463846FFF785
:109C700047FF012807D0642011F042F96D1CADB2F6
:109C8000062DD7D300200DF5317DF0BD00B80108B9
:109C9000945500202DE9F041ADF5307D354D4FF064
:109CA00000088DF8BC82344EA5F8008000243FE007
:109CB00000206F4607E056F832204968125C0A54CB
:109CC0003A54401C80B2298801EB410206EBC201E4
:109CD0000B8A5B1E8342EEDC288800EB400006EB1B
:109CE000C000008A401E81B2384600F0A3F98DF80A
:109CF000BC02288800EB400006EBC000C168008A67
:109D000000FB0411401E82B21C4800F04FF9288865
:109D1000012200EB400006EBC000C168008A01444C
:109D20006043401E0144AFA800F040F9641CA4B297
:109D3000288800EB400006EBC000408AA042B7D85C
:109D40002888401C80B228800A28AFD30C480178AC
:109D500021F001010170017841F006010170A0F8C5
:109D6000028000210120FFF73FFF0DF5307DBDE8A7
:109D7000F08100001000002000B801089455002078
:109D8000702400207CB5012108460CF09DFF0120C5
:109D90008DF8040002258DF8055000248DF806404A
:109DA0008DF807001820154E00906946304600F0E7
:109DB000FBFA05221146304600F032FB052206214F
:109DC000304600F02DFB05220721304600F028FB2D
:109DD000A02000908DF8045003208DF805008DF828
:109DE00006408DF807406946304600F0DDFA402015
:109DF00000906946304600F0D7FA7CBD0000024072
:109E0000F8B5002634460096FFF7BCFF00F0A0F836
:109E10002248641C8442FCD3214C0821204600F0D7
:109E200016FB1021204600F014FB062000F076F807
:109E30000821204600F00DFB0821204600F007FB1A
:109E40001021204600F005FB012000F067F80020FB
:109E500000F064F80821204600F0FBFA1148D0F821
:109E60001C0208B9FFF716FF0F4D2E800F4E00247D
:109E700005E0C0B22146FFF743FE641CA4B2288867
:109E800000EB400106EBC101498AA142F1D880B242
:109E9000401C80B228800A28E9D3F8BDFFFF0F00DC
:109EA00000000240000043421000002000B80108FA
:109EB0002DE9F0410546002416460F46012080F3A7
:109EC0001088DFF854800821404600F0C0FA1021C5
:109ED000404600F0BEFA032000F020F8C7F3074028
:109EE00000F01CF8C7F3072000F018F8F8B200F0F3
:109EF00015F806E0002000F011F8641C05F8010BCD
:109F0000A4B2B442F6D30821404600F0A2FA0020E1
:109F100080F31088BDE8F0810000024070B50B4C62
:109F20000546022120460DF099F80028F9D029466F
:109F300020460DF09CF8012120460DF08FF80028F6
:109F4000F9D020460DF091F8C0B270BD003001404C
:109F500010B5012186B008030CF0F2FE124C204629
:109F60000DF052F80021ADF808106015ADF80A00A8
:109F70003820ADF80C000720ADF80010ADF8100047
:109F8000ADF804104FF48270ADF80610ADF80E1065
:109F9000ADF80200694620460DF06BF8012120461D
:109FA0000DF028F806B010BD003001402DE9F04159
:109FB0000546002416460F46012080F31088DFF87E
:109FC00070800821404600F042FA1021404600F01F
:109FD00040FA0620FFF7A2FF0821404600F039FAB8
:109FE0000821404600F033FA1021404600F031FAD3
:109FF0000220FFF793FFC7F30740FFF78FFFC7F378
:10A000000720FFF78BFFF8B2FFF788FF05E02878FD
:10A01000FFF784FF641CA4B26D1CB442F7D308217F
:10A02000404600F016FA002080F31088BDE8F08169
:10A0300000000240027803E010F8013B1A44D2B25B
:10A04000491E89B2F8D210467047000070B51E4A0A
:10A05000907A012825D1002595721C491C480F24AF
:10A060004E780123F6B14D70D0F82852D0F8346202
:10A0700045EAC605D0F83062D0F82C02B60046EAB0
:10A0800040000543AC43CC708878CC78A04208D11E
:10A0900008710C78A04204D0D0710870002800D05C
:10A0A000937170BD4B70D0F82852D0F8346245EAF5
:10A0B000C605D0F83062D0F82C02B60046EA40005F
:10A0C0000543AC438C70DFE7D4120020C912002096
:10A0D000000042422DE9F041ADF57C7D00273D4670
:10A0E000ADF8E873FFF7AAF9142808D0664880F89D
:10A0F000A75311F041F80DF57C7DBDE8F081634870
:10A10000FFF7B4F9614C103C1428207006D04228A7
:10A1100079D00120FFF79DF92570ECE7FFF7B8F93A
:10A12000C4E90205A046BDF8E803FFF703F9FAAA5F
:10A130004FF4FA716846FFF71BF955A1684611F014
:10A140007FF8A080544C6E46F0B1E11901F58051C2
:10A1500081F8FD567F1CBFB2282FF6D34746304406
:10A160004EA111F06DF878800021001F0AE0BA8836
:10A170000A443244D378621802F5805282F8FD36E0
:10A18000491C89B28142F2DB45A1684611F058F8BA
:10A190004746A8F80400F0B10021621802F5805289
:10A1A00082F82557491C89B22829F6D330443BA1AF
:10A1B00011F046F87880002109380AE0BA880A448C
:10A1C0003244137A621802F5805282F82537491C0E
:10A1D00089B28142F2DB35A1684611F031F8B880CE
:10A1E000F8B10021621802F5805282F84D57491CDF
:10A1F00089B21429F6D3304428A111F021F87880CF
:10A2000000210D380BE03AE0BA880A443244137B4F
:10A21000621802F5805282F84D37491C89B281429A
:10A22000F2DB26A1684611F00BF8B880F0B10021EE
:10A23000621802F5805282F8B756491C89B2322959
:10A24000F6D3304415A110F0FBFF78800021C01F29
:10A250000AE0BA880A4432449379621802F58052BF
:10A2600082F8B736491C89B28142F2DB0021032013
:10A27000FFF7BAFC0120FFF7ECF801203BE70348A9
:10A28000FFF7EBF837E70000D42200203812002057
:10A2900041504E3D00000000D41200203B00000061
:10A2A000574946494E414D453D00000057494649F2
:10A2B00050415353574F52443D00000053455256AE
:10A2C00045523D002F4910B5884206D1012108466C
:10A2D0000CF006FD002101204FE02B49884206D1F9
:10A2E000012102200CF0FCFC0021022045E027495E
:10A2F000884206D1012104200CF0F2FC0021042048
:10A300003BE02349884206D1012108200CF0E8FCFB
:10A310000021082031E01F49884206D10121102088
:10A320000CF0DEFC0021102027E01B49884206D1FA
:10A33000012120200CF0D4FC002120201DE0174931
:10A34000884206D1012140200CF0CAFC00214020A7
:10A3500013E01349884206D1012180200CF0C0FC93
:10A360000021802009E00F4988420AD1841501218B
:10A3700020460CF0B5FC00212046BDE810400CF052
:10A38000AFBC10BD000002400004024000080240C3
:10A39000000C02400010024000140240001802406D
:10A3A000001C024000200240F0B5002201274FF0BF
:10A3B000030C0B6807FA02F52B40AB422CD1066860
:10A3C00053000CFA03F4A64306600E79D0F800E0BF
:10A3D0009E4046EA0E0606600E79012E01D0022E3E
:10A3E00012D18668A64386604E79D0F808E09E4078
:10A3F00046EA0E0686604668AE43466045688E793A
:10A400009640B6B235434560C568A543C560CC7972
:10A410009C40C3681C43C460521C102AC9D3F0BDC1
:10A420004B07DB0E9A40C90810B500EB8100016AAA
:10A430000F249C40A1430162016A1143016210BDD7
:10A440000246002012690A4200D001207047418371
:10A4500070470183704700002DE9F04F7C4E0025C6
:10A460002DED028B85B030782C46012852D14FF06B
:10A47000000986F8009006F1020898F80000DFF85D
:10A48000D4A14FF0010BF52804D098F819004F28FB
:10A490007DD080E098F8021098F8010041EA00248D
:10A4A0006B482146801CFFF709F908EB0401497845
:10A4B00018F8042041EA022181422BD198F80310B8
:10A4C000654FF1292BD06548F22953D0F32921D1CA
:10A4D0004C4680F8BC9280F8B0B2F520387087F80E
:10A4E00001900520B870F320F870592038710521CB
:10A4F0005948FFF7E3F8010A7971B87158480760C5
:10A500005749072008390860554801210C38FFF7E2
:10A510002BF9747005B0BDEC028BBDE8F08F52468C
:10A52000511901F5805181F8FD966D1CADB2282DB1
:10A53000F6D30020241F09E008EB00010B79111865
:10A5400001F5805181F8FD36401C80B2A042F3DB5A
:10A5500000210320FFF748FB0028DBD00CF0F6F9C0
:10A56000F52038704C4687F801900520B870F1202E
:10A57000BAE70CE080F8BCB280F8B1B2F5203870D0
:10A580004C4687F801900520B870F220ACE798F8A7
:10A590001A004B281CD02E4832A1801C10F050FE0F
:10A5A000060002D002218AF8021008EB0607B87BE9
:10A5B0002D4D41280FD0B87B5628ABD14846C5F861
:10A5C000AD9785F8B197C5F8AD9785F8B107A1E7C4
:10A5D0008AF802B09EE76946C146321902EB0900CB
:10A5E000027C0A55641C8846A4B24046092CF4D368
:10A5F0000FF09AF851EC100BFEF759F800EE100A24
:10A600009FED1A8A1A484A46C0EE080AC0EDEA0AC7
:10A61000B87E85F8AC0700204146331813441B7FF1
:10A620000B54401C80B20928F7D368460FF07CF821
:10A6300051EC100BFEF73BF800EE100AC0EE080AD2
:10A6400010EE900AC5F8AD0797F82700BDE70000A7
:10A6500012000020D4120020FC030020D45200205D
:10A66000AC640240524D4300D42200200000C84296
:10A67000D426002070B5144C40F2244631462046C2
:10A680000EF085FF00281ED0314620460EF01CFF3C
:10A690000E4D00212846FFF767F8314620460EF0A0
:10A6A00013FF0B492846FFF749F82088201D008832
:10A6B000291D4FF47A70086001212846FFF754F8ED
:10A6C00004490120087070BD001401402864024054
:10A6D000008800101200002010B5104C0E492046D2
:10A6E000FFF72CF800212046FFF73EF80C4C4021E4
:10A6F00020460EF045FF0028F9D0084C0949783C67
:10A700002046FFF71BF801212046FFF72DF80649E8
:10A710000120487010BD000000802020A06402408D
:10A720000014014000880010120000202DE9F043C1
:10A7300001218FB088050CF0C7FADFF88C904846ED
:10A74000FFF71CF84020050103900024CDE90545E2
:10A75000C60207940894CDE909461C4F0B944FF0AC
:10A760002068CDE900870C940D94694648460E9404
:10A77000FFF7ACF8012210214846FFF791F8DFF807
:10A780004890A9F178094846FEF7F8FF4FF47A702F
:10A79000CDE90340CDE9054507940894CDE9094684
:10A7A0000B480B940C940D94CDF800800E94CDE9D9
:10A7B000017069464846FFF789F801214846FEF7CF
:10A7C000D3FF0FB0BDE8F083A06402400414014041
:10A7D000140000207CB5012104200CF075FA164EFF
:10A7E000082206213046FFF71BFE082207213046CB
:10A7F000FFF716FE02218DF8051000258DF8065092
:10A800000124C0208DF8074000908DF8041069469F
:10A810003046FFF7C9FD600200908DF804408DF8C6
:10A82000065003208DF805008DF807406946304634
:10A83000FFF7BAFD7CBD0000000802402DE9F041A1
:10A84000FFF7C8FF4FF4E13000F078F8FFF76EFF34
:10A8500000F056F8244800250570857001214170EC
:10A86000C17042F210718160214E20483060204F4B
:10A870000E20083F3860A7F1040801214046FEF78A
:10A8800073FF1C4C657060780028FCD04FF4FA70A0
:10A8900010F036FB4FF4165000F050F8134900202A
:10A8A000154A103101EB000C135C401CC0B28CF84F
:10A8B00008300A28F6D3114A0020131803F58053F4
:10A8C00093F8F93601EB000C401CC0B28CF8133041
:10A8D0000428F2D331601920386001214046FEF788
:10A8E00043FF6570BDE8F081702A0020E407002076
:10A8F000AC6402401200002050B30108D4120020C2
:10A9000038B545208DF8000002208DF801000124A3
:10A910008DF802408DF80340684608F0C3F94720DF
:10A920008DF800008DF8014000208DF802008DF8B0
:10A930000340684608F0B6F938BD00001FB504466C
:10A94000012120200CF0FCF90020ADF80400009457
:10A95000ADF80600ADF80800ADF80C000C200D4C69
:10A96000ADF80A00694620460EF048FE0121204657
:10A970000EF0ADFD012240F2244120460EF026FEED
:10A98000102120460EF0A0FD0122C02120460EF02D
:10A99000A8FD1FBD001401400249C8790022CA71F8
:10A9A00070470000D412002002480068C00700D0A1
:10A9B00000BEFEE7F0ED00E002494AF6AA2008607A
:10A9C000704700000030004010B510F0D5FBBDE826
:10A9D0001040642010F094BA2DE9F04F83466AA02D
:10A9E000ADF57D7D002500689A460F46A946FB908F
:10A9F000ADF8E853042A25D8644C94F8AC03302110
:10AA000001EB101302EBC20000EB021260481618B3
:10AA1000337194F8AC0300F00F003030707194F88B
:10AA2000AB0301EB1010B07194F8AB0300F00F0012
:10AA30003030F071FEF702FD142807D084F8A79398
:10AA400010F09AFB0DF57D7DBDE8F08FDFF84081B9
:10AA5000A8F1240898F8000014280ED03046FEF71C
:10AA600005FD88F80000142807D042287ED0012078
:10AA7000FEF7EFFC88F80090E4E74FF47A70874225
:10AA800000D90746FEF704FDC8E902094E46FEF765
:10AA900051FC94F8AB13302000EB11118DF800102D
:10AAA00094F8AB1301F00F0130318DF8011094F8D8
:10AAB000AA1300EB11118DF8021094F8AA1301F0FB
:10AAC0000F0130318DF8031094F8A91300EB111128
:10AAD0008DF8041094F8A91301F00F0130318DF8AE
:10AAE000051094F8A81300EB11108DF8060094F8E7
:10AAF000A80300F00F0030308DF80700BAF1000F06
:10AB000003D0BAF1010F02D004E0542000E052203B
:10AB10008DF808003A208DF809000A236C4617E0EA
:10AB20000BEB550108780009B0FBF3F2C2EBC2024F
:10AB30001044621930309072087800F00F00B0FBBA
:10AB4000F3F1C1EBC10108443030AD1CD072ADB29D
:10AB5000B5EB470FE4D303EB470081B2FAAA2046D6
:10AB6000FEF738FCFAAA0221FBA800E007E0FEF796
:10AB700031FC0120FEF76DFC88F8006062E730468A
:10AB8000FEF76BFC5EE700000D0A0000D4220020F7
:10AB90004C1200202DE9F04F00262DED028BA3B0C2
:10ABA0008DF830608DF800608DF81060CDE9146686
:10ABB000CDE900668DF808608DF80C608DF8206096
:10ABC0008DF81460ADF818609FEDFE0A0796DFF867
:10ABD000F8938DED070AFD4C41F6B63504F12500DA
:10ABE0000A9004F59C5004F5804A01274FF0D50BDC
:10ABF000DFF8DC8304F580540990A0E094F8E60ABD
:10AC000028B384F8E66ABAF86C12D9F88C20484662
:10AC1000C2F57A7291421AD1D0F88C00C0F57A70E0
:10AC2000AAF86402E84800218830FEF79DFDE64856
:10AC3000E8498830FEF782FD88F800704FF47A709A
:10AC4000C9F88C00E04801218830FEF78DFD94F8AA
:10AC5000F20A20B384F8F26ABAF86E12D9F84420E6
:10AC60004846C2F57A72914219D1406CC0F57A70AB
:10AC7000AAF86602D44800214030FEF775FDD2489C
:10AC8000D5494030FEF75AFD88F801704FF47A70CC
:10AC9000C9F84400CC4801214030FEF765FD94F826
:10ACA000FE0A20B384F8FE6ABAF87012D9F81420AC
:10ACB0004846C2F57A72914219D14069C0F57A705E
:10ACC000AAF86802C04800211030FEF74DFDBE48CA
:10ACD000C2491030FEF732FD88F802704FF47A70E6
:10ACE000C9F81400B84801211030FEF73DFD94F872
:10ACF0000A0B20B384F80A6BBAF87212D9F82C2028
:10AD00004846C2F57A72914219D1C06AC0F57A708C
:10AD1000AAF86A02AC4800212830FEF725FDAA48AF
:10AD2000AF492830FEF70AFD88F803704FF47A70B7
:10AD3000C9F82C00A44801212830FEF715FD94F82D
:10AD4000E60A94F8F21A084494F8FE1A94F80A2BCA
:10AD50001144C8427FF452AF05F044BF017819B1E5
:10AD600006708DF8086010E0417819B146708DF8D2
:10AD700008700AE0817811B18670022003E0C17882
:10AD800019B1C67003208DF808009DF8080000EB8B
:10AD9000400101EB00118D4800EB011000F58050DF
:10ADA00090F88A1B9DF8080000EB4002C2EBC0122D
:10ADB0008C4810F83200C1280BD19DF8080000EB38
:10ADC0004002C2EBC012874800EBC200807808281E
:10ADD0000CD0082985F0D086DFE811F0C0202700CC
:10ADE0003F0ABD139D1B641DEC20E8248AF8BC7249
:10ADF0009DF8080030B1012807D002280FD00328A1
:10AE000008D10FE04FF4804101E04FF40051764843
:10AE1000FFF71DFB7548C0F8886205F0ADBE4FF422
:10AE20008051F4E74FF40061F1E79DF80800DFF886
:10AE3000B48100EB4001C1EBC01108EBC1004078C8
:10AE4000002107F059F88DF820008DF81060DFF828
:10AE50007C911BE09DF808009DF8101000EB40026B
:10AE600002EB001009EB001000EB011000F5805020
:10AE700090F8B50B9DF8201088429DF8100002D183
:10AE80008DF8200012E0401C8DF810009DF808009D
:10AE900000EB400101EB001009EB001000F58050C1
:10AEA00090F88B0B9DF810209042D3D89DF80800A5
:10AEB00000EB4001C1EBC01008EBC00080780A2213
:10AEC000B2EB101F9DF8080000EB4002C2EBC0106F
:10AED00008EBC000807801D100F00F008DF80C0065
:10AEE0009DF80C0010B910208DF80C009DF808009A
:10AEF0009DF80C1000EB4002C2EBC01208EBC20040
:10AF000008444078ADF818009DF8080000EB4001B7
:10AF1000C1EBC01108EBC1009DF80C10491C07F0F3
:10AF2000D0FB8DF800009DF8080000EB4001C1EB5C
:10AF3000C01108EBC1009DF80C10084480789DF802
:10AF40000010884245F018869DF80800424600EB44
:10AF50004001C1EBC01008EBC0004078002805F0AC
:10AF60000B869DF8080000EB4001C1EBC0109DF876
:10AF70000C1002EBC0000844C3789DF8080000EBF9
:10AF8000001101EB002109EBC10C9DF8201048468F
:10AF900001EB01110CEBC10101F5005181F8883082
:10AFA0009DF8081009EB01139DF82010194401F5D4
:10AFB000805181F8446B99F81410012937D19DF81C
:10AFC000081015E00000000000600240D4120020CC
:10AFD0001008002000880020008020102080001031
:10AFE00000880010E0620020001802400000424289
:10AFF00001EB410303EB01119DF8203000EB01113F
:10B0000001EB031129440B7843F080030B70BDF86A
:10B010001810B62905D0C52903D0D52901D0D929C2
:10B0200003D19DF80C10032901D2ADF81860BDF8CA
:10B030001810CE2913D013DCB9297DD009DC5A2988
:10B040008DD0B22979D0B529F7D0B62945F09485AD
:10B05000FDE3C32972D0C52971D0CA29F6D1F7E31F
:10B06000E129FCD006DCD52909D0D729E8D0D92997
:10B07000ECD182E2E5297CD0E729E7D1E9E39DF82C
:10B08000081001EB4103C3EBC11108EBC101C97802
:10B0900084F8A2119DF80810C84601EB410202EBAA
:10B0A0000112014600EB02109DF8202000EB021077
:10B0B00094F8A2212844A7EBD213027863F300028C
:10B0C00002709DF8080000EB400202EB00109DF8B2
:10B0D000202001EB001000EB021094F8A22128447C
:10B0E0005309027863F3410202709DF8080000EBF7
:10B0F000400202EB001001EB00129DF8200002EB71
:10B10000001000F5805090F8B60BC0F340029DF897
:10B11000080000EB001303EB002008EBC0019DF8D2
:10B12000200000EB001001EBC00000F5005090F88B
:10B130006400C0F3400003E0F2E3F2E3B8E3F1E3BC
:10B14000824252D09DF80800424600EB001101EB0C
:10B15000002008EBC0019DF8200000EB001001EB7F
:10B16000C00042F2640101449DF8080000EB400376
:10B1700000E0FDE303EB00109DF8203008EB001029
:10B1800000EB031000F5805090F8B60B43080878E8
:10B1900063F3410008709DF8080000EB400101EBEB
:10B1A00000109DF8201002EB001000EB011000F5DC
:10B1B000805090F8B60B800718D59DF80800D9216B
:10B1C00000EB001303EB002008EBC0029DF8200009
:10B1D00000EB001002EBC00000F5005080F85110A9
:10B1E0009DF808100220FEF7FFFC47E09DF80800DC
:10B1F00000EB001101EB002002EBC0019DF82000E4
:10B2000000EB001001EBC00000F5005080F8597011
:10B210009DF80800D92100EB001303EB002002EB9E
:10B22000C0039DF8200000EB001003EBC00000F508
:10B23000005080F851109DF8080000EB400101EB30
:10B24000001002EB00119DF8200001EB00104119E5
:10B25000087820F020030B709DF8080000EB001127
:10B2600001EB002008EBC0019DF8200000EB00106E
:10B2700001EBC00000F5005080F88A709DF80800CE
:10B28000434600EB400101EB001008EB00119DF874
:10B29000200001EB001000F5805090F8B60B00F094
:10B2A00001019DF8080000EB001202EB002008EB02
:10B2B000C0029DF8200000EB001002EBC00000F57A
:10B2C000005090F8640000F00100814204F0EC8529
:10B2D0009DF808009DF8202000EB001101EB0020F4
:10B2E000194603EBC00002EB021200EBC20042F26F
:10B2F000640210449DF8082002EB420303EB0212A3
:10B300009DF8203001EB021202EB031202F580528D
:10B3100092F8B62B037862F3000303709DF80800DF
:10B3200000EB400202EB00109DF8202001EB001022
:10B3300000EB021000F5805090F8B60BC0079DF8A6
:10B34000080039D000EB001202EB002001EBC00234
:10B350009DF8200000EB001002EBC00000F500504B
:10B3600090F88A0000289DF8080000EB001202EB1C
:10B37000002001EBC0029DF8200000EB001002EB62
:10B38000C00000F5005028D080F889609DF80800C2
:10B3900000EB400202EB001001EB00129DF82000D0
:10B3A00002EB00104219107820F00103137094F89A
:10B3B0006207A8B104F078BD00EB400202EB001078
:10B3C0009DF8202001EB001000EB021028440278C9
:10B3D00022F02003037004F09ABC80F88970E6E73D
:10B3E000487D0128E6D1486DCA8A9042E2D29DF894
:10B3F000080000EB001202EB002001EBC0029DF8F8
:10B40000200000EB001002EBC00000F5005090F8A7
:10B4100089000128CED19DF8080000EB001202EB54
:10B42000002001EBC0029DF8200000EB001002EBB1
:10B43000C00000F5005090F8C3000028BAD19DF874
:10B44000080000EB400202EB001001EB00129DF837
:10B45000200002EB001000F5805090F8B42B9DF80E
:10B46000080000EB001303EB002001EBC00000F527
:10B47000005080F845209DF80800C32200EB00131F
:10B4800003EB002001EBC0039DF8200000EB00104F
:10B4900003EBC00000F5005080F851209DF8080033
:10B4A00000EB400202EB001008EB00119DF82000B9
:10B4B00001EB001000F58050C0F8B86B9DF8081043
:10B4C0000220FEF791FB8DF83060414619E09DF8AF
:10B4D000080000EB001202EB002001EBC0029DF817
:10B4E000200000EB001002EBC0009DF8302010445B
:10B4F00000F5005080F88B609DF83000401C8DF8FE
:10B5000030009DF830001428E1D38DF8306019E048
:10B510009DF8080000EB001202EB002001EBC002D6
:10B520009DF8200000EB001002EBC0009DF83020D9
:10B53000104400F5005080F8A7609DF83000401CD2
:10B540008DF830009DF830000A28E1D332E79DF8ED
:10B55000080000EB001202EB002001EBC0029DF896
:10B56000200000EB001002EBC00000F5005090F846
:10B570004C00012804F0C1844FE49DF80810C8462F
:10B5800001EB410303EB011109EB011000F58050C1
:10B5900090F8900B00289DF80C0002D00A28EBD1FF
:10B5A00095E00828E8D18DF8306024E09DF8080087
:10B5B00000EB4001C1EBC0109DF8301002EBC00061
:10B5C0000844C07800F00F00092818D89DF808003A
:10B5D00000EB4001C1EBC0109DF8301002EBC00041
:10B5E0000844C07800F0F000902808D89DF830009A
:10B5F000401C8DF830009DF830000628D6D39DF809
:10B6000030000628B8D39DF8080000EB4001C1EBDC
:10B61000C01002EBC000C07801049DF8080000EBE8
:10B620004003C3EBC01002EBC000007941EA0023E5
:10B630009DF8080000EB4001C1EBC01002EBC00018
:10B64000407903439DF8080000EB001101EB002056
:10B6500008EBC00C9DF82000414600EB00100CEBFD
:10B66000C00000F50050C0F865309DF8080000EB00
:10B670004003C3EBC01002EBC000807903049DF8C7
:10B68000080000EB400CCCEBC01002EBC000C0790E
:10B6900043EA00239DF8080000EB400CCCEBC010FF
:10B6A00002EBC000007A03439DF8080000EB001293
:10B6B00002EB002001EBC0019DF8200000EB001020
:10B6C00001EBC00000F50050C0F86930A8E08DF82B
:10B6D000306024E09DF8080000EB4001C1EBC01091
:10B6E0009DF8301002EBC0000844C07800F00F0055
:10B6F000092818D89DF8080000EB4001C1EBC010E4
:10B700009DF8301002EBC0000844C07800F0F00053
:10B71000902808D89DF83000401C8DF830009DF826
:10B7200030000828D6D39DF830000828C5F02482C0
:10B730009DF8080000EB4001C1EBC01002EBC00017
:10B7400081799DF8080000EB4003C3EBC01002EBC9
:10B75000C000C07841EA00619DF8080000EB40039A
:10B76000C3EBC01002EBC000007903049DF8080091
:10B7700000EB400CCCEBC01002EBC000407943EA78
:10B78000002001439DF8080000EB001303EB0020AC
:10B7900008EBC0039DF8200000EB001003EBC00095
:10B7A00000F50050C0F865109DF8080000EB40015E
:10B7B000C1EBC01002EBC000817A9DF8080000EBDD
:10B7C0004003C3EBC01002EBC000C07941EA006146
:10B7D0009DF8080000EB4003C3EBC01002EBC00073
:10B7E000007A03049DF8080000EB400CCCEBC0107D
:10B7F00002EBC000407A43EA002001439DF80800B4
:10B8000000EB001202EB002008EBC0029DF82000C4
:10B8100000EB001002EBC00000F50050C0F869100A
:10B820009DF8080000EB001101EB002008EBC002BE
:10B830009DF82000414600EB001002EBC00000F52F
:10B84000005090F84C00032804F0FD8402E078E0FA
:10B85000FDE3FDE39DF8080000EB400202EB001061
:10B860009DF8202001EB001000EB021004F0E2BC78
:10B870009DF8080000EB001303EB002008EBC0016B
:10B8800004F07EBD9DF8080000EB001202EB0020E2
:10B8900001EBC0029DF8200000EB001002EBC0009D
:10B8A00000F5005090F85A00012804F0F38463E694
:10B8B0009DF8081001EB011303EB012100EBC1031C
:10B8C0009DF8201001EB011103EBC10101F50051BE
:10B8D00081F851B09DF8081001EB011202EB012133
:10B8E00000EBC10101F5005181F847709DF8081087
:10B8F00001EB410202EB011109EB01109DF8201050
:10B9000000EB01102844017841F02002F6E09DF898
:10B91000081001EB011303EB012109EBC101AFE7B3
:10B9200001E0C3E0ECE09DF8081001EB011202EB2E
:10B93000012100EBC10101F5005181F84760C322EC
:10B94000E5E79DF8081001EB410303EB011100EB63
:10B95000011101F5805191F8901B00299DF8081004
:10B9600001EB4103C3EBC11102EBC1015ED000E06A
:10B97000F0E3C9780B049DF8081001EB410CCCEB07
:10B98000C11102EBC101097943EA01239DF80810B6
:10B9900001EB410CCCEBC11108EBC10149790B4320
:10B9A0009DF8081001EB011202EB012100EBC1022E
:10B9B0009DF8201001EB011102EBC10101F50051CE
:10B9C000C1F880309DF8081001EB011202EB012153
:10B9D00000EBC1029DF8201001EB011102EBC10147
:10B9E00001F5005191F84C1002293ED09DF8081045
:10B9F000C52201EB011303EB012100EBC1039DF80C
:10BA0000201001EB011103EBC10101F5005181F898
:10BA100051209DF8081001EB011202EB012109EB06
:10BA2000C10000F5005080F84760A5E50B799DF84E
:10BA3000081001EB410CCCEBC11108EBC101C97836
:10BA400043EA01229DF8081001EB011303EB0121E9
:10BA500000EBC1039DF8201001EB011103EBC101C4
:10BA600001F50051C1F88020ACE79DF8081001EB0A
:10BA7000011202EB012100EBC10101F5005181F837
:10BA800047609DF80810032201EB011303EB01212D
:10BA900000EBC1039DF8201001EB011103EBC10184
:10BAA00001F5005181F84C20D9229BE39DF8081044
:10BAB00001EB011202EB012100EBC10101F5005184
:10BAC00081F847709DF8081001EB011303EB012189
:10BAD00000EBC1039DF8201001EB011103EBC10144
:10BAE00001F5005181F851B09DF8081001EB4102B9
:10BAF00002EB011109EB011004F01FBD02703BE5E0
:10BB00009DF80810CE4601EB410303EB011109EB50
:10BB1000011000F5805090F8900B00289DF80C0063
:10BB200002D00E28EBD19FE00C28E8D18DF83060D0
:10BB300024E09DF8081001EB4100C0EBC1109DF816
:10BB4000301002EBC0000844C07800F00F00092854
:10BB500018D89DF8081001EB4100C0EBC1109DF80A
:10BB6000301002EBC0000844C07800F0F0009028CC
:10BB700008D89DF83000401C8DF830009DF830004A
:10BB80000A28D6D39DF830000A28B8D30020CDE982
:10BB9000000030468DF830601FE0DDE900131B0225
:10BBA00043EA11630902CDE900139DF8081001EB87
:10BBB0004103C3EBC1119DF8303002EBC1011944C0
:10BBC000C978DDE9003C194340EA0C03CDE90013D4
:10BBD0009DF83010491C8DF830109DF83010052963
:10BBE000DBD3DDE9003C9DF8081001EB011808EB00
:10BBF00001210EEBC1099DF82010F04601EB011167
:10BC000009EBC10101F50059C9F86D304946C1F889
:10BC100071C00023CDE900338DF830001FE0DDE96D
:10BC200000131B0243EA11630902CDE900139DF8DA
:10BC3000081001EB4103C3EBC1119DF8303002EB5A
:10BC4000C1011944097ADDE9003C194340EA0C03BB
:10BC5000CDE900139DF83010491C8DF830109DF887
:10BC600030100529DBD39DE08DF8306024E09DF88D
:10BC7000081001EB4100C0EBC1109DF8301002EB41
:10BC8000C0000844C07800F00F00092818D89DF8BB
:10BC9000081001EB4100C0EBC1109DF8301002EB21
:10BCA000C0000844C07800F0F000902808D89DF843
:10BCB0003000401C8DF830009DF830000C28D6D3A1
:10BCC0009DF830000C28C4F057870020CDE9000013
:10BCD00030468DF830601FE0DDE900131B0243EAB7
:10BCE00011630902CDE900139DF8081001EB41032F
:10BCF000C3EBC1119DF8303002EBC1011944C97882
:10BD0000DDE9003C194340EA0C03CDE900139DF83E
:10BD10003010491C8DF830109DF830100629DBD307
:10BD2000DDE9003C9DF8081001EB011808EB01214A
:10BD30000EEBC1099DF82010F04601EB011109EB53
:10BD4000C10101F50059C9F86D304946C1F871C00B
:10BD50000023CDE900338DF830001FE0DDE900134A
:10BD60001B0243EA11630902CDE900139DF8081094
:10BD700001EB4103C3EBC1119DF8303002EBC1016F
:10BD80001944497ADDE9003C194340EA0C03CDE946
:10BD900000139DF83010491C8DF830109DF83010BC
:10BDA0000629DBD3DDE900129DF8080000EB001343
:10BDB00003EB002008EBC0039DF8200000EB00100F
:10BDC00003EBC00000F50053C3F875101846C0F827
:10BDD00079209DF80800F04600EB001101EB0020EF
:10BDE0000EEBC0029DF8200000EB001002EBC0003B
:10BDF00000F5005090F84C209DF8080000EB00136F
:10BE000003EB00200EEBC00000F5005090F8480056
:10BE100082427DD194F86207F0B39DF8080000EBF0
:10BE2000400101EB001108EB01109DF8201000EB20
:10BE300001102844017841F0080101709DF80810B4
:10BE40000220FDF7D1FE9DF820009DF8081000EBC0
:10BE50000110C117CDE9000100EB8001C1EB801199
:10BE600001EB0800C0F879609DF8081001EB0112A1
:10BE700002EB01229DF8201008EBC20201EB011138
:10BE800002EBC10142F26D02114410226930FCF74D
:10BE9000DCF99DF8080000E05EE000EB001101EB2A
:10BEA00000219DF8200008EBC10100EB001001EB20
:10BEB000C0010098653100EB8002C2EB801201F5F1
:10BEC000005102EB08000A6840F85D2F49684160A4
:10BED0009DF8081001EB410202EB011208EB021180
:10BEE0009DF8202001EB021101F5805191F8B41B5F
:10BEF00000F8011C09998A6A0262898D81849DF883
:10BF0000081001EB011202EB012208EBC20200E073
:10BF1000A4E09DF8201001EB011102EBC10101F535
:10BF20000051D1F8801081609DF8081001EB4102AA
:10BF300002EB011208EB02119DF8202001EB021127
:10BF400001F58051D1F8B81BC0F82610009881B2D5
:10BF50000820FDF749FE92E0C8F835609DF808001A
:10BF600000EB001101EB00219DF8200008EBC1015E
:10BF700000EB001001EBC00042F26D010144102201
:10BF80000A98FCF762F99DF8080000EB001101EB3C
:10BF900000219DF8200008EBC10100EB001001EB2F
:10BFA000C000653000F500504146026841F8192F85
:10BFB000406848609DF8080000EB400101EB00116B
:10BFC00008EB01109DF8201000EB011000F58050E7
:10BFD00090F8B41B88F8181009998A6AC8F83920B3
:10BFE000898DA8F83D109DF8080000EB001101EBC9
:10BFF00000219DF8200008EBC10100EB001001EBCF
:10C00000C00000F50050D0F88010C8F821109DF84D
:10C01000080000EB400101EB001108EB01109DF856
:10C02000201000EB011000F58050D0F8B81BC8F8C4
:10C030003F10D8F8540081B20220FCF7CBFF00215A
:10C040000620FDF7D1FDD8F85400401C01E082E045
:10C0500000E1C8F8540000210520F2E69DF8080030
:10C0600000EB400101EB001108EB01109DF82010DE
:10C0700000EB01102844017841F0040101709DF8A3
:10C08000080000EB001101EB002008EBC0029DF856
:10C090002000414600EB001002EBC00000F500500C
:10C0A00080F88A609DF8080000EB001303EB002085
:10C0B00008EBC0039DF8200000EB001003EBC0006C
:10C0C00000F5005080F851B09DF8080000EB001218
:10C0D00002EB002001EBC0029DF8200000EB0010F5
:10C0E00002EBC00000F5005090F84C00042844F02A
:10C0F00043859DF8080000EB400202EB00109DF81C
:10C10000202001EB001000EB02102844027842F0DE
:10C11000800303709DF8080000EB001202EB002082
:10C1200001EBC00000F5005080F847709DF8080052
:10C13000052300EB001202EB002008EBC0019DF884
:10C14000200000EB001001EBC00000F5005080F86B
:10C150004C306AE402E05A46FFF7D9BB84F8A07677
:10C160009DF8081001EB011202EB012100EBC10266
:10C170009DF8201001EB011102EBC10101F5005106
:10C1800091F84C1000299DF8081001EB011202EB08
:10C1900001210ED000EBC1029DF8201001EB01112E
:10C1A00002EBC10101F5005191F84E10B22928D0DF
:10C1B0003BE400EBC10101F5005181F847609DF8B7
:10C1C000081001EB011202EB012100EBC1029DF806
:10C1D000201001EB011102EBC10101F5005181F8C2
:10C1E0004C705A469DF8081001EB011303EB012136
:10C1F00009EBC10304F088BC00F5005080F8512021
:10C2000013E49DF8081001EB011202EB012100EB91
:10C21000C10101F5005181F847609DF80810B22274
:10C2200001EB011303EB012100EBC1039DF820108A
:10C2300001EB011103EBC10101F5005181F851201F
:10C240009DF8081001EB011202EB012109EBC1027C
:10C2500004F088BC84F8A0667DE79DF8080000EB38
:10C260004001C1EBC010FE4911F83000042809D08C
:10C270009DF8080000EB4002C2EBC01011F830003E
:10C28000152801D1ADF818009DF80800F44900EB1D
:10C290004002C2EBC01001EBC00042789DF80800DC
:10C2A00000EB4003C3EBC01011F8300042EA00205D
:10C2B000A0F58051303922D09DF8080000EB4001F4
:10C2C000C1EBC010E64901EBC00042789DF80800C0
:10C2D00000EB4003C3EBC01011F8300042EA00202D
:10C2E000A0F58052313A0CD09DF8080000EB4002D6
:10C2F000C2EBC01011F83000022804D019E0A620CB
:10C3000015E0A72013E09DF8080000EB4002C2EB07
:10C31000C01001EBC00002799DF8080000EB40035B
:10C32000C3EBC01001EBC000C07842EA0020ADF8BA
:10C3300018009DF80800DFF82C9300EB001101EBCA
:10C34000002109EBC10101F5005191F846108DF86B
:10C3500020109DF808109DF8202009EB01111144D0
:10C3600001F5805181F8446B99F81400012810D12F
:10C370009DF8080000EB400101EB001109EB0110F2
:10C380009DF8201000EB01102844017841F0800155
:10C390000170BDF8180043F23002811A904272D049
:10C3A00009DC042870D015286FD0A6280DD0A72846
:10C3B00044F0E28305E1B1F5C06F67D0A1F5C0613B
:10C3C000013979D00429F3D1FEE39DF8080000EB90
:10C3D000001101EB002009EBC00000F500504946B8
:10C3E00080F847609DF8080000EB001202EB002087
:10C3F00009EBC0029DF8200000EB001002EBC0002A
:10C4000000F5005090F84C00032840D09DF808003B
:10C4100000EB001202EB002001EBC0029DF82000AF
:10C4200000EB001002EBC00000F5005090F84C004B
:10C43000082842D09DF8080000EB001202EB002013
:10C4400001EBC0029DF8200000EB001002EBC000E1
:10C4500000F5005090F84C000D2843D09DF80800DE
:10C4600000EB001202EB002001EBC0029DF820005F
:10C4700000EB001002EBC00000F5005090F85100F6
:10C48000A52844D054E02CE18AE147E36CE39DF811
:10C490000800042200EB001303EB002001EBC003B3
:10C4A0009DF8200000EB001003EBC00000F50050E9
:10C4B00080F84C20A8228FE398E39DF80800092219
:10C4C00000EB001303EB002001EBC0039DF82000FC
:10C4D00000EB001003EBC00000F5005080F84C208A
:10C4E000A92279E39DF808000E2200EB001303EB6C
:10C4F000002001EBC0039DF8200000EB001003EBCF
:10C50000C00000F5005080F84C20A22264E39DF8A2
:10C51000080000EB400202EB00109DF8202001EB28
:10C52000001000EB02102844027842F0040202706E
:10C530009DF8080000EB001202EB002001EBC002A6
:10C540009DF8200000EB001002EBC00000F5005049
:10C5500090F84E00A12804F00F839DF8080000EB2E
:10C56000001202EB002001EBC0029DF8200000EB5E
:10C57000001002EBC00000F5005090F84E209DF82E
:10C58000080000EB001303EB002001EBC0039DF853
:10C59000200000EB001003EBC00000F5005080F815
:10C5A00051209DF80800A12200EB001303EB0020AE
:10C5B00009EBC0019DF8200000EB001001EBC0006A
:10C5C000FEE39DF8080000EB001101EB002009EBF1
:10C5D000C00000F50050494680F847609DF808000B
:10C5E00000EB001202EB002009EBC0029DF82000D6
:10C5F00000EB001002EBC00000F5005090F84C007A
:10C6000005289DF8080000EB001202EB00200ED078
:10C6100001EBC0029DF8200000EB001002EBC0000F
:10C6200000F5005090F84C00092808D020E001EBFC
:10C63000C00000F5005080F84760062200E00A22A2
:10C640009DF8080000EB001303EB002001EBC00392
:10C650009DF8200000EB001003EBC00004E0000098
:10C66000E0620020D412002000F5005080F84C2039
:10C670009DF8080000EB001202EB002001EBC00265
:10C680009DF8200000EB001002EBC00000F5005008
:10C6900090F85100A42822D19DF8080000EB400238
:10C6A00002EB00109DF8202001EB001000EB0210BF
:10C6B0002844027842F0200202709DF8080000EB46
:10C6C000001202EB002001EBC0029DF8200000EBFD
:10C6D000001002EBC00000F5005080F88960A12234
:10C6E0007AE28DF8306016A9FD4A13E09DF8080043
:10C6F00000EB4003C3EBC0109DF8303002EBC000EC
:10C700001844C0789DF83030C8549DF83000401C63
:10C710008DF830009DF830000628E7D3062116A8D2
:10C720000EF004FCCDE91406149B000AC018B046B4
:10C7300046EB08014FF480720023FBF743FD9DF8A0
:10C74000080000EB001101EB002009EBC0039DF88D
:10C75000200000EB001003EBC00000F5005080F853
:10C7600050209DF8080000EB001202EB002009EBBE
:10C77000C00000F5005080F847809DF8080000EBED
:10C78000001202EB002009EBC0029DF8200000EB34
:10C79000001002EBC00000F5005080F84C701AE267
:10C7A0009DF8080000EB001101EB002009EBC0022E
:10C7B0009DF82000494600EB001002EBC00000F598
:10C7C000005090F84C00062831D19DF8080000EB8D
:10C7D000001202EB002001EBC00000F5005080F8D1
:10C7E00047609DF80800072200EB001303EB0020D0
:10C7F00001EBC0039DF8200000EB001003EBC0002C
:10C8000000F5005080F84C209DF80800A72200EBAE
:10C81000001303EB002001EBC0039DF8200000EBA8
:10C82000001003EBC00000F5005080F851209DF887
:10C83000080000EB001202EB002001EBC0029DF8A3
:10C84000200000EB001002EBC00000F5005090F853
:10C850004C0001289DF8080000EB001202EB0020BC
:10C860005ED001EBC0029DF8200000EB001002EB4F
:10C87000C00000F5005090F84C0007289DF8080013
:10C8800000EB001202EB002052D001EBC0029DF839
:10C89000200000EB001002EBC00000F5005090F803
:10C8A0004C000B289DF8080000EB001202EB002062
:10C8B00059D001EBC0029DF8200000EB001002EB04
:10C8C000C00000F5005090F84C000C289DF80800BE
:10C8D00000EB001202EB00205FD001EBC0029DF8DC
:10C8E000200000EB001002EBC00000F5005090F8B3
:10C8F0004C000E2859D09DF8080000EB001202EB06
:10C90000002001EBC0029DF8200000EB001002EBBC
:10C91000C00000F5005090F84C000F287ED018E4BD
:10C9200001EBC00000F5005080F84760022206E0ED
:10C9300001EBC00000F5005080F8476008229DF828
:10C94000080000EB001303EB002001EBC0039DF88F
:10C95000200000EB001003EBC00000F5005080F851
:10C960004C20A32238E101EBC00000F5005080F814
:10C9700047609DF808000C2200EB001303EB002039
:10C9800001EBC0039DF8200000EB001003EBC0009A
:10C9900000F5005080F84C20A1E601EBC00000F546
:10C9A000005080F847600D22C9E79DF808000F226B
:10C9B00000EB001303EB002001EBC00C9DF82000FE
:10C9C00000EB00100CEBC00000F5005080F84C208C
:10C9D0009DF80800A12200EB001303EB002001EBFF
:10C9E000C00C9DF8200000EB00100CEBC00000F51F
:10C9F000005080F851209DF8080000EB001303EB75
:10CA0000002001EBC00C9DF8200000EB00100CEBA7
:10CA1000C00000F5005080F84E2000E019E09DF8BD
:10CA2000080000EB400202EB00109DF8202001EB13
:10CA3000001000EB02102844027842F080020270DD
:10CA40009DF8080000EB400202EB001009EB00101B
:10CA5000F2E39DF8080000EB001202EB002001EB6E
:10CA6000C0029DF8200000EB001002EBC00000F5B2
:10CA7000005090F84E00A12834D09DF80800A32261
:10CA800000EB001303EB00209DF8203001EBC00009
:10CA900003EB031300EBC30000F5005080F85120B6
:10CAA0009DF8080000EB001202EB002001EBC00231
:10CAB0009DF8200000EB001002EBC00000F50050D4
:10CAC00090F84E00A22804F057809DF8080000EB73
:10CAD000001202EB002009EBC000FEF7A2BF00002D
:10CAE000E06200209DF80800A12200EB001303EB98
:10CAF000002001EBC0039DF8200000EB001003EBC9
:10CB0000C00000F5005080F851209DF8080000EBAF
:10CB1000001202EB002009EBC000FDE39DF80800C5
:10CB2000A12200EB001101EB002009EBC0039DF8EE
:10CB3000200000EB001003EBC00000F5005080F86F
:10CB40004E209DF8080000EB001303EB002009EBDA
:10CB5000C0039DF8200000EB001003EBC00000F5BF
:10CB6000005080F85120B0E79DF8080000EB00115C
:10CB700001EB002009EBC0029DF82000494600EBC4
:10CB8000001002EBC00000F5005090F84C000628A1
:10CB900043F0F2879DF8080000EB001202EB002042
:10CBA00001EBC00000F5005080F847609DF80800D8
:10CBB000072200EB001303EB002001EBC0039DF8FC
:10CBC000200000EB001000E037E303EBC00000F5AD
:10CBD000005080F84C20A7229DF8080000EB0013BD
:10CBE00003EB002009EBC00103F0CABB9DF808006D
:10CBF00000EB001101EB002109EBC10101F500512F
:10CC0000484681F847609DF80810A72201EB011300
:10CC100003EB012109EBC1039DF8201001EB011189
:10CC200003EBC10101F5005181F851209DF8081076
:10CC3000DFF828CD01EB4102C2EBC1110CEBC101C1
:10CC4000497930299DF8081001EB410244D0C2EB2C
:10CC5000C1110CEBC101497931299DF808107CD034
:10CC600001EB4102C2EBC1110CEBC101497933293F
:10CC70009DF8081001EB410270D0C2EBC1110CEB22
:10CC8000C101497934299DF8081001EB410202EBFA
:10CC900001119DF8202000EB011101EB0211294444
:10CCA0000A7872D022F001020A709DF8081001EB98
:10CCB000410202EB011100EB01129DF8201002EB82
:10CCC00001114A19117821F0020313700021CDE9F6
:10CCD00000118DF83060DBE102EB01119DF820209E
:10CCE00000EB011101EB021129440A7822F0010244
:10CCF0000A709DF8081001EB410202EB01119DF84A
:10CD0000202000EB011101EB021129440A7822F0E6
:10CD100002030B709DF8081001EB011202EB0121D8
:10CD200000EBC1039DF8201001EB011103EBC101E1
:10CD300001F5005191F84F103129C7D19DF8081025
:10CD400001EB410202EB01119DF8202000EB0111E3
:10CD500001EB021129440A7801E017E02EE122F0EC
:10CD600020030B709DF8081001EB011202EB01216A
:10CD70009DF8202000EBC10102EB021201EBC20181
:10CD800001F5005181F88960A0E737E101EB01125C
:10CD900002EB012100EBC1029DF8201001EB011113
:10CDA00002EBC10101F5005191F88A1000299DF8AC
:10CDB000081001EB011202EB012100EBC10200E0BF
:10CDC000FDE39DF8201001EB011102EBC10101F51B
:10CDD00000517CD081F889609DF8081001EB410278
:10CDE00002EB011100EB01129DF8201002EB011182
:10CDF0004A19117821F0010313709DF8081001EB16
:10CE0000410202EB01119DF8202000EB011101EB22
:10CE1000021129440A7822F002020A7094F862177B
:10CE20000029B1D1417D0129AED1416DC28A914223
:10CE3000AAD29DF8081001EB011202EB012100EBD0
:10CE4000C1029DF8201001EB011102EBC10101F5B7
:10CE5000005191F88910012996D19DF8081001EB35
:10CE6000011202EB012100EBC1029DF8201001EB41
:10CE7000011102EBC10101F5005191F8C310002925
:10CE8000CFD19DF808104FF0104201EB011303EBD6
:10CE9000012100EBC1039DF8201001EB011103EB10
:10CEA000C10101F500514A659DF8081001EB4102EE
:10CEB00002EB011100EB01129DF8201002EB0111B1
:10CEC00001F5805191F8B42B9DF8081000E062E064
:10CED00001EB011303EB012100EBC10101F500514E
:10CEE00081F845209DF8081001EB011202EB0121A9
:10CEF00000EBC1029DF8201001EB011102EBC10112
:10CF000001F5005191F84C209DF8081001EB011338
:10CF100003EB012100EBC10101F5005191F848102C
:10CF20008A4299D19DF8081001EB011202EB012110
:10CF300000EBC1029DF8201001EB011102EBC101D1
:10CF400001F5005181F852609DF80810A42201EB10
:10CF5000011303EB012100EBC1039DF8201001EB4D
:10CF6000011103EBC10101F5005181F84E209DF83C
:10CF70000810A32201EB011303EB012100EBC10315
:10CF80009DF8201001EB011103EBC10101F50051E7
:10CF900081F851209AE681F889709DF8081001EB1C
:10CFA000410202EB011100EB01129DF8201002EB8F
:10CFB00001114A19117841F001031DE702EB01113B
:10CFC0009DF8202000EB011101EB021129440A78A1
:10CFD00042F001020A709DF8081001EB410202EBD9
:10CFE000011100EB01129DF8201002EB01114A190A
:10CFF000117841F002031370A22214E022F0200203
:10D000000A709DF8081001EB410202EB011100EBE0
:10D0100001129DF8201002EB01114A19117821F03C
:10D0200002031370A9229DF8081001EB011303EB12
:10D03000012100EBC1039DF8201001EB011103EB6E
:10D04000C10101F5005181F84E203FE6DDE90012F3
:10D05000120142EA11720901CDE900129DF808108F
:10D0600001EB4102C2EBC1119DF830200CEBC10174
:10D0700011448979DDE900383039CA17194342EA89
:10D080000802CDE900129DF83010491C8DF83010CF
:10D090009DF830100629D9D39DF80810009A01EBAD
:10D0A000011303EB012100EBC1039DF8201001EBFC
:10D0B000011103EBC10101F50051C1F86520002207
:10D0C000CDE900228DF8306021E0DDE90012120187
:10D0D00042EA11720901CDE900129DF8081001EB36
:10D0E0004102C2EBC1119DF830200CEBC10111448B
:10D0F000497BDDE900383039CA17194342EA080292
:10D10000CDE900129DF83010491C8DF830109DF8C3
:10D1100030100429D9D39DF80810009A01EB0113AF
:10D1200003EB012100EBC1039DF8201001EB01117D
:10D1300003EBC10101F50051C1F880200022CDE9C7
:10D1400000228DF8306021E0DDE90012120142EA90
:10D1500011720901CDE900129DF8081001EB41029E
:10D16000C2EBC1119DF830200CEBC1011144497C88
:10D17000DDE900383039CA17194342EA0802CDE91F
:10D1800000129DF83010491C8DF830109DF83010B9
:10D190000629D9D39DF80810009A01EB011303EB7F
:10D1A000012100EBC1039DF8201001EB011103EBFD
:10D1B000C10101F50051C1F869209DF8081001EB8B
:10D1C0004102C2EBC1110CEBC1014A799DF8081074
:10D1D00001EB011303EB012100EBC1039DF82010CB
:10D1E00001EB011103EBC10101F5005181F84F2062
:10D1F0009DF8081001EB410202EB011100EB011256
:10D200009DF8201002EB011101F5805191F8B62B29
:10D210009DF8081001EB011303EB012100EBC103A2
:10D220009DF8200000EB001003EBC00000F500505B
:10D2300080F8642003F0A0BCEFE39DF8080000EB49
:10D24000001101EB002009EBC00000F5005080F850
:10D2500047609DF8080000EB001202EB002009EB8C
:10D26000C0019DF8200000EB001001EBC00000F5AC
:10D27000005090F84C000A2879D09DF8080000EB87
:10D28000001101EB002009EBC0029DF82000494687
:10D2900000EB001002EBC00000F5005090F84C20AD
:10D2A0009DF8080000EB001303EB002009EBC00021
:10D2B00000F5005090F84800824213D194F86207BC
:10D2C00058B39DF808009DF8201000EB400202EBD7
:10D2D000001009EB001000EB01102844017841F028
:10D2E000080101709DF80800A72100EB001202EB75
:10D2F000002009EBC0029DF82000CC4600EB001096
:10D3000002EBC00000F5005080F851109DF80800B5
:10D31000A22100EB001201E0FCE33CE002EB002064
:10D3200009EBC0029DF8200000EB001002EBC000EA
:10D3300000F5005080F84E109DF8080000EB001139
:10D3400001EB00200CEBC0019DF8200000EB001069
:10D3500001EBC00000F5005080F88A600021CDE9A3
:10D3600000118DF83060DFF8F485A3E0FFE79DF849
:10D3700008000B2100EB001202EB00229DF82000B8
:10D3800009EBC20200EB001002EBC00000F50050F8
:10D3900080F84C10A6E7C846C1F835609DF8080033
:10D3A00000EB001101EB00219DF8200009EBC10109
:10D3B00000EB001001EBC00042F26D0101441022AD
:10D3C0000A98FAF742FF9DF8080000EB001101EB04
:10D3D00000219DF8200008EBC10100EB001001EBDB
:10D3E000C000653000F500504146026841F8192F31
:10D3F000406848609DF8080000EB400101EB001117
:10D4000008EB01109DF8201000EB011000F5805092
:10D4100090F8B41B88F818109DF8080000EB001174
:10D4200001EB00219DF8200008EBC10100EB00108A
:10D4300001EBC00000F50050D0F88010C8F82110B2
:10D44000099940468A6A40F8392F898D8180D8F839
:10D45000540081B20220FBF7BDFD00210620FCF73D
:10D46000C3FBD8F85410491CC8F8541000210520FB
:10D47000FCF7BAFB36E7090141EA10710001CDE97A
:10D4800000019DF8080000EB4001C1EBC0109DF8C1
:10D49000301008EBC0000844C07ADDE900233038C2
:10D4A000C11710431943CDE900019DF83000401C1D
:10D4B0008DF830009DF830000A28DDE90001DAD34C
:10D4C0009DF8082002EB021303EB02220CEBC203CF
:10D4D0009DF8202002EB021203EBC20202F500537A
:10D4E000C3F86D001A46C2F871100020CDE90000A3
:10D4F0008DF8306020E0DDE90001090141EA10719A
:10D500000001CDE900019DF8080000EB4001C1EBEE
:10D51000C0109DF8301008EBC0000844407DDDE9E4
:10D5200000233038C11710431943CDE900019DF89D
:10D530003000401C8DF830009DF830000A28DAD306
:10D54000DDE900129DF8080000EB001303EB00205A
:10D550000CEBC003FDE39DF8080000EB4001C1EBBC
:10D56000C010FE4911F83000042809D09DF80800C9
:10D5700000EB4002C2EBC01011F83000152801D1B9
:10D58000ADF818009DF80800894600EB4002C2EB98
:10D59000C01001EBC00042789DF8080000EB40038A
:10D5A000C3EBC01011F8300042EA0020A0F5805112
:10D5B000303924D09DF8080000EB400100E082E102
:10D5C000C1EBC01009EBC000494642789DF8080045
:10D5D00000EB4003C3EBC01019F8300042EA002012
:10D5E000A0F58052313A0CD09DF8080000EB4002C3
:10D5F000C2EBC01011F83000022804D019E0A620B8
:10D6000015E0A72013E09DF8080000EB4002C2EBF4
:10D61000C01001EBC00002799DF8080000EB400348
:10D62000C3EBC01009EBC000C07842EA0020ADF89F
:10D6300018009DF8080000EB001101EB0021C8481C
:10D6400000EBC10101F5005191F846208DF8202032
:10D650009DF8081000EB01129DF82010114401F50F
:10D66000805181F8446B017D012910D19DF808108B
:10D6700001EB410202EB01119DF8202000EB0111AA
:10D6800001EB021129440A7842F080020A70BDF8C9
:10D690001810A7297DD007DC04297BD015297AD062
:10D6A000A62943F069823DE001F51D61B1F5804195
:10D6B00004D0112970D01229F3D1FDE39DF8081090
:10D6C00001EB011202EB012100EBC1029DF82010D9
:10D6D00001EB011102EBC10101F5005191F84C1071
:10D6E0000029DED19DF8081001EB011202EB0121A7
:10D6F00000EBC10101F5005181F847609DF8081069
:10D7000001EB011202EB012100EBC1029DF8201098
:10D7100001EB011102EBC10101F5005181F84C70E0
:10D72000A7229DE19DF8081001EB011202EB0121F7
:10D7300000EBC10101F5005181F847609DF8081028
:10D7400001EB011202EB012100EBC1029DF8201058
:10D7500001EB011102EBC10101F5005191F84C10F0
:10D7600002292DD09DF8081001EB011202EB0121D6
:10D7700000EBC1029DF8201001EB011102EBC10189
:10D7800001F5005191F84C1005292ED09DF8081094
:10D7900003E09DE0F0E023E248E201EB011202EB3E
:10D7A000012100EBC1029DF8201001EB011102EBF9
:10D7B000C10101F5005191F85110A5292AD03AE094
:10D7C0009DF80810032201EB011303EB012100EB8C
:10D7D000C1039DF8201001EB011103EBC10101F51C
:10D7E000005181F84C20A9223AE19DF80810062248
:10D7F00001EB011303EB012100EBC1039DF82010A5
:10D8000001EB011103EBC10101F5005181F84C203E
:10D81000A22225E19DF8081001EB410202EB011163
:10D820009DF8202000EB011101EB021129440A7838
:10D8300042F004020A709DF8081001EB011202EB9D
:10D84000012100EBC1029DF8201001EB011102EB58
:10D85000C10101F5005191F84E10A12903F08C810E
:10D860009DF8081001EB011202EB012100EBC1024F
:10D870009DF8201001EB011102EBC10101F50051EF
:10D8800091F84E209DF8081001EB011303EB0121E4
:10D8900000EBC1039DF8201001EB011103EBC10166
:10D8A00001F5005181F851209DF80810A12201EBEB
:10D8B000011303EB012100EBC1039DF8200000EBF5
:10D8C000001003EBC00000F5005080F84E20B1E4DA
:10D8D0009DF8081001EB011202EB012100EBC102DF
:10D8E0009DF8201001EB011102EBC10101F500517F
:10D8F00091F85110A42922D19DF8081001EB4102A2
:10D9000002EB01119DF8202000EB011101EB021147
:10D9100029440A7842F020020A709DF8081001EBB1
:10D92000011202EB012100EBC1029DF8201001EB76
:10D93000011102EBC10101F5005181F889609DF8E8
:10D94000081001EB011202EB012100EBC10101F50E
:10D95000005181F84760A12204E00000E06200204D
:10D96000D41200209DF8081001EB011303EB0121F4
:10D9700000EBC10102F004BD9DF8081001EB01129B
:10D9800002EB012100EBC1029DF8201001EB011117
:10D9900002EBC10101F5005191F84C1001299DF8ED
:10D9A000081001EB011202EB012137D000EBC1029C
:10D9B0009DF8201001EB011102EBC10101F50051AE
:10D9C00091F84C1004299DF8081001EB011202EBAC
:10D9D00001212BD000EBC1029DF8201001EB0111B9
:10D9E00002EBC10101F5005191F84C1006299DF898
:10D9F000081001EB011202EB01213BD000EBC10248
:10DA00009DF8201001EB011102EBC10101F500515D
:10DA100091F84C1007297ED00CE470E000EBC101B6
:10DA200001F5005181F84760022206E000EBC101D8
:10DA300001F5005181F8476005229DF8081001EBBF
:10DA4000011303EB012100EBC1039DF8201001EB52
:10DA5000011103EBC10101F5005181F84C20A32213
:10DA60009DF8081001EB011303EB012100EBC1034A
:10DA700003F04AB800EBC10101F5005181F847609D
:10DA80009DF80810072301EB011202EB012100EBC6
:10DA9000C10C9DF8201001EB01110CEBC10101F547
:10DAA000005181F84C309DF80810A12301EB0112C0
:10DAB00002EB012100EBC10C9DF8201001EB0111DC
:10DAC0000CEBC10101F5005181F851309DF80810AF
:10DAD00001EB410202EB01119DF8202000EB011146
:10DAE00001EB021129440A7842F080030B709DF883
:10DAF000081001EB410202EB011100EB01109DF84F
:10DB0000201000EB01102844017841F0040101705D
:10DB1000DDE600E05FE09DF8081001EB011202EB8A
:10DB2000012100EBC1029DF8201001EB011102EB75
:10DB3000C10101F5005191F84E10A12930D09DF896
:10DB40000810A32201EB011303EB01219DF8203003
:10DB500000EBC10103EB031301EBC30101F500511D
:10DB600081F851209DF8081001EB011202EB012110
:10DB700000EBC1029DF8201001EB011102EBC10185
:10DB800001F5005191F84E10A229C1D09DF808105E
:10DB900001EB011202EB012100EBC100FDF741BFD7
:10DBA0009DF80810A12201EB011303EB012100EB0A
:10DBB000C1039DF8201001EB011103EBC10101F538
:10DBC000005181F851209DF8081001EB011202EB81
:10DBD000012100EBC10000F5005080F8477076E6A7
:10DBE0009DF80810A12201EB011303EB012100EBCA
:10DBF000C1039DF8201001EB011103EBC10101F5F8
:10DC0000005181F851209DF8081001EB011303EB3E
:10DC1000012100EBC1039DF8201001EB011103EB82
:10DC2000C10101F5005181F84E20AFE79DF80810C1
:10DC300001EB011202EB012100EBC10101F50051E2
:10DC400081F847609DF80810A72201EB011303EB50
:10DC5000012100EBC1039DF8201001EB011103EB42
:10DC6000C10101F5005181F851209DF80810CC4602
:10DC700001EB4102C2EBC11109EBC1014979302925
:10DC80009DF8081001EB41024FD0C2EBC1110CEB23
:10DC9000C101497931299DF808107DD001EB41027D
:10DCA000C2EBC1110CEBC101497933299DF8081071
:10DCB00001EB410271D0C2EBC1110CEBC1014979FA
:10DCC00034299DF8081001EB410267D0C2EBC11165
:10DCD0000CEBC1014979352970D09DF8081001EB92
:10DCE000410202EB01119DF8202000EB011101EB34
:10DCF000021129440A7822F001020A709DF80810E6
:10DD000001EB410202EB011100EB01129DF8201022
:10DD100002EB01114A19117821F00203137000215E
:10DD2000CDE900118DF83060D8E102EB01119DF8CA
:10DD3000202000EB011101EB021129440A7822F0A6
:10DD400001020A709DF8081001EB410202EB01117B
:10DD500000E0D1E39DF8202000EB011101EB02115E
:10DD600029440A7822F002030B709DF8081001EB99
:10DD7000011202EB012100EBC1039DF8201001EB21
:10DD8000011103EBC10101F5005191F84F10312948
:10DD9000C5D19DF8081002E011E029E148E101EB4E
:10DDA000410202EB011100EB01129DF8201002EB81
:10DDB00001114A19117821F02003AFE758E101EB76
:10DDC000011202EB012100EBC1029DF8201001EBD2
:10DDD000011102EBC10101F5005191F88A100029EF
:10DDE0009DF8081001EB011202EB012100EBC102CA
:10DDF0009DF8201001EB011102EBC10101F500516A
:10DE00007DD081F889609DF8081001EB410202EB9A
:10DE1000011100EB01129DF8201002EB01114A19CB
:10DE2000117821F0010313709DF8081001EB4102F5
:10DE300002EB01119DF8202000EB011101EB021112
:10DE400029440A7822F002020A7094F86217002925
:10DE50009ED1417D01299BD1416DC28A9142BFF47F
:10DE60005EAF9DF8081001EB011202EB012100EBFF
:10DE7000C1029DF8201001EB011102EBC10101F577
:10DE8000005191F889100129E2D19DF8081001EBA9
:10DE9000011202EB012100EBC1029DF8201001EB01
:10DEA000011102EBC10101F5005191F8C3100029E5
:10DEB000CED14FF0104200E094E19DF8081001EB44
:10DEC000011303EB012100EBC1039DF8201001EBCE
:10DED000011103EBC10101F500514A659DF80810DD
:10DEE00001EB410202EB011100EB01129DF8201041
:10DEF00002EB011101F5805191F8B42B00E064E0D0
:10DF00009DF8081001EB011303EB012100EBC101A7
:10DF100001F5005181F845209DF8081001EB011230
:10DF200002EB012100EBC1029DF8201001EB011171
:10DF300002EBC10101F5005191F84C209DF8081049
:10DF400001EB011303EB012100EBC10101F50051CD
:10DF500091F848108A4297D19DF8081001EB011200
:10DF600002EB012100EBC1029DF8201001EB011131
:10DF700002EBC10101F5005181F852609DF80810D3
:10DF8000A42201EB011303EB012100EBC1039DF877
:10DF9000201001EB011103EBC10101F5005181F8E3
:10DFA0004E209DF80810A32201EB011303EB012181
:10DFB00000EBC1039DF8201001EB011103EBC1013F
:10DFC00001F5005181F85120A9E681F889709DF88A
:10DFD000081001EB410202EB011100EB01129DF868
:10DFE000201002EB01114A19117841F001031AE7E0
:10DFF00002EB01119DF8202000EB011101EB021151
:10E0000029440A7842F001020A709DF8081001EBD9
:10E01000410202EB011100EB01129DF8201002EB0E
:10E0200001114A19117841F002031370A22220E075
:10E0300002EB01119DF8202000EB011101EB021110
:10E0400029440A7822F020020A709DF8081001EB9A
:10E05000410202EB011100EB01129DF8201002EBCE
:10E0600001114A19117821F002031370A92200E06E
:10E07000A1229DF8081001EB011303EB012100EB35
:10E08000C1039DF8201001EB011103EBC10101F563
:10E09000005181F84E2042E6DDE90012120142EA09
:10E0A00011720901CDE900129DF8081001EB41023F
:10E0B000C2EBC1119DF830200CEBC10111448979EC
:10E0C000DDE900383039CA17194342EA0802CDE9C0
:10E0D00000129DF83010491C8DF830109DF830105A
:10E0E0000829D9D39DF80810009A01EB011303EB1E
:10E0F000012100EBC1039DF8201001EB011103EB9E
:10E10000C10101F50051C1F865200022CDE90022CE
:10E110008DF8306021E0DDE90012120142EA11724F
:10E120000901CDE900129DF8081001EB4102C2EB94
:10E13000C1119DF830200CEBC1011144C97BDDE910
:10E1400000383039CA17194342EA0802CDE90012F3
:10E150009DF83010491C8DF830109DF830100629BC
:10E16000D9D39DF80810009A01EB011303EB0121AC
:10E1700000EBC1039DF8201001EB011103EBC1017D
:10E1800001F50051C1F880200022CDE900228DF870
:10E19000306021E0DDE90012120142EA117209014A
:10E1A000CDE900129DF8081001EB4102C2EBC1114C
:10E1B0009DF830200CEBC1011144497DDDE90038A8
:10E1C0003039CA17194342EA0802CDE900129DF816
:10E1D0003010491C8DF830109DF830100829D9D323
:10E1E000FEF7D8BF9DF80810804601EB011202EB44
:10E1F000012200EBC20000F5005080F847609DF856
:10E20000080000EB001202EB002008EBC0019DF8B3
:10E21000200000EB001001EBC00000F5005090F86A
:10E220004C00032876D09DF8080000EB001101EBAC
:10E23000002008EBC0029DF82000414600EB0010D2
:10E2400002EBC00000F5005090F84C209DF808004B
:10E2500000EB001303EB002008EBC00000F50050BA
:10E2600090F84800824213D194F86207E8B39DF811
:10E2700008009DF8201000EB400202EB001008EBB4
:10E28000001000EB01102844017841F008010170F2
:10E290009DF8080000EB001101EB002008EBC00125
:10E2A0009DF8200000EB001001EBC00000F50050CD
:10E2B00080F88A609DF80800A72100EB001202EBAD
:10E2C000002008EBC0029DF8200000EB001002EBDC
:10E2D000C00000F5005080F851109DF80800A22100
:10E2E00000EB001202EB002000E027E008EBC00288
:10E2F0009DF8200000EB001002EBC00000F500507C
:10E3000080F84E100021CDE900118DF83060CC4628
:10E31000A2E0FFE79DF80800042100EB001202EBE9
:10E3200000229DF8200008EBC20200EB001002EB77
:10E33000C00000F5005080F84C10A9E7C1F8356026
:10E340009DF8080000EB001101EB00219DF8200072
:10E3500008EBC10100EB001001EBC00042F26D01BF
:10E36000014410220A98F9F770FF9DF8080000EBAD
:10E37000001101EB00219DF8200008EBC10100EB2A
:10E38000001001EBC000653000F500504146026806
:10E3900041F8192F406848609DF8080000EB4001E3
:10E3A00001EB001108EB01109DF8201000EB0110AB
:10E3B00000F5805090F8B41B88F818109DF80800FC
:10E3C00000EB001101EB00219DF8200008EBC101DA
:10E3D00000EB001001EBC00000F50050D0F88010F9
:10E3E000C8F82110099940468A6A40F8392F898D6A
:10E3F0008180D8F8540081B20220FAF7EBFD0021A9
:10E400000620FBF7F1FBD8F85400401CC8F8540074
:10E4100000210520FBF7E8FB3AE7090141EA10710A
:10E420000001CDE900019DF8080000EB4001C1EBBF
:10E43000C0109DF830100CEBC0000844C07ADDE934
:10E4400000233038C11710431943CDE900019DF86E
:10E450003000401C8DF830009DF830000C28DDE9BC
:10E460000001DAD39DF8082002EB021303EB02222D
:10E4700008EBC2039DF8202002EB021203EBC2025C
:10E4800002F50053C3F86D001A46C2F8711000205F
:10E49000CDE9000001468DF830601FE000980901C9
:10E4A00041EA10710001CDE900019DF8080000EB80
:10E4B0004001C1EBC0109DF830100CEBC0000844C7
:10E4C000C07DDDE900233038C11710431943CDE981
:10E4D00000019DF83000401C8DF830009DF83000A0
:10E4E0000C28DBD3DDE900129DF8080000EB0013D7
:10E4F00003EB002008EBC0039DF8200000EB0010A8
:10E5000003EBC00000F50053C3F875101846C0F8BF
:10E51000792002F031BBFE4B9DF808009DF82010D9
:10E5200003EB0010084400F5805080F8446B9DF820
:10E530000800DFF8E08300EB4001C1EBC01008EBFE
:10E54000C000407870280AD19DF8080000EB400117
:10E55000C1EBC01008EBC0008078FA282DD09DF8E0
:10E56000080000EB4001C1EBC01008EBC000407890
:10E570009DF8080000EB4001C1EBC01018F8300016
:10E580009DF8080000EB001101EB002003EBC00038
:10E5900000F5005090F846008DF820009DF8080026
:10E5A0009DF8201003EB0010084400F5805080F81F
:10E5B000446B187D012804D014E0B120ADF8180098
:10E5C000DEE79DF8080000EB400101EB00109DF82C
:10E5D000201003EB001000EB01102844017841F0FB
:10E5E00080010170BDF8180001284BD065287DD04E
:10E5F000B1288ED0B6288CD19DF8080000EB001110
:10E6000001EB002003EBC0019DF8200000EB00109F
:10E6100001EBC00000F5005090F84C000128EAD151
:10E620009DF8080000EB001101EB002003EBC00097
:10E6300000F5005080F847609DF8080000EB0011DD
:10E6400001EB002003EBC0019DF8200000EB00105F
:10E6500001EBC00000F5005080F84C709DF80800F8
:10E66000B12100EB001202EB002003EBC0029DF889
:10E67000200000EB001002EBC00000F5005080F815
:10E68000511046E79DF8080000EB4001C1EBC010B7
:10E6900008EBC00000790128F3D00228F1D003284C
:10E6A000EFD00528EDD19DF8080000EB001101EB3B
:10E6B000002003EBC0019DF8200000EB001001EBEF
:10E6C000C00000F5005090F84C000028D9D19DF80A
:10E6D000080000EB001101EB002003EBC00000F587
:10E6E000005080F847609DF8080000E036E000EB3D
:10E6F000001101EB002003EBC0019DF8200000EBAE
:10E70000001001EBC00000F5005080F84C709DF83F
:10E710000800B62100EB001202EB002003EBC00260
:10E720009DF8200000EB001002EBC00000F5005047
:10E7300080F851109DF80800B22100EB001202EBA6
:10E74000002003EBC0029DF8200000EB001002EB5C
:10E75000C00000F5005080F84E10DAE69DF8080081
:10E7600000EB4001C1EBC01008EBC0000079B922FA
:10E77000ADF818209DF8080000EB4001C1EBC01077
:10E7800008EBC000007900F00F018DF814108DF82F
:10E7900030601FE09DF8080000EB400101EB001025
:10E7A00003EB00119DF8300001EB001000F58050E4
:10E7B00090F8B51B9DF8080000EB400CCCEBC010A6
:10E7C00018F830005038814214D09DF83000401CB9
:10E7D0008DF830009DF8080000EB400101EB0010BF
:10E7E00003EB001000F5805090F88B0B9DF8301073
:10E7F0008842CFD89DF830009DF8141008448DF859
:10E8000020009DF8080000EB001101EB002003EB55
:10E81000C00C9DF8200000EB00100CEBC00000F5D0
:10E82000005090F84C00012814D09DF8080000EB2F
:10E83000001101EB002003EBC0019DF8200000EB6C
:10E84000001001EBC00000F5005090F84C000128CA
:10E8500042F092819DF8080000EB001101EB0020CE
:10E8600003EBC00000F5005080F847609DF80800F9
:10E87000022100EB001C0CEB002003EBC00C9DF808
:10E88000200000EB00100CEBC00000F5005080F8F9
:10E890004C109DF8080000EB001101EB002003EB89
:10E8A000C001F9E39DF8080000EB400101EB001105
:10E8B000174800EB011000F5805090F8900B20B144
:10E8C000012871D00228C3D19CE2DFF844909DF862
:10E8D000081009EB410000F58040B0F86402801F89
:10E8E00081B29DF80800DFF82C8000EB4002C2EBFB
:10E8F000C01208EBC200401CFAF7F6FECDE9140680
:10E900009DF8081009EB410000F5804004E000008C
:10E91000D4120020E0620020B0F864129DF80800D4
:10E9200001EB080200EB4001C1EBC0106FF00401E5
:10E9300001EBC0001044042108F0AAFCC117CDE986
:10E940000001DDE91423504059400843BBD19DF834
:10E95000080009EB001000F5805080F8446B9DF82A
:10E96000080000EB4002C2EBC012404600EBC200C0
:10E970000079ADF81800BDF818003128A3D19DF832
:10E98000081009EB410000F58040B0F86402412115
:10E99000183890FBF1F0C117CDE9000184F8440567
:10E9A0008DF83060B046CCE0D5E09DF8080000EB73
:10E9B0004001C1EBC011FE4800EBC1019DF83000E1
:10E9C00000EB80100844017D9DF8302009EB020027
:10E9D00000F5805080F845159DF8080000EB4001D7
:10E9E000C1EBC011F24800EBC1019DF8300000EB13
:10E9F0008010084408211A3008F016FC8DED070A33
:10EA000010EE100A9DF8302009EB021101F580513B
:10EA1000C1F855059DF8080000EB4001C1EBC0119D
:10EA2000E34800EBC1019DF8300000EB8010084482
:10EA30000821323008F0F8FB8DED070A10EE100ABD
:10EA40009DF8302009EB021101F58051C1F8510504
:10EA50009DF8080000EB4001C1EBC011D44800EB69
:10EA6000C1019DF8300000EB8010084408213A30C5
:10EA700008F0DAFB8DED070A10EE100A9DF8302041
:10EA800009EB021101F58051C1F859059DF8080004
:10EA900000EB4001C1EBC011C54800EBC1019DF87E
:10EAA000300000EB801008440821423008F0BCFB25
:10EAB0008DED070A10EE100A9DF8302009EB0211C7
:10EAC00001F58051C1F85D059DF8080000EB40019B
:10EAD00001EB001109EB01109DF8301000EB011063
:10EAE0002844017841F0800101709DF8081009EB7D
:10EAF000410000F58040B0F86412AD4801449DF833
:10EB0000080000EB4002C2EBC0104FF0FF3202EBF6
:10EB1000C000095C9DF8080000EB001202EB002227
:10EB20009DF8200009EBC20300EB001003EBC000CE
:10EB300000F5005080F888109DF83000401C8DF8DA
:10EB400030009DF83000DDE90012401A78EB020039
:10EB5000FFF62BAFDDE49DF80800DFF8548200EBF0
:10EB60004001C1EBC01008EBC000437D9DF80800D8
:10EB700000EB4002C2EBC01008EBC000807D43EA0E
:10EB80000020C317CDE900039DF80800152100EB14
:10EB90004002C2EBC01008EBC000FAF78FFDCDE9D0
:10EBA0001406DDE90003DDF850C0734080EA0C0074
:10EBB0001843CFD19DF8080000EB4001C1EBC01114
:10EBC000404618F83120521E8DF82020DFF8E491DD
:10EBD0009DF808104A4609EB01139DF820101944CE
:10EBE00001F5805181F8446B9DF82010494401F5EE
:10EBF000805181F845659DF8201009EB011101F560
:10EC00008051C1F855659DF8081001EB4103C3EB35
:10EC1000C11100EBC1018B799DF8081001EB410C8B
:10EC2000CCEBC11100EBC101497943EA012100EEAF
:10EC3000101AF8EE400A9FED600A9DF8081080EE69
:10EC4000801A01EB4103C3EBC11100EBC1010B7949
:10EC50009DF8081001EB410CCCEBC11100EBC10198
:10EC6000C97843EA012100EE901A9DF82010F8EED1
:10EC7000600A71EE200A10EE903A02EB011101F5E4
:10EC80008051C1F851359DF8081001EB4103C3EBE9
:10EC9000C11100EBC1018B7A9DF8081001EB410C0A
:10ECA000CCEBC11100EBC101497A43EA012100EE2E
:10ECB000901A9DF80810B8EE601AC1EE000A01EB38
:10ECC0004103C3EBC11100EBC1010B7A9DF80810A1
:10ECD00001EB410CCCEBC11100EBC101C97943EA56
:10ECE000012100EE101A9DF82010B8EE400A30EE17
:10ECF000800A10EE103A02EB011101F58051C1F8C3
:10ED000059359DF8081001EB4102C2EBC11100EB2F
:10ED1000C100C07A00069DF8080000EB4001C1EB7D
:10ED2000C01008EBC000027B9DF8080000EB400318
:10ED3000C3EBC01008EBC000C07A42EA00200AD43E
:10ED400000EE100ADFED1D0AB8EE400A20EE200AA0
:10ED500010EE100A0BE0404280B2F9F743FC9FED41
:10ED6000181B53EC112BF9F74BFBF9F7A0FC9DF89E
:10ED7000202009EB021101F58051C1F85D059DF8D5
:10ED800008009DF8202000EB400101EB001009EB8A
:10ED9000001000EB02102844027842F0800202705A
:10EDA0009DF8080000EB4002C2EBC0120CE000002E
:10EDB000E0620020D412002000FF7F470000803D69
:10EDC000000000000000B0BF08EBC200C27D9DF84B
:10EDD000080000EB001303EB002009EBC0039DF8D3
:10EDE000200000EB001003EBC00000F5005080F89D
:10EDF00088209DF8080000EB400202EB001009EBB0
:10EE00000010D0E09DF80800DFF8809400EB40018E
:10EE1000C1EBC01009EBC000C3799DF8080000EBFE
:10EE20004002C2EBC01009EBC000007A43EA0020A8
:10EE3000C317CDE900039DF80800072100EB40024D
:10EE4000C2EBC01009EBC000FAF738FCCDE914069C
:10EE5000DDE90010149B7040594001437ED19DF8BC
:10EE6000080000EB4001C1EBC01119F83100401E51
:10EE70008DF82000DFF818849DF8081008EB0110C9
:10EE800000F5805080F8446B9DF8201008EB0100DD
:10EE900000F5805080F845659DF8080000EB4001C2
:10EEA000C1EBC01109EBC1008079F9F79BFB41EC84
:10EEB000110B9FEDF80B0AF0CFFE9DF80800B0EEA5
:10EEC000408AF0EE608A00EB4001C1EBC01109EB13
:10EED000C10002799DF8080000EB4001C1EBC011B0
:10EEE00009EBC100C07842EA0020F9F77BFB53EC44
:10EEF000182BF9F7F7FAF9F7DAFB9DF8201008EB71
:10EF0000011101F58051C1F855059DF8201008EB5D
:10EF1000011000F58050C0F851659DF8201008EBF5
:10EF2000011000F58050C0F859659DF8201008EBDD
:10EF3000011000F58050C0F85D659DF8080000EBF9
:10EF4000400101EB001108EB01109DF8201000EBCF
:10EF500001102844017841F0800200E092E2027042
:10EF60009DF8080000EB4001C1EBC01109EBC100A6
:10EF7000427A9DF8080000EB001101EB00219DF89A
:10EF8000200008EBC10300EB001003EBC00000F50C
:10EF9000005080F888209DF8080000EB400101EB4C
:10EFA000001108EB011000F5805090F88B0B84F8ED
:10EFB0004405CFE59DF80800DFF8D08200EB400162
:10EFC000C1EBC01008EBC0004146C3789DF80800B3
:10EFD00000EB4002C2EBC01008EBC000807843EAAF
:10EFE00000208DF80C009DF8080000EB4002C2EBF9
:10EFF000C0109DF80C2008EBC000104443789DF829
:10F00000080000EB4002C2EBC0109DF80C2001EBA1
:10F01000C000805C43EA0020C317CDE900039DF8DF
:10F0200008009DF80C1000EB4002C2EBC01008EB8A
:10F03000C000FAF743FBCDE91406DDE90010149B8C
:10F04000704059400143B4D19DF8080000EB4001E5
:10F05000C1EBC01008EBC00040788DF820008DF89F
:10F0600030608B491CE09DF8080000EB400202EB89
:10F0700000109DF8302001EB001000EB021000F5AD
:10F08000805090F8B50B9DF8202090429DF83000FC
:10F0900003D18DF8200013E0FEE3401C8DF8300012
:10F0A0009DF8080000EB400202EB001001EB00109D
:10F0B00000F5805090F88B0B9DF830209042D2D80C
:10F0C0009DF8080000EB400202EB001001EB00127B
:10F0D0009DF8200002EB00102844027842F08002E4
:10F0E00002709DF8080000EB4002C2EBC01008EB74
:10F0F000C0000079ADF818009DF808009DF82020A8
:10F1000001EB0010104400F5805080F8446BBDF80E
:10F110001800F32806D006DC05287DD0F12807D09A
:10F12000F22890D156E2F42877D0F6288BD153E21A
:10F130009DF8080000EB001202EB002001EBC0027A
:10F140009DF8200000EB001002EBC00000F500501D
:10F1500090F84C0000289DF8080025D000EB4002F4
:10F1600002EB00109DF8202001EB001000EB0210D4
:10F1700000F5805090F8BD0BC00714D09DF8080032
:10F180008C4600EB001202EB002001EBC0029DF860
:10F19000200000EB001002EBC00000F5005090F8DA
:10F1A000D200C00724D0C1E000EB001202EB002027
:10F1B00001EBC0029DF8200000EB001002EBC00044
:10F1C00000F5005080F84C709DF80800F42200EB28
:10F1D000001303EB002001EBC0039DF8200000EBBF
:10F1E000001003EBC00000F5005080F851209DE0B6
:10F1F0009DF8080000EB001202EB00200CEBC002AF
:10F200009DF8200000EB001002EBC00000F500505C
:10F2100090F8C400C0B301E059E2F1E18DF830602C
:10F220002AE09DF8080000EB001202EB00209DF898
:10F2300020200CEBC00002EB021200EBC2009DF894
:10F240003020104400F5005090F8C5209DF80800CB
:10F2500000EB400303EB00109DF830300CEB001086
:10F26000184400F5805090F8920B824208D19DF826
:10F270003000401C8DF830009DF830000428D0D3B9
:10F280009DF83000042832D050E00000E0620020F9
:10F29000D412002000000000000024409DF8080067
:10F2A00000EB001202EB00200CEBC0029DF82000E6
:10F2B00000EB001002EBC0009DF83020104400F578
:10F2C000005090F8C5009DF8082002EB420303EBC4
:10F2D00002129DF830300CEB02121A4402F58052F3
:10F2E00092F8922B904208D19DF83000401C8DF886
:10F2F00030009DF830000A28D0D39DF830000A284D
:10F3000014D09DF8080000EB001202EB002001EB86
:10F31000C0029DF8200000EB001002EBC00042F29A
:10F32000D2021044027842F0010202709DF80C00F3
:10F33000112844D09DF80C0014289DF8080000EB1B
:10F34000400202EB00107CD09DF8202001EB001061
:10F3500000EB02102844027822F0040202709DF8AB
:10F36000080000EB001202EB002001EBC0029DF848
:10F37000200000EB001002EBC00000F5005090F8F8
:10F38000D200C0077ED09DF8080000EB001202EB0F
:10F39000002001EBC0029DF8200000EB001002EB02
:10F3A000C00000F50050A0F8D06005229DF80800CC
:10F3B00000EB001303EB002001EBC0016CE29DF8B1
:10F3C000080000EB400202EB001001EB00129DF878
:10F3D000200002EB00104219107840F00403137073
:10F3E0008DF83060424625E09DF8080000EB4003B0
:10F3F000C3EBC01002EBC0039DF830001844437902
:10F400009DF8080000EB001C0CEB002001EBC00C89
:10F410009DF8200000EB00100CEBC00C9DF83000B4
:10F42000604400F5005080F88B309DF830305B1C54
:10F430008DF830309DF830000A28D5D38DF8306033
:10F4400028E02CE09DF8080000EB4003C3EBC0105F
:10F450009DF8303002EBC0001844C37B9DF80800D3
:10F4600000EB001C0CEB002001EBC00C9DF8200011
:10F4700000EB00100CEBC0009DF830C0604400F5BC
:10F48000005000E08EE280F8A4309DF83000401C6F
:10F490008DF830009DF830000228D3D389E501EBC8
:10F4A00000129DF8200002EB00104219107840F085
:10F4B000040313708DF83060424625E09DF8080083
:10F4C00000EB4003C3EBC01002EBC0039DF830001B
:10F4D000184443799DF8080000EB001C0CEB002059
:10F4E00001EBC00C9DF8200000EB00100CEBC00CF1
:10F4F0009DF83000604400F5005080F88B309DF896
:10F5000030305B1C8DF830309DF830000A28D5D3A0
:10F510008DF830601FE09DF8303002EBC0001844D9
:10F52000C37B9DF8080000EB001C0CEB002001EBF6
:10F53000C0089DF820009DF830C000EB001008EBDB
:10F54000C000604400F5005080F8A4309DF8300001
:10F55000401C8DF830009DF8300002289DF808000E
:10F5600000EB4003C3EBC010D5D302EBC0039DF802
:10F5700030001844407C03049DF8080000EB400C68
:10F58000CCEBC01002EBC00C9DF830006044807CD6
:10F5900043EA00239DF8080000EB400CCCEBC010C0
:10F5A00002EBC0029DF830001044C07C03439DF87C
:10F5B000080000EB001202EB002001EBC0019DF8F7
:10F5C000200000EB001001EBC00000F50050C0F877
:10F5D000B830EEE4F122E9E69DF80800032200EBE2
:10F5E000001303EB002001EBC0039DF8200000EBAB
:10F5F000001003EBC00000F5005080F84C20E9E754
:10F600009DF80800022200EB001303EB002001EB41
:10F61000C0039DF8200000EB001003EBC00000F5D4
:10F62000005080F84C209DF80800F62200EB0013F3
:10F6300003EB002001EBC0039DF8200000EB00105D
:10F6400003EBC00000F5005080F851209DF8080041
:10F6500000EB001202EB002001EBC0029DF820003D
:10F6600000EB001002EBC00000F5005080F8C47001
:10F670008DF83060424625E09DF8080000EB40031D
:10F68000C3EBC0109DF8303002EBC0001844437942
:10F690009DF8080000EB001C0CEB002001EBC00CF7
:10F6A0009DF8200000EB00100CEBC0009DF830C06E
:10F6B000604400F5005080F8C5309DF83000401CD3
:10F6C0008DF830009DF830000A28D5D36AE19DF806
:10F6D000080000EB4002C2EBC01008EBC0008379C9
:10F6E0009DF8080000EB400CCCEBC01008EBC0000C
:10F6F000407943EA00229DF8080000EB001303EB79
:10F70000002001EBC0039DF8200000EB001003EB8C
:10F71000C00000F50050A0F8D0209DF8080000EBD4
:10F72000001202EB002001EBC0029DF8200000EB6C
:10F73000001002EBC00000F50050B0F8D0209DF89A
:10F74000080000EB400303EB001001EB001000F594
:10F750008050B0F89E0B8242B8D39DF80800F12289
:10F7600000EB001303EB002001EBC00C9DF8200020
:10F7700000EB00100CEBC00000F5005080F85120A9
:10F780009DF8080000EB001202EB002001EBC00125
:10F790009DF8200000EB001001EBC00042F2D20106
:10F7A0000844017821F00101FEF7B1B99DF8080085
:10F7B00000EB4001C1EBC010FE4A02EBC000007933
:10F7C0008DF820008DF81060DFF8EC831BE09DF8C9
:10F7D00008009DF8101000EB400303EB001008EB4D
:10F7E000001000EB011000F5805090F8B50B9DF86B
:10F7F000201088429DF8100002D18DF8200012E000
:10F80000401C8DF810009DF8080000EB400101EB52
:10F81000001008EB001000F5805090F88B3B9DF82D
:10F8200010008342D3D89DF8080000EB4001C1EBE3
:10F83000C01002EBC000C078ADF81800BDF8180089
:10F84000182812D2DFE800F0110C0E1179797179C5
:10F850007311111175797979797711117911797994
:10F860001A2000E00D208DF80C009DF80C00001F00
:10F87000C1B29DF80800914600EB4003C3EBC013F2
:10F8800002EBC300C01CF9F747FD8DF800009DF89E
:10F89000080000EB400100E0FCE3C1EBC0119DF863
:10F8A0000C0009EBC101084410F8010C9DF8001090
:10F8B000884277D19DF808004A4600EB4001C1EB31
:10F8C000C01009EBC000407800286BD09DF80800FC
:10F8D00000EB4001C1EBC0109DF80C1002EBC00022
:10F8E0000844C3789DF8080000EB001101EB0021EB
:10F8F00008EBC10C9DF82010404601EB01110CEB08
:10F90000C10101F5005181F888309DF8081008EB1D
:10F9100001139DF82010194401F5805181F8446BC2
:10F9200098F8141001290AD01AE007209BE7082054
:10F9300099E70C2097E70A2095E7062093E79DF8C2
:10F94000081001EB410303EB01119DF8203000EB9F
:10F95000011101EB031129440B7843F080030B7074
:10F96000BDF81810CE2912D012DCB9297ED008DCDF
:10F970005A29AAD0B2297AD0B529F7D0B62998D178
:10F98000FEE3C32974D0C52973D0CA2991D1F8E305
:10F99000E129FCD007DCD5290AD0D72995D0D9296F
:10F9A00087D1CCE25CE3E5297DD0E729E7D1E9E323
:10F9B0009DF8081001EB4103C3EBC11109EBC10134
:10F9C000C97884F8A2119DF8081001EB410202EBFE
:10F9D0000112014600EB02109DF8202000EB0210FE
:10F9E00094F8A2212844A7EBD213027863F3000213
:10F9F00002709DF8080000EB400202EB00109DF839
:10FA0000202001EB001000EB021094F8A221284402
:10FA10005309027863F3410202709DF8080000EB7D
:10FA2000400202EB00109DF8202001EB001000EBDB
:10FA3000021000F5805090F8B60BC0F340029DF81C
:10FA400008009DF8201000EB001303EB002008EBEA
:10FA5000C00001EB011100EBC10000F5005090F86F
:10FA60006400C0F34000824257D003E0FDE3FDE3B1
:10FA7000FDE3FDE39DF8080000EB001101EB002021
:10FA800008EBC0029DF82000414600EB001002EB9D
:10FA9000C00042F2640210449DF8082002EB4203C9
:10FAA00003EB021200E0F4E39DF8203008EB0212B1
:10FAB00002EB031202F5805292F8B62B530802783B
:10FAC00063F3410202709DF8080000EB400202EB74
:10FAD00000109DF8202001EB001000EB021000F553
:10FAE000805090F8B60B800718D59DF80800D922F1
:10FAF00000EB001303EB002008EBC0019DF8200091
:10FB000000EB001001EBC00000F5005080F8512020
:10FB10009DF808100220FAF767F847E09DF8080002
:10FB200000EB001202EB002001EBC0029DF8200068
:10FB300000EB001002EBC00000F5005080F8597097
:10FB40009DF80800D92200EB001303EB002001EB25
:10FB5000C0039DF8200000EB001003EBC00000F58F
:10FB6000005080F851209DF8080000EB400202EBA5
:10FB7000001001EB00129DF8200002EB001042196A
:10FB8000107820F0200313709DF8080000EB00129D
:10FB900002EB002008EBC0019DF8200000EB0010F4
:10FBA00001EBC00000F5005080F88A709DF8080055
:10FBB00004E00000E0620020D412002000EB4001CD
:10FBC00001EB001008EB00119DF82000434601EB0B
:10FBD000001000F5805090F8B60B00F001019DF880
:10FBE000080000EB001202EB002008EBC0029DF8B9
:10FBF000200000EB001002EBC00000F5005090F870
:10FC0000640000F00100814271D09DF808009DF869
:10FC1000202000EB001101EB0020194603EBC0008F
:10FC200002EB021200EBC20042F2640210449DF8A3
:10FC3000082002EB420303EB02129DF8203001EB97
:10FC4000021202EB031202F5805292F8B62B0378EF
:10FC500062F3000303709DF8080000EB400202EB22
:10FC600000109DF8202001EB001000EB021000F5C1
:10FC7000805090F8B60BC0079DF8080038D000EB14
:10FC8000001202EB002001EBC0029DF8200000EB07
:10FC9000001002EBC00000F5005090F88A00002828
:10FCA0009DF8080000EB001202EB002001EBC002FF
:10FCB0009DF8200000EB001002EBC00000F50050A2
:10FCC00038D080F889609DF8080000EB400202EB14
:10FCD000001001EB00129DF8200002EB0010421909
:10FCE000107820F00103137094F8620728B3DBE06A
:10FCF00000EB400202EB00109DF8202001EB001009
:10FD000000EB02102844027822F0200202709DF8D5
:10FD1000080000EB001202EB002001EBC0019DF88F
:10FD2000200000EB001001EBC00000F5005080F84F
:10FD30008960B9E080F88970D6E7487D012868D1EC
:10FD4000486DCA8A904264D29DF8080000EB001208
:10FD500002EB002001EBC0029DF8200000EB001038
:10FD600002EBC00000F5005090F88900012850D146
:10FD70009DF8080000EB001202EB002001EBC0022E
:10FD80009DF8200000EB001002EBC00000F50050D1
:10FD900090F8C300E8BB9DF8080000EB400202EBBE
:10FDA000001001EB00129DF8200002EB001000F59E
:10FDB000805090F8B42B9DF8080000EB001303EB83
:10FDC000002001EBC00000F5005080F845209DF8B0
:10FDD0000800C32200EB001303EB002001EBC0037B
:10FDE0009DF8200000EB001003EBC00000F5005070
:10FDF00080F851209DF8080000EB400202EB001053
:10FE000008EB00119DF8200001EB001000F5805078
:10FE100000E049E0C0F8B86B9DF808100220F9F73F
:10FE2000E3FE8DF83060414619E09DF8080000EBD4
:10FE3000001202EB002001EBC0029DF8200000EB55
:10FE4000001002EBC0009DF83020104400F5005077
:10FE500080F88B609DF83000401C8DF830009DF8D4
:10FE600030001428E1D38DF8306019E09DF80800C7
:10FE700000EB001202EB002001EBC0029DF8200015
:10FE800000EB001002EBC0009DF83020104400F59C
:10FE9000005080F8A7609DF83000401C8DF83000BD
:10FEA0009DF830000A28E1D39DF808009DF8202035
:10FEB00000EB400101EB0010414608EB001000EBA5
:10FEC000021000F5805090F8B60B80077BF53FAB31
:10FED0009DF80800D92200EB001303EB002001EB92
:10FEE000C0039DF8200000EB001003EBC00000F5FC
:10FEF000005080F85120FBF72ABB9DF8080000EB6A
:10FF0000001202EB002001EBC00000F5005080F869
:10FF100047609DF80800022200EB001303EB00206D
:10FF200001EBC0039DF8200000EB001003EBC000C4
:10FF300000F5005080F84C20B622FBF799BC9DF8E4
:10FF4000081001EB410303EB011108EB011000F570
:10FF5000805090F8900B00289DF80C0002D00A28E1
:10FF60007ED198E00828FBD18DF8306024E09DF820
:10FF7000080000EB4001C1EBC0109DF8301002EB0F
:10FF8000C0000844C07800F00F00092818D89DF878
:10FF9000080000EB4001C1EBC0109DF8301002EBEF
:10FFA000C0000844C07800F0F000902808D89DF800
:10FFB0003000401C8DF830009DF830000628D6D364
:10FFC0009DF8300006284BD39DF8080000EB400157
:10FFD000C1EBC01002EBC000C07801049DF808001E
:10FFE00000EB4003C3EBC01002EBC000007941EA14
:10FFF00000239DF8080000EB4001C1EBC01002EBAC
:020000040801F1
:10000000C000407903439DF8080000EB001101EBAC
:10001000002008EBC00C9DF82000414600EB0010CA
:100020000CEBC00000F50050C0F865309DF80800EA
:1000300000EB4003C3EBC01002EBC0008079030467
:100040009DF8080000EB400CCCEBC01002EBC000A8
:10005000C07943EA00239DF8080000EB400C00E063
:10006000C8E0CCEBC01002EBC000007A03439DF85F
:10007000080000EB001202EB002001EBC0019DF82C
:10008000200000EB001001EBC00000F50050C0F8AC
:100090006930ACE074E18DF8306024E09DF8080030
:1000A00000EB4001C1EBC0109DF8301002EBC00026
:1000B0000844C07800F00F00092818D89DF80800FF
:1000C00000EB4001C1EBC0109DF8301002EBC00006
:1000D0000844C07800F0F000902808D89DF830005F
:1000E000401C8DF830009DF830000828D6D39DF8CC
:1000F000300008287ED39DF8080000EB4001C1EBDA
:10010000C01002EBC00081799DF8080000EB4003AD
:10011000C3EBC01002EBC000C07841EA00619DF85B
:10012000080000EB4003C3EBC01002EBC0000079F5
:1001300003049DF8080000EB400CCCEBC01002EB70
:10014000C000407943EA002001439DF8080000EB1D
:10015000001303EB002008EBC0039DF8200000EB28
:10016000001003EBC00000F50050C0F865109DF8CA
:10017000080000EB4001C1EBC01002EBC00002E040
:1001800006E1E6E0EEE3817A9DF8080000EB40032B
:10019000C3EBC01002EBC000C07941EA00619DF8DA
:1001A000080000EB4003C3EBC01002EBC000007A74
:1001B00003049DF8080000EB400CCCEBC01002EBF0
:1001C000C000407A43EA002001439DF8080000EB9C
:1001D000001202EB002008EBC0029DF8200000EBAB
:1001E000001002EBC00000F50050C0F869109DF847
:1001F000080000E03AE200EB001101EB002008EB00
:10020000C0029DF82000414600EB001002EBC00048
:1002100000F5005090F84C00032814D09DF8080019
:1002200000EB400202EB001001EB00129DF82000F1
:1002300002EB001000F5805090F8B60B80077BF5BC
:1002400021AB5A4679E69DF8080000EB001202EB5C
:10025000002001EBC00000F5005080F847609DF8D9
:100260000800042200EB001303E074E03FE140E0EB
:100270006DE103EB002001EBC0039DF8200000EBD3
:10028000001003EBC00000F5005080F84C20C522A0
:1002900053E6EDE39DF8080000EB001202EB0020AE
:1002A00001EBC0029DF8200000EB001002EBC00043
:1002B00000F5005080F85A609DF80800B62200EB67
:1002C000001303EB002001EBC0039DF8200000EBBE
:1002D000001003EBC00000F5005080F851209DF89D
:1002E000080000EB001202EB002008EBC000FBF757
:1002F00098BB9DF8081001EB011303EB012100EB03
:10030000C1039DF8201001EB011103EBC10101F5C0
:10031000005181F851B09DF8081001EB011202EB79
:10032000012100EBC10101F5005181F847709DF8F2
:10033000081001EB410202EB011108EB01109DF8DE
:10034000201000EB01102844017841F02001FDF756
:10035000DEBB5A460CE09DF8081001EB011202EBDF
:10036000012100EBC10101F5005181F84760C32272
:100370009DF8081001EB011303EB012108EBC1010B
:100380009DF8200000EB001001EBC000FBF734BF2C
:100390009DF8081001EB410303EB011100EB011183
:1003A00001F5805191F8901B00299DF8081001EB90
:1003B0004103C3EBC11102EBC10158D0C9780B0452
:1003C0009DF8081001EB410CCCEBC11102EBC1010F
:1003D000097943EA01239DF8081001EB410CCCEBAD
:1003E000C11109EBC10149790B439DF8081001EBDC
:1003F000011202EB012100EBC1029DF8201001EB7C
:10040000011102EBC10101F50051C1F880309DF8E6
:10041000081001EB011202EB012100EBC1029DF873
:10042000201001EB011102EBC10101F5005191F81F
:100430004C1002293AD09DF80810C52201EB011397
:1004400003EB012100EBC1039DF8201001EB01112A
:1004500003EBC10101F5005181F851209DF808100E
:1004600001EB011202EB012108EBC1003FE70B7920
:100470009DF8081001EB410CCCEBC11109EBC10157
:10048000C97843EA01229DF8081001EB011303EB40
:10049000012100EBC1039DF8201001EB011103EBDA
:1004A000C10101F50051C1F88020B0E79DF80810A6
:1004B00001EB011202EB012100EBC10101F500513A
:1004C00081F847609DF80810032201EB011303EB4C
:1004D000012100EBC1039DF8201001EB011103EB9A
:1004E000C10101F5005181F84C20D92204E39DF8A7
:1004F000081001EB011202EB012100EBC10101F533
:10050000005181F847709DF8081001EB011303EBCF
:10051000012100EBC1039DF8201001EB011103EB59
:10052000C10101F5005181F851B09DF8081001EBAF
:10053000410202EB011108EB01109DF8201000EBC5
:1005400001102844017841F00402FBF7D7BA9DF866
:100550000810C64601EB410303EB011108EB011043
:1005600000F5805090F8900B00289DF80C0002D008
:100570000E287BD1A0E00C2878D18DF8306024E0E3
:100580009DF8081001EB4100C0EBC1109DF8301040
:1005900002EBC0000844C07800F00F00092818D80A
:1005A0009DF8081001EB4100C0EBC1109DF8301020
:1005B00002EBC0000844C07800F0F000902808D892
:1005C0009DF83010491C8DF830109DF830000A2835
:1005D000D6D39DF830000A2848D30020CDE900008A
:1005E00030468DF830601FE0DDE90031090241EA54
:1005F00013611B02CDE900319DF8081001EB4103A6
:10060000C3EBC1119DF8303002EBC1011944C97828
:10061000DDE9003C194340EA0C03CDE900139DF8E5
:100620003010491C8DF830109DF830100529DBD3AF
:10063000DDE9003C9DF8081001EB011808EB0121F1
:100640000EEBC1099DF82010F04601EB011109EBFA
:10065000C10101F50059C9F86D304946C1F871C0B2
:100660000023CDE900338DF8300020E0D2E0DDE951
:1006700000131B0243EA11630902CDE900139DF840
:10068000081001EB4103C3EBC1119DF8303002EBC0
:10069000C1011944097ADDE9003C194340EA0C0321
:1006A000CDE900139DF83010491C8DF830109DF8ED
:1006B00030100529DBD39CE08DF8306024E09DF8F4
:1006C000081001EB4100C0EBC1109DF8301002EBA7
:1006D000C0000844C07800F00F00092818D89DF821
:1006E000081001EB4100C0EBC1109DF8301002EB87
:1006F000C0000844C07800F0F000902808D89DF8A9
:100700003000401C8DF830009DF830000C28D6D306
:100710009DF830000C287DD30020CDE90000304644
:100720008DF830601FE0DDE90031090241EA136114
:100730001B02CDE900319DF8081001EB4103C3EB2A
:10074000C1119DF8303002EBC1011944C978DDE9CF
:10075000003C194340EA0C03CDE900139DF830102A
:10076000491C8DF830109DF830100629DBD3DDE9E7
:10077000003C9DF8081001EB011808EB01210EEB7D
:10078000C1099DF82010F04601EB011109EBC101F0
:1007900001F50059C9F86D304946C1F871C0002310
:1007A000CDE900338DF830001FE0DDE900131B02B6
:1007B00043EA11630902CDE900139DF8081001EB2B
:1007C0004103C3EBC1119DF8303002EBC101194464
:1007D000497ADDE9003C194340EA0C03CDE90013F6
:1007E0009DF83010491C8DF830109DF83010062906
:1007F000DBD3DDE900129DF8080000EB001303EBEA
:10080000002008EBC0039DF8200000EB001003EB74
:10081000C00000E02BE100F50053C3F87510184646
:10082000C0F879209DF80800F04600EB001101EBBC
:1008300000200EEBC0029DF8200000EB001002EB40
:10084000C00000F5005090F84C209DF8080000EB27
:10085000001303EB00200EEBC00000F5005090F8F1
:10086000480082427DD194F86207B0B19DF808003B
:1008700000EB400101EB001108EB01109DF8201086
:1008800000EB01102844017841F0080101709DF847
:1008900008100220F9F7A8F980E0C8F835609DF843
:1008A000080000EB001101EB00219DF8200008EB8F
:1008B000C10100EB001001EBC00042F26D010144E8
:1008C00010220A98F7F7C1FC9DF8080000EB001110
:1008D00001EB00219DF8200008EBC10100EB0010A6
:1008E00001EBC000653000F500504146026841F858
:1008F000192F406848609DF8080000EB400101EBAB
:10090000001108EB01109DF8201000EB011000F51C
:10091000805090F8B41B88F818109DF8080000EB80
:10092000001101EB00219DF8200008EBC10100EB54
:10093000001001EBC00000F50050D0F88010C8F89E
:100940002110099940468A6A40F8392F898D8180A3
:10095000D8F8540081B20220F8F73CFB00210620B1
:1009600001E00AE026E1F9F73FF9D8F85400401C0D
:10097000C8F85400002105208CE79DF8080000EB22
:10098000400101EB001108EB01109DF8201000EB75
:1009900001102844017841F0040101709DF808001D
:1009A00000EB001101EB002008EBC0029DF82000D5
:1009B000414600EB001002EBC00000F5005080F84B
:1009C0008A609DF8080000EB001303EB002008EBA1
:1009D000C0039DF8200000EB001003EBC00000F501
:1009E000005080F851B09DF8080000EB001202EBB7
:1009F000002001EBC0029DF8200000EB001002EB8C
:100A0000C00000F5005090F84C0004282FD19DF84C
:100A1000080000EB400202EB00109DF8202001EBE3
:100A2000001000EB02102844027842F080020270AD
:100A30009DF8080000EB001202EB002001EBC00063
:100A400000F5005080F847709DF80800052200EB83
:100A5000001303EB002008EBC0019DF8200000EB21
:100A6000001001EBC00000F5005080F84C2083E03E
:100A700084F8A0769DF8081001EB011202EB012129
:100A800000EBC1029DF8201001EB011102EBC10146
:100A900001F5005191F84C1000299DF8081001EB68
:100AA000011202EB01210ED000EBC1029DF82010D3
:100AB00001EB011102EBC10101F5005191F84E105B
:100AC000B22928D058E000EBC10101F5005181F8AE
:100AD00047609DF8081001EB011202EB012100EBC9
:100AE000C1029DF8201001EB011102EBC10101F5DB
:100AF000005181F84C705A469DF8081001EB011323
:100B000003EB012108EBC1039DF8200000EB00106E
:100B100003EBC0003AE49DF8081001EB011202EB70
:100B2000012100EBC10101F5005181F847609DF8FA
:100B30000810B22201EB011303EB012100EBC1030A
:100B40009DF8201001EB011103EBC10101F50051EB
:100B500081F851209DF8081001EB011202EB0121F0
:100B600008EBC1029DF8200000EB001002EBC00072
:100B700000F5005080F84E6094F8A703B0B121480A
:100B80009DF8081000EB410000F58040B0F86412B9
:100B90009DF80800012300EB4002C2EBC0121A4886
:100BA00000EBC2009DF80820F9F716FF8DF83060C1
:100BB000154913E084F8A066FFF7CBBB9DF8080049
:100BC00000EB4002C2EBC0109DF8302001EBC000EA
:100BD00086549DF83000401C8DF830009DF83000A0
:100BE0001428EBD3094801784278114482781144E3
:100BF000C278D1427AF4B2A823B0BDEC028BBDE832
:100C0000F08F0000D4120020E062002010080020C5
:100C10002DE9F74F90B00020ADF80000ADF80400CA
:100C2000ADF80400ADF804008DF810008DF8140044
:100C30008DF81800CDE90800CDE90800ADF83C00BA
:100C4000FAA2D2E90032CDE90232FAA2D2E90032A8
:100C5000CDE90A32F94A1071109800EB400202EB1C
:100C60000010F74A02EB001E0EF58050834690F804
:100C70008A0B8DF81000109802EB001007900844C2
:100C800000F58050824690F8443B1098042B00EB0E
:100C9000001404EB0020144604EBC00001EB011427
:100CA00000EBC4070D900EEB011007F5005500F5A1
:100CB00080591FD105208AF8440B002085F84C008C
:100CC00099F8B60B20F0800389F8B63B9BF88A3B75
:100CD000A120072B0ED2DFE803F00D040B0B060852
:100CE0000A00E52004E0B12002E0312000E0F1201C
:100CF00085F85100D248007D012870D09DF8108001
:100D00001098DDF848C000EB001404EB0020CC4C38
:100D1000022304EBC00000F500500190109841221E
:100D2000C84EC0EB001000EB8004ACF1A10CB8F190
:100D3000070F7CD2DFE818F07B0007009502E5037F
:100D400074055006C40699F8B50B4FF000084146EB
:100D500001F086FD8DF8140095F84C10019890F87C
:100D60004800814203D10198012180F847109AF888
:100D7000440B401C8AF8440B129BA221A620CE2BC8
:100D80007ED012DC4FF0A502B92B7AD006DCB22B54
:100D900078D0B52B36D0B62B49D10DE1C32B72D00C
:100DA000C52B71D0CA2BF7D1FBE0E12B6DD006DC4F
:100DB000D52B09D0D72B69D0D92BEDD110E0E52B5D
:100DC00070D0E72BE8D136E2F52006F834009DF824
:100DD000140006EBC4056870A970D5200AE0EFE3A3
:100DE000F52006F834009DF8140006EBC405687081
:100DF000A970D920E8702846032101F062FC28710F
:100E000005200CE2F52106F834109DF8141006EBCD
:100E1000C40779709BF8901B4FF0B50959B1696D03
:100E2000B1F1104F38D34FF01041002200E099E2A9
:100E3000CDE9081233E0686DB0F5100F05D34FF41B
:100E400010000021CDE9080102E0686DCDE9080835
:100E5000BA7040460FE0BDF80000C0F10200C200C9
:100E6000DDE90801F7F7DFF9BDF800103944C87073
:100E7000BDF80000401CADF80000BDF8000006E021
:100E800033E127E0A3E081E024E1FAE0DEE103289A
:100E9000E1D387F80690EDE06A6DCDE90828B870D7
:100EA000404610E0BCE1BDF80000C0F10300C20004
:100EB000DDE90801F7F7B7F9BDF800103944C8704B
:100EC000BDF80000401CADF80000BDF8000004288B
:100ED000E9D359E0F52106F834109DF8141006EB1B
:100EE000C40779709BF8901B4FF0B90949B1696D3F
:100EF000B1F1104F2CD0696DCDE90818B87040469B
:100F00003CE0686DB0F5100F05D0696DCDE90818AB
:100F1000BA70404615E04FF410000021CDE90801F9
:100F2000F6E7BDF80000C0F10200C200DDE90801EB
:100F3000F7F779F9BDF800103944C870BDF8000022
:100F4000401CADF80000BDF800000328E9D3A0E77D
:100F50004FF010410022CDE90812CFE7BDF80000A4
:100F6000C0F10300C200DDE90801F7F75CF9BDF844
:100F700000103944C870BDF80000401CADF80000F6
:100F8000BDF800000428E9D348469BE0F52006F8A8
:100F900034009DF8140006EBC4056870A970C320E6
:100FA00028E7F52006F834009DF8140006EBC40588
:100FB0006870A970CA201DE7F52006F834009DF876
:100FC000140006EBC4056870A970B62012E7F5207E
:100FD00006F834009DF8140006EBC40778709BF8FF
:100FE000900BB22110B1BA7040463CE0A420B8701A
:100FF00040460EE0D5F88000BDF80020C2F10102A5
:10100000D200D040BDF800203A44D070BDF80000B6
:10101000401CADF80000BDF800000228EAD3797149
:101020003846052101F04DFBB8717CE10169323091
:101030003130300001693230453030001008002076
:10104000D412002080590020D5F88000BDF800207F
:10105000C2F10202D200D040BDF800203A44D07064
:10106000BDF80000401CADF80000BDF800000328EA
:10107000EAD3B9713846062101F023FBF871082044
:10108000CDE0F52106F834109DF8141006EBC407E6
:101090007970B87040460EE0D5F88400BDF80010B5
:1010A000C1F10301C900C840BDF800103944C8703F
:1010B000BDF80000401CADF80000BDF80000042899
:1010C000EAD3E120F8713846072101F0FAFA3872C4
:1010D0000920A4E0F52006F834009DF8140006EB82
:1010E000C4056870A970C52084E6F52006F83400B0
:1010F0009DF8140006EBC40568709BF8900B4FF048
:10110000CE0918B1AE20A87040465CE0AC20A870B3
:10111000404615E007F50050D0F86D0007F5005186
:10112000D1F87110BDF80020C2F10402D200F7F727
:101130007AF8BDF800102944C870BDF80000401CC2
:10114000ADF80000BDF800000528E3D3404615E0E7
:1011500007F50050D0F8750007F50051D1F8791067
:10116000BDF80020C2F10402D200F7F75CF8BDF828
:10117000001029440872BDF80000401CADF80000C2
:10118000BDF800000528E3D385F80D9028460D2111
:1011900001F097FAA8730F2041E007F50050D0F84E
:1011A0006D0007F50051D1F87110BDF80020C2F1B3
:1011B0000502D200F7F737F8BDF800102944C870CF
:1011C000BDF80000401CADF80000BDF80000062886
:1011D000E3D3404615E007F50050D0F8750007F559
:1011E0000051D1F87910BDF80020C2F10502D200FB
:1011F000F7F719F8BDF8001029444872BDF800004F
:10120000401CADF80000BDF800000628E3D385F8C7
:101210000F9028460F2101F054FA28741120ACE2F7
:10122000F52006F834009DF8140006EBC40568703C
:10123000A970E520DEE5F52006F834009DF81400DD
:1012400006EBC4056870A970E720D3E5F52006F821
:1012500034009DF8140006EBC4056870A970D7200F
:10126000C8E599F8B50B8DF8140095F84C10019865
:1012700090F84800814203D10198012180F847107D
:101280009AF8441B491C8AF8441B9DF8140020B1AD
:101290009DF81400401E8DF81400BCF10A0F61D2B5
:1012A000DFE80CF0F6F54B7FDFF4F305F26106F8AA
:1012B00034309DF8140006EBC40740307870BA70E3
:1012C0003020F870387195F85000000978717879FD
:1012D0000A28787901D2303000E03730787195F8FB
:1012E000500000F00F00B871B8790A28B87901D21F
:1012F000303000E03730B8710320F871781C0721D6
:10130000F8F70AF838720920ADF83C0095F84C005F
:10131000042802D1052085F84C000199002081F8AD
:10132000470006201CE0072027E22871032068718F
:10133000681C0521F7F7F0FFFEE3042306F83430BC
:101340009DF8141006EBC4004031417082700521F5
:10135000C170ADF83C3095F84C00022802D1032052
:1013600085F84C0002E106F834309DF8140006EBD5
:10137000C40540306870AA703120E87032202871AE
:1013800003206871681C0521F7F7C6FFA8710720C4
:10139000ADF83C0099F8B60B20F0200189F8B61B97
:1013A000F1E306F834309DF8140006EBC407403032
:1013B0007870BA703121F970302038716A6DB2F5E9
:1013C000100F00D23220787195F85200012803D016
:1013D00095F8520010B103E0B97101E03220B87104
:1013E0000021ADF8001012E0686DBDF80020C2F1D8
:1013F00005029200D040BDF8002000F00F003A44F2
:101400003030D071BDF80000401CADF80000BDF8D0
:1014100000000628E8D332207873ADF8001013E0FE
:10142000D5F88000BDF80010C1F103018900C84063
:10143000BDF8001000F00F00394430308873BDF85B
:101440000000401CADF80000BDF800000428E7D300
:101450000320B874781C1221F7F75EFFF87414208B
:101460008FE306F834309DF8140006EBC4074030D3
:101470007870BA703220F870312139717871B87192
:101480000021ADF8001018E07EE056E156E16EE074
:101490005DE0D5F88000BDF80020C2F103029200A3
:1014A000D040BDF8002000F00F003A443030D07139
:1014B000BDF80000401CADF80000BDF80000042895
:1014C000E7D3ADF80010302008E0BDF80010394433
:1014D000C872BDF80010491CADF80010BDF800102E
:1014E0001929F2D3032087F82400781C2421F7F768
:1014F00013FF87F82500262043E306EBC40148705C
:101500005BE099F8B50B8DF8140095F84C10019834
:1015100090F84800814203D10198012180F84710DA
:101520009AF8440B401C8AF8440B9DF8140020B133
:101530009DF81400401E8DF81400BCF10A0F15D25E
:10154000DFE80CF005152F5AFDFCFB14223F0422A6
:1015500006F834209DF8141006EBC40040314170A9
:10156000512181700521C170ADF83C200BE306F8D4
:1015700034309DF8140006EBC40540306870AA7042
:101580003120E8703520D0E606F834309DF814009C
:1015900006EBC40540306870AA703220E870302035
:1015A000C3E6042306F834309DF8141006EBC4009B
:1015B0004031417082700521C170ADF83C30E2E2EB
:1015C000FDE306F834309DF8140006EBC405403006
:1015D0006870AA703120E870322028710320687189
:1015E000681C0521F7F798FEA87199F8B60B20F052
:1015F000200189F8B61B96E606F834309DF81400F1
:1016000006EBC40740307870BA703120F8703A7138
:10161000696DB1F1104F09D03221797195F85210EE
:10162000012905D095F8520038B102E03021F4E7E5
:10163000B8710022ADF8002014E03220F8E7686DA0
:10164000BDF80010C1F107018900C840BDF80010C5
:1016500000F00F0039443030C871BDF80000401C64
:10166000ADF80000BDF800000828E8D33220F87378
:10167000ADF8002013E0D5F88000BDF80010C1F1EE
:1016800005018900C840BDF8001000F00F00394482
:1016900030300874BDF80000401CADF80000BDF803
:1016A00000000628E7D33020B875ADF8002008E028
:1016B000BDF800103944C875BDF80010491CADF8DC
:1016C0000010BDF800100629F2D37877ADF800209D
:1016D00008E0BDF8001039448877BDF80010491CB7
:1016E000ADF80010BDF800100629F2D387F82400E9
:1016F000ADF8002009E0BDF80010394481F825005C
:10170000BDF80010491CADF80010BDF80010062906
:10171000F1D387F82B00ADF8002009E0BDF80010E8
:10172000394481F82C00BDF80010491CADF80010B8
:10173000BDF800100629F1D302E06CE066E01DE080
:1017400087F83200ADF8002009E0BDF800103944F8
:1017500081F83300BDF80010491CADF80010BDF849
:1017600000100629F1D3032087F83900781C3921AD
:10177000F7F7D2FD87F83A003B2002E206F8343052
:101780009DF8140006EBC40740307870BA70322020
:10179000F8703121397133217971B8710021ADF8B8
:1017A000001013E0D5F88000BDF80020C2F105025A
:1017B0009200D040BDF8002000F00F003A443030D5
:1017C000D071BDF80000401CADF80000BDF800006D
:1017D0000628E7D3ADF80010302008E0BDF800106F
:1017E00039444873BDF80010491CADF80010BDF82D
:1017F00000101929F2D3032087F82600781C26212F
:10180000F7F78AFD87F827002820BAE1102006F8AC
:101810003400302071E6102006F8340031206CE6E8
:1018200099F8B50B8DF81400BDF800000D9A00EB87
:10183000001002EBC00000F5005090F84C20019819
:1018400090F84800824203D10198012280F8472095
:101850009AF8440B401C8AF8440B0027ADF800703E
:1018600010E0BDF800200EEB021000F5805090F85B
:10187000B50B9DF8142090420AD0BDF80000401C22
:10188000ADF800009BF88B0BBDF800209042E8D823
:10189000BDF800200EEB021000F5805090F8B40B5C
:1018A000081A401C8DF818009DF8140020B19DF80E
:1018B0001400401E8DF8140095F84D000F2805D235
:1018C00095F84D00401C85F84D0001E085F84D70FD
:1018D00012986521B1384FF0FA0809287BD2DFE869
:1018E00000F0050C437A7A647A1D2F009DF81400ED
:1018F000503006F83400202166E09DF81400503086
:1019000006F8340095F84D0006EBC40540F03000B1
:1019100068700120A870E8702F7136E09DF81400FF
:10192000503006F8340095F84D0006EBC40540F041
:1019300030006870A9700120E8709DF8180023E05D
:101940009DF81400503006F8340095F84D0006EB71
:10195000C40540F030006870A9700120E8709DF85F
:10196000180040F010000FE09DF81400503006F809
:10197000340095F84D0006EBC40540F03000687067
:101980000120A870E8700520287128460521F8F785
:1019900081F8CDE9080768710898000AA87103204A
:1019A000E87185F80880FFF793BB95F84E0085F83D
:1019B000510085F84E709DF81400503006F8340040
:1019C00095F84D0040F0C00106EBC400417080F86E
:1019D00002800320D5E088E0BDF80020079810447D
:1019E00041F6443210440278521C02709BF8900B6E
:1019F00030B1491CC9B2012836D0022875D144E063
:101A00001298312802D045286FD116E00020ADF899
:101A1000000002A90CE0BDF80000BDF8003006EBA4
:101A2000C402085CD054BDF80000401CADF80000B2
:101A3000BDF800000728EED375E40020ADF80000E3
:101A40000AA90CE0BDF80000BDF8003006EBC402A6
:101A5000085CD054BDF80000401CADF80000BDF893
:101A600000000728EED35EE48DF814109DF81400F2
:101A700006F8340006EBC405032068700027AF7039
:101A8000EB702F71092068710EE08DF814109DF82D
:101A9000140006F8340006EBC40503206870002724
:101AA000AF70EF702F716B7128460621F7F706FEB5
:101AB000CDE90807000AE8710898A871FFF7DFBAB6
:101AC000F7499AF8440B401C8AF8440B99F8B50B77
:101AD0008DF814001298F3287DD007DC05287BD000
:101AE000F12808D0F2284ED113E04CE0F42874D04D
:101AF000F62848D1FAE0F52006F834009DF81400E5
:101B000006EBC40568700027AF700520E870F1206F
:101B10001EE1F52006F834009DF8141006EBC40011
:101B2000804641704FF0000980F80290F221017167
:101B300095F8C210417100E014E195F8C200012847
:101B40002CD095F8C20020287ED00620ADF83C00AD
:101B5000BDF83C0088F803004046BDF83C10F7F79C
:101B6000ADFDCDE90809BDF83C20000A08F80200E7
:101B7000BDF83C20089808EB02014870BDF83C0015
:101B8000801CADF83C00C748C74D109931B30129FE
:101B900078D0022977D0032976D18AE12520ADF8C3
:101BA0003C004946ADF8009010E0BDF80000384414
:101BB00000F5005090F89520BDF8003008EB0300C8
:101BC0008271BDF80000401CADF80000BDF80000B7
:101BD0000F28EAD303E058E0C6E0ACE035E1ADF809
:101BE000001010E0BDF80000384400F5005090F8F7
:101BF000A720BDF8003008EB03004275BDF80000D7
:101C0000401CADF80000BDF800000A28EAD395F8A2
:101C1000BC2088F81F20ADF8001011E0BDF80000CE
:101C2000384400F5005090F8BD10BDF8002008EBD6
:101C3000020080F82010BDF80000401CADF8000044
:101C4000BDF80000052800E001E0E7D380E70A20A6
:101C5000ADF83C0048460EE0BDF80000384400F501
:101C6000005090F8BD10BDF8002008EB0200817113
:101C7000BDF80000401CADF80000BDF800000428CD
:101C8000EAD365E7EFE0FBE012E1F52006F8340067
:101C90009DF8141006EBC400804641704FF0000917
:101CA00080F80290F322027195F8C22042710C2252
:101CB000ADF83C2095F8BC208271ADF8009010E0A2
:101CC000BDF80000384400F5005090F8BD10BDF894
:101CD000002008EB0200C171BDF80000401CADF807
:101CE0000000BDF800000528EAD331E70620ADF872
:101CF0003C00F52006F834009DF8140006EBC405FE
:101D000068700027AF70BDF83C00E870F6202871BD
:101D100099F8BC0B68712846BDF83C10F7F7CEFC6B
:101D2000CDE90807BDF83C10000A6854BDF83C1026
:101D30000898294421E7F52006F834009DF814009E
:101D400006EBC40568700027AF700520E870F4202A
:101D5000287128460521F7F7B1FCCDE90807000AEC
:101D600068710898A87146E440F21320ADF83C0071
:101D7000F52006F834009DF8140006EBC4077870CF
:101D8000BDF83C00000AB870BDF83C00F8700520B2
:101D900038714FF0000840460EE0BDF800200EEB11
:101DA000020000F5805090F8920BBDF800203A44F4
:101DB0005071BDF80000401CADF8000000E093E059
:101DC000BDF800000A28E8D3BBF89E0B8946000A3C
:101DD000F873BBF89E0B387435F8D00F000A78748E
:101DE0002888B8742988109801EB802081B20320DC
:101DF000F7F784F84546ADF8008049464FF4007285
:101E00000FE0BDF80000084400F5805090F8A601EE
:101E1000BDF800303B44D874BDF80000401CADF85C
:101E20000000BDF800009042EBD33846BDF83C10EE
:101E3000F7F744FCCDE90805BDF83C10000A7854DA
:101E4000BDF83C100898394497E6BDF83C1079B3CA
:101E50008021F8F7FCFABDF83C00C5F8A400124850
:101E60000121A03031E0BDF83C1009B30821F8F79A
:101E7000EEFABDF83C0068670B480121703024E0A1
:101E8000BDF83C00A0B14FF480710848F8F7DFFAC4
:101E9000BDF83C00C5F8BC0003480121B83014E08F
:101EA000D4120020000C02400060024000000240FA
:101EB0000DE0BDF83C1051B14FF48061F8F7C7FA5E
:101EC000BDF83C00E86501210948F7F74DFC0948D9
:101ED00090F8A703002807D006EBC4000023BDF844
:101EE0003C10109AF8F778FD13B0BDE8F08F0000B1
:101EF00058600240D42200202DE9F04700242DED47
:101F0000048B804689469FED1E9B25462646E200AF
:101F100040464946F6F787F9C7B22046F6F762FB16
:101F200041EC110BB0EE490AF0EE690A07F094FE9D
:101F3000380907F00F0100EB8000B0EE408AF0EEA8
:101F4000608A01EB4000F6F74DFB53EC182BF6F7D7
:101F500057FA41EC180B28463146F6F750FB53EC84
:101F6000182BF6F7A6F9F6F77DFB641CE4B20546DC
:101F70000E46082CCBD3BDEC048BBDE8F0870000E7
:101F8000000000000000594070B50E4D40F224449E
:101F90002146284607F0FBFA012812D12988284655
:101FA0002A1D1188214607F08FFA0748012180F881
:101FB000E51A0648D0F88C000549C0F57A70A1F8FA
:101FC0006C0270BD00440040D4220020006002403A
:101FD000D452002010B50B4C40F22441204607F0AB
:101FE000D6FA01280DD12088201D0088064801213D
:101FF00080F8F11A0548406C0549C0F57A70A1F8DF
:102000006E0210BD004C0040D4220020006002404F
:10201000D452002010B50B4C40F22441204607F06A
:10202000B6FA01280CD12088A0880748012180F841
:10203000FD1A064840690649C0F57A70A1F8700299
:1020400010BD000000500040D4220020006002407B
:10205000D452002010B50B4C40F22441204607F02A
:1020600096FA01280DD12088201D008806480121FC
:1020700080F8091B0548C06A0549C0F57A70A1F8C7
:10208000720210BD00480040D422002000600240CF
:10209000D452002010B5124C10492046F7F74EFBE1
:1020A00000212046F7F760FB0E4C4021204607F048
:1020B00067FA0028F9D080210B48F8F7CAF9084CD4
:1020C0000A49183C2046F7F739FB01212046F7F76B
:1020D0004BFB07490120087110BD00000080202043
:1020E000A060024000440040000C02400088002034
:1020F0001008002010B5124C10492046F7F71EFBBF
:1021000000212046F7F730FB0E4C4021204607F017
:1021100037FA0028F9D008210B48F8F79AF9084C4B
:102120000A49303C2046F7F709FB01212046F7F722
:102130001BFB07490120087110BD00002080002012
:1021400070600240004C0040000C024000802010F3
:102150001008002010B5124C10492046F7F7EEFA8F
:1021600000212046F7F700FB0E4C4021204607F0E7
:1021700007FA0028F9D04FF480710B48F8F769F995
:10218000074C0A49A83C2046F7F7D8FA0121204617
:10219000F7F7EAFA06490120087110BD008000280F
:1021A000B860024000500040000002402080001053
:1021B0001008002010B5124C10492046F7F7BEFA5F
:1021C00000212046F7F7D0FA0E4C4021204607F0B8
:1021D000D7F90028F9D04FF480610B48F8F739F9A6
:1021E000074C0A49303C2046F7F7A8FA012120465F
:1021F000F7F7BAFA06490120087110BD00800018EF
:102200005860024000480040000C02400088001066
:10221000100800202DE9F047012190B0480504F096
:1022200053FD8648F7F7AAFA402738010024CDE984
:102230000540C50107940894CDE9094546040C946E
:102240000D94DFF8FC917F480B94CDE90207CDE9AE
:10225000006969460E947948F7F738FB012210218E
:102260007648F7F71DFBDFF8D4A1AAF1180A50460B
:10227000F7F784FA4FF47A78CDE90348E811CDE90D
:10228000054007940894CDE909456F480B940C94D8
:102290000D9400960E94CDE9019069465046F7F7EB
:1022A00015FB01215046F7F75FFADFF890A1AAF17C
:1022B000300A5046F7F762FAE811CDE90540079475
:1022C0000894CDE909450C940D94DFF8809160489D
:1022D0000B94CDE90207CDE9006969460E9450469A
:1022E000F7F7F4FA012210215046F7F7D9FADFF890
:1022F0004CA1AAF1600A5046F7F740FACDE903482D
:10230000E811CDE9054007940894CDE90945514805
:102310000B940C940D9400960E94CDE901906946AF
:102320005046F7F7D3FA01215046F7F71DFADFF8C8
:102330000CA10AF1180A5046F7F720FAE811CDE986
:10234000054007940894CDE909450C940D94DFF8F5
:10235000089142480B94CDE90207CDE9006969462E
:102360000E945046F7F7B2FA012210215046F7F7C3
:1023700097FADFF8C8A0AAF1900A5046F7F7FEF9DD
:10238000CDE90348E811CDE9054007940894CDE96B
:10239000094533480B940C940D9400960E94CDE9A6
:1023A000019069465046F7F791FA01215046F7F738
:1023B000DBF9DFF88890A9F148094846F7F7DEF91C
:1023C0000397E811CDE9054007940894CDE9094544
:1023D00025480B940C940D94224F00960E94CDE951
:1023E000017069464846F7F771FA01221021484604
:1023F000F7F756FADFF84490A9F178094846F7F75D
:10240000BDF9CDE90348E811CDE9054007940894EA
:10241000CDE9094515480B940C940D9400960E9443
:10242000CDE9017069464846F7F750FA0121484660
:10243000F7F79AF910B0BDE8F0870000A0600240FD
:102440000444004080590020E0620020044C004019
:10245000D85B0020C866002004500040305E002099
:10246000B06A00200448004088600020986E002078
:102470002DE9FC410121084604F026FC012104203D
:1024800004F022FC0121082004F01EFC0121402060
:1024900004F01AFCDFF8FC80072205214046F7F71C
:1024A000BFFF072206214046F7F7BAFF072208219F
:1024B0004046F7F7B5FF072209214046F7F7B0FF7E
:1024C000354F08220A213846F7F7AAFF08220B21C8
:1024D0003846F7F7A5FF082202214046F7F7A0FF8C
:1024E00008220C213846F7F79BFF02268DF805607D
:1024F00000244FF459708DF80640012500908DF8A6
:1025000007508DF8046069464046F7F74DFF8DF897
:1025100005604FF4E0508DF8064000908DF80750AC
:102520008DF8046069463846F7F73EFF4FF4916036
:1025300000908DF806408DF8045069464046F7F744
:1025400033FF280200908DF806408DF8045069464C
:102550001248F7F729FF8DF806404FF4F040104C71
:1025600000908DF8045069462046F7F71DFFA90337
:102570002046F7F76CFF69032046F7F768FFA114C0
:102580002046F7F764FFE1142046F7F760FFBDE847
:10259000FC810000000C02400008024000000240E4
:1025A0000018024070B50024FFF762FFFFF732FE0B
:1025B00000F022F80E4D002185F8E01A012285F87E
:1025C000E02A0C48017081704170C2704FF47A713A
:1025D0008160042085F8E00A04E0204600F062F9FA
:1025E000641CE4B295F8E00AA042F6D870BD000081
:1025F000D422002084550020F8B511208DF8000069
:1026000002258DF8015001248DF802408DF8034019
:10261000684600F047FB26208DF800008DF8014049
:1026200000268DF802608DF80340684600F03AFB02
:102630000E208DF800008DF801508DF802408DF8C5
:102640000340684600F02EFB27208DF800008DF82F
:1026500001408DF802608DF80340684600F022FBCF
:102660000F208DF800008DF801508DF802408DF894
:102670000340684600F016FB34208DF800008DF80A
:1026800001408DF802608DF80340684600F00AFBB7
:102690002F208DF800008DF801508DF802408DF844
:1026A0000340684600F0FEFA35208DF800008DF8F2
:1026B00001408DF802608DF80340684600F0F2FAA0
:1026C000F8BD01B9102110F8012B10F8013B491E8B
:1026D0005A400904090CF8D102F07F00704700004D
:1026E0002DE9FF5F14460F464FF480564FF4806883
:1026F0004FF4C0694FF00C0A40F2244B002580B122
:10270000012830D0022851D0032871D1012188043A
:1027100004F0FEFA0097012C6DD0022C70D094B317
:1027200077E00121480404F0F3FA0097012C03D06C
:10273000022C06D054B10DE0ADF80460ADF808806D
:1027400008E0ADF80460ADF8089003E0ADF804507F
:10275000ADF80850ADF80650ADF80C50ADF80AA031
:1027600069463B4C5DE00121C80404F0D1FA0097B2
:10277000012C03D0022C07D05CB10EE0ADF8046050
:10278000ADF8088009E040E0ADF80460ADF80890CD
:1027900003E0ADF80450ADF80850ADF80650ADF8C0
:1027A0000C50ADF80AA069462A4C3AE00121080510
:1027B00004F0AEFA0097012C03D0022C06D054B1DD
:1027C0000DE0ADF80460ADF8088008E0ADF80460F5
:1027D000ADF8089003E0ADF80450ADF80850ADF83E
:1027E0000650ADF80C50ADF80AA069461A4C18E036
:1027F0002CE000E004E0ADF80460ADF8088008E0EB
:10280000ADF80460ADF8089003E0ADF80450ADF801
:102810000850124CADF80650ADF80C50ADF80AA0B7
:102820006946204606F0EAFE0121204606F04FFEEA
:1028300001225946204606F0C9FE1021204606F026
:1028400043FE0122C021204606F04BFEBDE8FF9F5B
:1028500000440040004C0040005000400048004050
:102860002DE9FC410024CDE900446F466422002399
:10287000F5F7A8FC0E460546104619460A22002325
:10288000F5F7A0FC010102F00F000818385504F11B
:102890000104E4B228463146082CE7D3DDE9000103
:1028A000BDE8FC812DE9F84F8C4E804600250420C0
:1028B00086F8E00A08EB480101EB0810A6F58057FE
:1028C00007EB0014009404F5805494F8910B012850
:1028D00003D10021404600F009F908EB4802BA464E
:1028E00007EB8207A7F21C5707F500574FF00009C6
:1028F00087F8009087F8029087F8019087F8039096
:102900000521B96087F8309087F83290012087F868
:10291000310087F83300D4F88C0B00EB80004000C6
:10292000B86394F8892BD4F8841B4046A7F6E427B3
:10293000FFF7D6FE94F88A1B08EB081202EB08207A
:10294000674A072902EBC00B0BF5005015D2DFE8F0
:1029500001F01404060A0C0E1A00052100E00F21F4
:1029600080F8481009E00721FAE70421F8E7D4F8D5
:102970008C1B64225143C7F81C1B9AF81410D046D4
:10298000012902D017E00321EAE780F848900120EE
:10299000C7F8EC0A534F80213846F7F75AFD082153
:1029A0003846F7F756FDB9154F48F7F752FD391578
:1029B0003846F7F74EFD4FF0A10EC24669E005EB31
:1029C000051300210BEBC3004C3000F500500173E0
:1029D000012383734173C173D4F88C3B94F88B7BD0
:1029E0007B4303EB83039B004361009B03EB0513D5
:1029F00003F5805383F8B61B00F84C1994F88A1B32
:102A0000072944D2DFE801F0430408080A0C0E004D
:102A1000E52180F851103AE07146FAE7B121F8E774
:102A20003121F6E7F12180F8511000212BE001EB74
:102A3000011202EB01220AEBC20701EB410202EB99
:102A400001120AEB0212002002F5805915E002EB98
:102A5000001C0CF5805C9CF8B4CB93F8BC8BC4458F
:102A600009D193F8B4CB00EB001807EBC80808F5C0
:102A7000005888F8C3C0401CC0B299F88BCB84457D
:102A8000E5D8491CC9B296F8E00A8842CFD86D1C37
:102A9000EDB294F88B0B5246A84290D8002086F8ED
:102AA000E10A00EB400101EB001102EB011101F51D
:102AB000805191F88A3B052B09D291F88A3B33B1BA
:102AC00096F8E13A91F88B1B194486F8E11A401CFC
:102AD000C0B20428E5D3BDE8F88F0000D42200205E
:102AE000D4120020000C0240000002402DE9F04109
:102AF000054663484FF480425310066861488414C9
:102B0000C71439B1C5B1012D18D0022D18D0032D2D
:102B10001BD117E035B1012D06D0022D06D0032DB3
:102B200013D105E0114604E0194602E0214600E019
:102B30003946F7F78EFC08E0114604E0194602E03A
:102B4000214600E03946F7F782FC642008F0D8F906
:102B500000224FF416512846FFF7C2FD4A4905EB03
:102B6000450001EB800000F58050002280F8162B14
:102B7000C0F8182B05EB450000EB051001EB001029
:102B800000F58050D0F88C3B01F58041C1F8B83297
:102B9000012381F8B13290F88A1B3C4C962305EB57
:102BA0008500204406290AD2DFE801F00903050563
:102BB0000733762102E0837001E06E218170C5EB5E
:102BC0000511334B01EB8101C02403F8314003EBC5
:102BD000C10462700821A170E27006F00F0105EBDC
:102BE000051211442171807860712020A071E1717B
:102BF000802020724C2060725420A0722548264FFD
:102C00000B2645B1012D0FD0022D25D0032D14D157
:102C10002DE06621D2E78021F7F719FCC7F8A46000
:102C20001D480121A03006E00821F7F710FC7E675F
:102C3000194801217030F6F797FD184890F8A7035E
:102C400028B1204600232A460B21F7F7C5FEBDE830
:102C5000F041642008F054B94FF480711048F7F740
:102C6000F6FBC7F8BC600C480121B830E3E74FF42D
:102C70008061F7F7ECFBFE65074801215830DAE781
:102C8000187AFF1F00180240D41200208072002022
:102C900080590020000C024000600240D422002035
:102CA0000000024030B50F23C27801780125FAB147
:102CB000144A126801F1E02102F4E062C2F5E06218
:102CC000C2F30722C2F10404D3404278A2408478C0
:102CD0001C401443220181F80024007800F01F01F9
:102CE0008D404009800000F1E020C0F8005130BD67
:102CF00001F01F0085404809800000F1E020C0F885
:102D0000805130BD0CED00E0024A11400143024801
:102D10000160704780FFFF1F08ED00E010B5002143
:102D2000074B0A46002003EBC004401CC0B26254AB
:102D30008028F8D3491CC9B20829F3D310BD00007C
:102D4000837C00202DE9FE4F0026171A8146701E55
:102D50003546A3EB010A8846002F02DD4FF0010142
:102D600002E003D14FF00001019102E0C7F100073A
:102D70000190BAF1000F02DD4FF0010002E003D133
:102D80004FF00000009002E0C7F1000A00905046AA
:102D9000574501DD3C4600E00446601C4FF0000B47
:102DA000029016E008F0FF0109F0FF000C9A00F015
:102DB00015F83E445544A64202DD0199361B89446C
:102DC000A54202DD00992D1B88440BF101001FFA7A
:102DD00080FB02998B45E5DBBDE8FE8F30B5CC0862
:102DE00001F0070301259D40EBB2064D05EBC00540
:102DF000C808285C0AB1184302E063EA0000C04337
:102E0000285530BD837C00202DE9FC4101210A209A
:102E100003F05AFF01248DF8044000264FF4C050FF
:102E20008DF80660032700908DF805708DF8074037
:102E300069464648F7F7B8FA8DF804408DF8066001
:102E40008DF80570A5028DF80740414C0095694644
:102E50002046F7F7A9FAC82008F052F8294620467C
:102E6000F7F7F5FAC82008F04BF829462046F7F79F
:102E7000F0FAC82008F044F80021FD2000F04AFADA
:102E80000021122000F046FA0021AE2000F042FAA4
:102E90000021D52000F03EFA0021A02000F03AFAEF
:102EA0000021A82000F036FA00213F2000F032FA7D
:102EB0000021D32000F02EFA0021084600F02AFA63
:102EC0000021402000F026FA0021A02000F022FA84
:102ED0000021C02000F01EFA0021DA2000F01AFACA
:102EE0000021122000F016FA0021812000F012FAD1
:102EF00000217F2000F00EFA0021D92000F00AFA0C
:102F00000021822000F006FA0021DB2000F002FA06
:102F10000021342000F0FEF90021A42000F0FAF98D
:102F20000021A62000F0F6F90021202000F0F2F99F
:102F30000021084600F0EEF9FFF7F0FE0021AF2077
:102F400000F0E8F900F054F8BDE8FC81000C024004
:102F5000000402400346012000E05843491EC9B264
:102F6000FBD270472DE9F84F82460A980D46504330
:102F70006421B0FBF1F0984600F0FF0B4FF001091F
:102F80000AEB02072B4600245046FAB21946CDF848
:102F90000090FFF7D7FE05EB0806F3B2FAB2F1B2E4
:102FA0005046CDF80090FFF7CDFE5246F3B22946C9
:102FB0001046CDF80090FFF7C5FEF3B2FAB2F8B2B2
:102FC0002946CDF80090FFF7BDFE4F460AEB0B06F1
:102FD00009E02819C3B2C1B2F2B250460097FFF718
:102FE000B1FE641CE4B24445F3D3BDE8F88F0000A1
:102FF00070B50025B020294600F08CF90021084664
:1030000000F088F90021102000F084F9084E002417
:1030100006EBC4000121405D00F07CF9641CE4B2C1
:10302000802CF5D36D1CEDB2082DF0D370BD0000DF
:10303000837C002070B50B4C05460221204604F02D
:103040000DF80028F9D02946204604F010F8012197
:10305000204604F003F80028F9D0204604F005F8D3
:10306000C0B270BD003800402DE9FC4F1D468846B7
:1030700081468B460090082B0ED0680700D00120B7
:1030800000EBD500690810FB01F0C0B2203A02F055
:10309000FF0A0026019046E00620F7E7082D10D031
:1030A0000C2D14D0102D16D0182D3FD121490AEB2C
:1030B000CA0001EB80000027845DE0070FD00B9A67
:1030C00010E01D490AEB4A0001EB4000F3E70AEB70
:1030D0004A001A49EDE71A4901EB0A10EBE70B9891
:1030E00030B3002241464846FFF778FE7F1C640853
:1030F00008F10100FFB200F0FF08082FDDD309F14D
:10310000010000F0FF09082D0AD00099A9EB010089
:10311000B0EB550F04D10BF10800894600F0FF0B0E
:10312000761CD846F6B201988642B7D3BDE8FC8F2C
:103130000122D7E7ECCB010860BF010888C1010874
:10314000FCC501082DE9FF4F81B04FF00007DDE914
:103150000F8A1E00934681463D4611D11046F5F771
:1031600041FA41EC100B06F0DFFC9FED2F1B51ECF8
:10317000100B53EC112BF5F79CF8F5F754FAC6B287
:10318000B8F1080F00D1022700243AE00E98301A57
:10319000A0420AD107EB580101FB0490C0B243469C
:1031A0004FF02E02CDF800A03BE002DA4FF001050F
:1031B00001E04FF0000506EB0500A0EB0400A0F1D4
:1031C0000100C1B24FF00A00FFF7C4FEBBFBF0F0F4
:1031D0000A21B0FBF1F201FB1200CDF800A0B8B15A
:1031E00005EB090207EB580101FB042101F0FF0C7C
:1031F0003030C2B2434660460299FFF735FF641C87
:10320000E4B27019A042C1D805B03046BDE8F08FD5
:1032100005EB090107EB580000FB0410C0B2434660
:1032200030220299E9E70000000000000000F03FB2
:103230002DE9FF4F81B0064600900F464FF0000A7F
:103240008946580700D0012000EBD30004900020ED
:1032500032E0002029E00E98002410F80A500AF10C
:1032600001001FFA80FAE80701D00F9A02E00F98D8
:1032700048B3002239463046FFF7B0FD7F1C641C7E
:103280006D08E4B2FFB2082CEDD3761C0098F6B2BC
:10329000311A0398814204D109F10800009E00F020
:1032A000FF0908F101004F46C0B2039980468842E9
:1032B000D1D30BF10100C0B2049983468842C8D330
:1032C00005B0BDE8F08F0122D4E72DE9F8431D4693
:1032D000DDE908781646894604460EE03B46494635
:1032E0002046CDF80080FFF7BFFE082F0ED004EB7C
:1032F0005700C4B26D1EEDB2761C002D04D032789A
:10330000202A01D37E2AE9D9BDE8F883A41DE4B2BE
:10331000F0E700002DE9F041114C06464FF400653E
:1033200000292946204602D0F7F793F801E0F7F785
:103330008EF84FF4805739462046F7F788F839461B
:103340000848F7F786F83046FFF774FE39462046FE
:10335000F7F77FF829462046BDE8F041F7F779B83E
:10336000000C0240000402402DE9F04F89B04FF0FC
:10337000000B5E46ADF800B0ADF804B0ADF808B093
:10338000ADF80CB0ADF810B0ADF814B0F74C5D4628
:1033900094F8A106A4F580590106DFF8D4A309F535
:1033A0008040049071D4EEE394F86407022802D1BF
:1033B0000720ADF81400BDF8140051465044807940
:1033C000BDF814205244D27840EA0260BDF81420BF
:1033D00052441279BDF81430120453445B7942EA26
:1033E00003221043E34A536898424FD05060BDF81F
:1033F000140008448078BDF814200A44527840EA4A
:103400000227B4F82A26BDF814003844801C8242F2
:103410003CD3B4F82A06BDF81420C01B801A801EC5
:10342000A4F82A06BDF81400554650443946F6F76C
:1034300045F9BDF81410394429444978BDF81420E1
:103440003A44AA5C41EA022181427BD194F8A70365
:1034500040B1B81CBDF8142081B2A8180123042281
:10346000F7F7BAFABDF814102B462944097901F090
:1034700001010791BDF81410294489790025C1F391
:103480004201A7F10708069115E0FCE3A4F82A66BB
:1034900009B0BDE8F08FBDF814004119C818C07913
:1034A000DDE90621F6F70CFBBDF814104A19D11816
:1034B000C8716D1CADB24545EDDBBDF814109A46E0
:1034C0005818C079012184F86217C4F8686684F836
:1034D0006666049981F8A662C1F8A86294F8641738
:1034E000032903D094F86417012903D1A24A0121CA
:1034F000C2F88812ADF80C6011287DD00BDCA0F169
:103500000B00062813D2DFE810F0FE0861099C09C1
:103510009609B30B1E00A22870D004DC12286ED0CE
:10352000A12804D130E3A3286AD0A42869D00020C0
:103530005146BDF8142002448E54401C80B2052828
:10354000F7D3F6E3F6E3ADF80060F5E1BDF800006F
:103550004D4600EB400101EB001009EB001000F5B7
:10356000805090F88A0B07287DD2DFE800F07C04B9
:103570000404047CA600ADF804608CE0BDF81400DF
:10358000BDF80C10014401EB0A00007AA8B3012831
:1035900002D0022875D113E0BDF8000000EB400115
:1035A00001EB0010BDF8041005EB001000EB01105A
:1035B00041F6B6310844017821F00401017060E061
:1035C000BDF8000000EB400101EB0010BDF8041055
:1035D00005EB001000EB011041F6B631084401780C
:1035E00021F008010170BDF8000000EB400101EB83
:1035F000001005EB001005E0FDE342E0FCE3FCE316
:10360000FCE3FCE3BDF8041000EB011000F5805072
:10361000C0F8B86BBDF800100220F6F7E5FA0020FC
:10362000BDF8001001EB011202EB012105EBC10214
:10363000BDF8041001EB011102EBC101014401F5D9
:10364000005181F88B60401C80B21428E8D3002020
:10365000BDF8001001EB011202EB012105EBC102E4
:10366000BDF8041000E062E101EB011102EBC101C1
:10367000014401F5005181F8A760401C80B20A287E
:10368000E6D3BDF80C00401CADF80C00BDF80400FA
:10369000401CADF80400BDF8000000EB400101EB58
:1036A000001005EB001000F5805090F88B0BBDF872
:1036B000041088423FF662AF39E1ADF8046025E1BD
:1036C000BDF81400BDF80C10D44608446044007ADC
:1036D000042805D005DC58B101284FD002287DD13F
:1036E00032E108287BD010287AD0202876D1E7E173
:1036F000BDF8000000EB001101EB002005EBC0015C
:10370000BDF8040000EB001001EBC00000F5005014
:1037100090F8C200102824D1BDF8000000EB001181
:1037200001EB002005EBC001BDF8040000EB001028
:1037300001EBC00000F5005080F8C260BDF8000049
:10374000F32100EB001202EB002005EBC002BDF8F4
:10375000040000EB001002EBC00000F5005080F800
:103760005110BDF80C00401CC9E00000D42200201C
:1037700094720020180A002000004042BDF80000AA
:10378000F22100EB001202EB002005EBC002BDF8B5
:10379000040000EB001002EBC00000F5005080F8C0
:1037A0005110BDF8000000EB400101EB0010BDF826
:1037B000041005EB001000EB011041F6B63108448F
:1037C000017821F004010170BDF81400BDF80C105F
:1037D00008446044017ABDF8000002E091E0B3E0E3
:1037E000F2E000EB001202EB002005EBC002BDF896
:1037F000040000EB001002EBC00000F5005080F860
:10380000C2100020BDF81410BDF80C201144014472
:1038100061444A7ABDF8001001EB011303EB01216A
:1038200005EBC103BDF8041001EB011103EBC1016D
:10383000014401F5005181F89520401C80B20F2809
:10384000E0D30020BDF81410BDF80C201144014451
:1038500061440A7EBDF8001001EB011303EB012166
:1038600005EBC103BDF8041001EB011103EBC1012D
:10387000014401F5005181F8A720401C80B20A28BC
:10388000E0D3BDF81400BDF80C100844604490F873
:103890002210BDF8000000EB001202EB002005EB47
:1038A000C002BDF8040000EB001002EBC00000F500
:1038B000005080F8BC100020BDF81410BDF80C209A
:1038C00011440144614491F82320BDF8001001EB3C
:1038D000011303EB012105EBC103BDF8041001EB5B
:1038E000011103EBC101014401F5005181F8BD2034
:1038F000401C80B20528DFD3BDF80C002030ADF8A5
:103900000C00BDF80400401CADF80400BDF8000038
:1039100000EB400101EB001005EB001000F58050BA
:1039200090F88B0BBDF8041088423FF6C9AEBDF885
:103930000000401CADF8000094F8E00ABDF800104B
:1039400088423FF603AEFCE5BDF80000F22100EB33
:10395000001202EB002005EBC002BDF8040000EBF2
:10396000001002EBC00000F5005080F85110BDF8C7
:10397000000000EB400101EB0010BDF8041005EB66
:10398000001000EB011041F6B6310844017821F037
:1039900004010170BDF81400BDF80C100844504437
:1039A000017ABDF8000000EB001202EB002005EBED
:1039B000C002BDF8040000EB001002EBC00000F5EF
:1039C000005080F8C210CCE6BDF80000F32100EBF7
:1039D000001202EB002005EBC002BDF8040000EB72
:1039E000001002EBC00000F5005080F85110BDF847
:1039F000000000EB400101EB0010BDF8041005EBE6
:103A0000001000EB011041F6B6310844017821F0B6
:103A100004010170BDF81400BDF80C1008446044A6
:103A2000017ABDF8000000EB001202EB002005EB6C
:103A3000C002BDF8040000EB001002EBC00000F56E
:103A4000005080F8C210BDF81400BDF80C100844F6
:103A50006044417ABDF8000000EB001202EB002048
:103A600005EBC002BDF8040000EB001002EBC00043
:103A700000F5005080F8BC100020BDF81410BDF80F
:103A80000C201144014461448A7ABDF8001001EB16
:103A9000011303EB012105EBC103BDF8041001EB99
:103AA000011103EBC101014401F5005181F8BD2072
:103AB000401C80B20528E0D3BDF80C00C01D1EE7F5
:103AC000BDF80000F22100EB001202EB002005EB34
:103AD000C002BDF8040000EB001002EBC00000F5CE
:103AE000005080F85110BDF8000000EB400101EBE0
:103AF0000010BDF8041005EB001000EB011041F6BA
:103B0000B6310844017821F004010170BDF81400B9
:103B1000BDF80C1008446044017ABDF8000000EBC9
:103B2000001202EB002005EBC002BDF8040000EB20
:103B3000001002EBC00000F5005080F8C210002019
:103B4000BDF81410BDF80C201144014461444A7AB8
:103B5000BDF8001001EB011303EB012105EBC103DC
:103B6000BDF8041001EB011103EBC101014401F5A3
:103B7000005181F8BD20401C80B20428E0D3BDF87C
:103B80000C00401DBBE6FDE3B91E0D2091FBF0F0DB
:103B9000C0B20790ADF80060D6E1B046ADF8046061
:103BA0004D46ABE1BDF8000000EB400101EB001019
:103BB000BDF8041005EB001000EB011000F580507B
:103BC00090F8B60B80077DD40BEB8B0101EBCB009B
:103BD000BDF81410014401EB0A00007A0021FEF741
:103BE0008BF9BDF8002002EB420303EB0212BDF893
:103BF000043005EB021202EB031202F5805292F838
:103C0000B42B424088EA010002435BD1BDF80000BA
:103C100000EB001101EB002005EBC001BDF8040032
:103C200000EB001001EBC00000F5005090F8890097
:103C300001287DD1BDF8141050465144497BBDF890
:103C400014205244927A41EA0262BDF814105144A1
:103C5000C97ABDF81430090453441B7B41EA03219F
:103C60000A43BDF8001001EB011303EB012105EB42
:103C7000C103BDF8041001EB011103EBC10101F513
:103C800000514A6500E0FDE3BDF814100144097DD0
:103C9000BDF814200244527C41EA0261BDF81420B0
:103CA0000244927CBDF8143012040AEB0300C07C7D
:103CB00042EA00200143BDF8000000EB400202EBA5
:103CC000001000E015E1BDF8042005EB001000EB4A
:103CD000021000F58050C0F8B81BBDF8000000EBE2
:103CE000400101EB0010BDF8041005EB001000EBE3
:103CF000011041F6B6310844017841F0200101700D
:103D0000BDF800100220F5F76FFFBDF8000000EBD2
:103D1000400101EB0010BDF8041005EB001000EBB2
:103D2000011000F5805090F8B41BBDF8000002E0CF
:103D300068E010E1E5E300EB001202EB002005EB88
:103D4000C00000F5005080F84510BDF8000000EB01
:103D5000400101EB001005EB001000F5805090F8D9
:103D60008A0B012804D002284FD003284AD14CE006
:103D7000BDF814100AEB0100407A10B1012841D1BE
:103D800041E0BDF8000000EB400101EB001005EB45
:103D9000001000F5805090F8900B0028BDF800004E
:103DA00000EB001101EB002005EBC001BDF80400A1
:103DB00000EB001001EBC00000F50050406D03D097
:103DC000B0F1104F03D104E0B0F5100F01D0B521D0
:103DD00000E0C321BDF8000000EB001202EB002060
:103DE00005EBC002BDF8040000EB001002EBC000C0
:103DF00000F5005004E0FDE37CE1FCE3CAE2ABE047
:103E000080F851106EE0B921E4E7BDF8000000EB46
:103E1000001101EB002005EBC001BDF8040000EB30
:103E2000001001EBC00000F5005090F84C10BDF8F8
:103E3000000000EB001202EB002005EBC00000F5D3
:103E4000005090F8480081424CD1BDF81400504415
:103E5000807BBDF8142000045244D27B40EA022249
:103E6000BDF814005044007C0243BDF8000000EB94
:103E7000001303EB002005EBC003BDF8040000EBCA
:103E8000001003EBC00000F50050C0F88020BDF822
:103E900014005044417ABDF8000000EB001202EB20
:103EA000002005EBC002BDF8040000EB001002EB9F
:103EB000C00000F5005080F85210BDF80000A421A9
:103EC00000EB001202EB002005EBC002BDF804007D
:103ED00000EB001002EBC00000F5005080F84E101F
:103EE000A32177E70BF10100079900F0FF0B8B4549
:103EF00015D2BDF80400401CADF80400BDF8000068
:103F000000EB400101EB001005EB001000F58050C4
:103F100090F88B0BBDF8041088423FF643AEBDF815
:103F2000000000EB400101EB001105EB011000F572
:103F3000805090F88B0BBDF8041088420BD8BDF868
:103F40000000401CADF8000094F8E00ABDF8001035
:103F500088423FF622AE22E1ADF800604BE0ADF8BA
:103F60000460B0464D4621E0BDF814100AEB010094
:103F7000007A0021FDF7C0FFBDF8002002EB4203EC
:103F800003EB021305EB0312BDF8043002EB03123E
:103F900002F5805292F8B42B424088EA01000243B5
:103FA00030D0BDF80400401CADF80400BDF800009E
:103FB00000EB400101EB001105EB011000F5805012
:103FC00090F88B0BBDF804108842CDD8BDF80000E6
:103FD00000EB400101EB001105EB011000F58050F2
:103FE00090F88B0BBDF804108842B4D8BDF80000DF
:103FF000401CADF8000094F8E00ABDF800108842BB
:10400000ADD8CCE0BDF80000BDF8042000EB4001C5
:1040100001EB0010294605EB001000EB021000F543
:10402000805090F8B42BBDF8000000EB001303EBB8
:10403000002005EBC00000F5005080F84520BDF8D9
:10404000000000EB400202EB001005EB001000F551
:10405000805090F88A0B012838D0022801D003281C
:10406000B4D1BDF8000000EB001202EB002001EB20
:10407000C002BDF8040000EB001002EBC00000F528
:10408000005090F84C20BDF8000000EB001303EB4B
:10409000002001EBC00000F5005090F8480082427B
:1040A00094D1BDF80000AA2200EB001303EB00201E
:1040B00001EBC003BDF8040000EB001003EBC000EF
:1040C00000F5005080F84E20A32200E0CA22BDF87F
:1040D000000000EB001303EB002005EBC001BDF86E
:1040E000040000EB001001EBC00000F5005080F868
:1040F00051206BE7ADF800604BE0ADF8046023E0C1
:10410000BDF814100AEB0100007AB0460021FDF75B
:10411000F3FEBDF8002002EB420303EB021309EBB0
:104120000312BDF8043002EB031202F5805292F83C
:10413000B42B88EA0108424052EA080230D0BDF8A8
:104140000400401CADF80400BDF8000000EB400185
:1041500001EB001109EB011000F5805090F88B0B7A
:10416000BDF804108842CBD8BDF8000000EB400138
:1041700001EB001109EB011000F5805090F88B0B5A
:10418000BDF8041088420AD8BDF80000401CADF804
:10419000000094F8E00ABDF800108842ADD872E142
:1041A000BDF80000BDF8042000EB400101EB001059
:1041B000494609EB001000EB021000F5805090F822
:1041C000B42BBDF8000000EB001303EB002009EB5B
:1041D000C00000F5005080F84520BDF8142052447E
:1041E000527ABDF81430120453449B7A42EA0322F7
:1041F000BDF814300AEB0300C07A0243BDF800009A
:1042000000EB001303EB002001EBC003BDF804003A
:1042100000EB001003EBC00000F50050C0F8802058
:10422000BDF8000000EB400202EB001001EB0010B3
:1042300000F5805090F88A0B01284AD0022801D05E
:10424000032891D1BDF8000000EB001202EB002022
:1042500001EBC002BDF8040000EB001002EBC0004F
:1042600000F5005090F84C20BDF8000000EB001362
:1042700003EB002001EBC00000F5005090F848006F
:104280008242DED1BDF80000A52200EB001303EB53
:10429000002001EBC003BDF8040000EB001003EBAD
:1042A000C00000F5005080F84E20BDF80000A322A9
:1042B00000EB001303EB002009EBC001BDF8040084
:1042C00000EB001001EBC00000F5005080F8512019
:1042D0004AE7BDF8000000EB001202EB002001EB02
:1042E000C002BDF8040000EB001002EBC00000F5B6
:1042F000005090F84C20BDF8000000EB001303EBD9
:10430000002001EBC00000F5005090F84800824208
:10431000DED1BDF80000B22200EB001303EB002059
:1043200001EBC003BDF8040000EB001003EBC0007C
:1043300000F5005080F84E20BDF80000E52200EBAB
:10434000001303EB002001EBC003BDF8040000EBF9
:10435000001003EBC00000F5005080F85120002D44
:10436000B6D1BDF804000128B2D1BDF8000000EBC1
:10437000001202EB002009EBC001BDF8040000EBC5
:10438000001000E0F7E301EBC00000F50050D0F8AA
:104390008000E9E6BDF8140055465044007A05282F
:1043A00071D2BDF814002844007A401EADF8000018
:1043B0000020BDF8001001EB410202EB011109EBF6
:1043C000011101EB001101F5805181F8B46BBDF8CA
:1043D000001001EB410303EB011109EB011101EBAB
:1043E000001101F5805181F8B56B401C80B2102896
:1043F000DFD3BDF814002844807B0021FDF77CFD4D
:1044000008437DD0BDF81400AA462844407ABDF880
:10441000141000042944897A40EA0120BDF81410E0
:104420002944C97A0843C117FDF766FDBDF800109D
:1044300001EB410202EB011209EB021101F580517F
:10444000C1F8840BBDF814002844007BB04600215D
:10445000FDF752FDBDF8001001EB410202EB011225
:1044600009EB021101F5805181F8880BBDF81400A9
:104470002844407B0021FDF73FFDBDF8001001EB13
:10448000410201E0F3E3A1E202EB011209EB0211A8
:1044900001F5805181F8890BBDF814002844807B18
:1044A0000021FDF729FDBDF8001001EB410202EBF0
:1044B000011209EB021101F5805181F88A0BBDF858
:1044C00014002844C07B0021FDF716FDBDF8001044
:1044D00001EB410202EB011209EB021101F58051DF
:1044E00081F88B0BBDF814002844007C0021FDF7F7
:1044F00003FDBDF8001001EB410202EB011201E0E7
:10450000EBE0DFE309EB021101F58051C1F88C0B00
:10451000BDF814002844407C0021FDF7EDFCBDF8F7
:10452000001001EB410202EB011209EB021101F54F
:10453000805181F8900BBDF8000000EB400101EBC9
:10454000001109EB011000F5805090F88A0BADF8CE
:1045500004800628C84660D0AEE0BDF81400BDF85F
:104560000410014401EB0A00807C0021FDF7C4FC2B
:10457000BDF804100325B1FBF5F2BDF8001001EB06
:10458000410303EB011308EB031101EB021101F5E9
:10459000805181F8B40BBDF81400BDF8041001443B
:1045A00001EB0A00C07C0021FDF7A6FCBDF8041059
:1045B000B1FBF5F2BDF8001001EB410303EB011371
:1045C00008EB031101EB021101F5805181F8B50BE5
:1045D000BDF81400BDF80410014401EB0A00007D91
:1045E0000021FDF789FCBDF80410B1FBF5F2BDF820
:1045F000001001E0ECE1F4E101EB410303EB0113F6
:1046000008EB031101EB021101F5805181F8BC0B9D
:10461000BDF80400C01CADF80400BDF8000000EBBC
:10462000400101EB001108EB011000F5805090F8FB
:104630008B0BBDF8041000EB400088428DD84CE095
:10464000BDF81400BDF80410554608442844807C89
:104650000021FDF751FCBDF8001001EB410202EB17
:10466000011208EB0211BDF80420520801EB0211FF
:1046700001F5805181F8B40BBDF81400BDF80410A9
:1046800008442844C07C0021FDF736FCBDF800102A
:1046900001EB410202EB011208EB0211BDF804200C
:1046A000520801EB021101F5805181F8B50BBDF8FC
:1046B0000400801CADF80400BDF8000000EB4001D0
:1046C00001EB001108EB011000F5805090F88B0B06
:1046D000BDF80410B1EB400FB2D3BDF800100220BA
:1046E000F5F782FABDF80000C0B2FEF7DBF8BDF8BE
:1046F0000000012100EB400209EB820000F5805030
:1047000080F87116D4E2BDF8140055465044007A82
:1047100084F8AD03BDF814005044407A84F8AC032B
:10472000BDF814005044807A84F8AB03BDF814003F
:104730005044C07A84F8AA03BDF814002844007BD2
:1047400084F8A903BDF814002844407B84F8A8032A
:1047500004F56A74F5F76AF9F5F72CF92078A4F5F1
:104760006A74FF2829D1F5F7DBF8BDF81400284456
:10477000007A84F8AD03BDF814002844407A84F828
:10478000AC03BDF814002844807A84F8AB03BDF86C
:1047900014002844C07A84F8AA03BDF81400284401
:1047A000007B84F8A903BDF814002844407B84F8FA
:1047B000A803F5F73BF9F5F7FDF8D9F8540008B16F
:1047C0000F2000E00E2084F8660771E2102084F8C4
:1047D0006607BDF8141050465144097A84F8AD13A9
:1047E000BDF814105144497A84F8AC13BDF8141084
:1047F0005144897A84F8AB13BDF814105144C97A36
:1048000084F8AA13BDF814100144097B84F8A91395
:10481000BDF814100AEB0100407B84F8A80304F5EE
:104820006A74F5F703F902F0F9FAA060A068A068CD
:10483000A4F56A743CE20E2084F8660784F8A1614E
:1048400036E2ADF800604D463EE0ADF8046016E09B
:10485000BDF8000000EB400101EB0010BDF80410B2
:1048600005EB001000EB011000F5805090F8B60B3E
:10487000C00714D1BDF80400401CADF80400BDF819
:10488000000000EB400101EB001005EB001000F50B
:10489000805090F88B0BBDF804108842D8D8BDF832
:1048A000000000EB400101EB001005EB001000F5EB
:1048B000805090F88B0BBDF80410884208D8BDF8E2
:1048C0000000401CADF80000BDF800000428BCD377
:1048D000BDF80000042870D3F84A5670F84901204A
:1048E000C1F88802C1F8880294F8A50100286ED0AA
:1048F0000D2084F86607BDF8140053465044407AF2
:10490000BDF814105144097A40EA0120ADF80800BE
:10491000BDF814005044C07ABDF814105144897A8F
:1049200040EA0120508000204FF40078BDF81410B8
:1049300001441944097B05EB000C0CF5805C8CF8F4
:10494000A611401C80B24045F0D35088904600F23A
:10495000FF3081B20120F4F73DFB002837D084F806
:10496000A161B8F8021064225143BDF80820B1FBE0
:10497000F2F184F8A0110121A971B8F80210491CC4
:10498000A8F80210B8F80200BDF8081088421ED935
:1049900094F89C0140F0010084F89C0194F89C017B
:1049A00020F00600801C84F89C01BDF80800A4F8E3
:1049B0009E010021012052E1FFE7102084F86607E4
:1049C00094F89C0140F0800084F89C0170E19FE025
:1049D000BDF814100AEB0100007A84F8A10111203F
:1049E000F1E6ADF800603EE0ADF8046016E0BDF819
:1049F000000000EB400101EB0010BDF8041009EBD2
:104A0000001000EB011000F5805090F8B60BC007C5
:104A100014D1BDF80400401CADF80400BDF800003E
:104A200000EB400101EB001009EB001000F5805095
:104A300090F88B0BBDF804108842D8D8BDF8000060
:104A400000EB400101EB001009EB001000F5805075
:104A500090F88B0BBDF80410884208D8BDF8000010
:104A6000401CADF80000BDF800000428BCD3BDF820
:104A7000000004287ED3DFF844C28CF8016090491E
:104A80004FF00108C1F88882C1F8888294F8A50126
:104A9000F0B3122084F86607BDF814005546504460
:104AA000007A84F8A10194F8A101401EADF800003D
:104AB0000020BDF81410014429444A7ABDF80010C2
:104AC00001EB410303EB011109EB0111014401F575
:104AD000805181F8922B401C80B20A28E9D3BDF89E
:104AE00014002844007DBDF814102944C97C40EA14
:104AF0000120ADF80800BDF814002844807DBDF801
:104B000014102944497D40EA0120ACF8020000E07D
:104B10005CE000204FF40071BDF8142002442A44E8
:104B2000D37D09EB000202F5805282F8A631401CC9
:104B300080B28842F0D3BCF802006546BDF8001090
:104B400000EB8120401E81B20320F4F743FAE8B362
:104B50006988284664225143BDF80820B1FBF2F170
:104B600084F8A0114A4689F806806988491C698042
:104B7000698801E09CE0C9E0BDF80830994243D95A
:104B8000002041F6BD33BDF8001001EB410505EBF7
:104B9000011102EB011101EB001119440D7845F0F0
:104BA00001050D70401C80B21028ECD3BDF8000048
:104BB00000EB400101EB001002EB001041F69C31CC
:104BC0000844037843F00103037000E049E0BDF8B6
:104BD000000000EB400303EB001002EB0010084460
:104BE000017821F00601891C0170BDF80810BDF89C
:104BF000000000EB400303EB001009EB001000F590
:104C00008050A0F89E1B27E04088012829D1002071
:104C100041F6BD33BDF8001001EB410505EB011174
:104C200002EB011101EB001119440D7825F001058B
:104C30000D70401C80B21028ECD3BDF8000000EBD2
:104C4000400101EB001009EB001141F69C300844D3
:104C5000017821F001010170BDF800100220F4F785
:104C6000C3FF1748C0F88862C0F8886220E045E0BA
:104C7000D9F854004D460A21B0FBF1F1BDF81420DB
:104C80005244127A914213D1BDF814100AEB01007C
:104C9000007A18B1686D0A38686503E06E65102007
:104CA00084F8660700210520F4F79EFF0120A87113
:104CB000B4F82A0610B3002051461BE0180A002061
:104CC0000000424200202946BDF8142002448E54C0
:104CD000401C80B20528F7D3FEF7D8BBBDF81420DE
:104CE0003A4402440A449278BDF814300344CA544A
:104CF000401C80B2B4F82A268242EFD8B4F82A06C3
:104D000000287EF451AB09B0BDE8F08F94F8640739
:104D10004FF47A78B8B101287ED0DFF8F8B3FE49B5
:104D2000FE4F0891022878D00328ECD194F8A10610
:104D3000C0F3C3000928E6D2DFE800F014F8F72634
:104D4000F6F5F4F3F20094F8A106C0F3C3000E28C0
:104D5000D9D2DFE800F007EBEA19E92727EC39633D
:104D60008793D3DA94F8A10620F07800083087E121
:104D700094F8A10620F07800103081E194F8A106A3
:104D800020F0780018307BE1E5A118E194F8A10645
:104D900020F07800203073E194F8A10620F078002C
:104DA00028306DE1DEA1DF4806F04AFA0028AAD0DB
:104DB00094F8A10620F07800383061E194F8A1065B
:104DC00020F0780040305BE1D7A1D64806F038FAF1
:104DD000002898D04A46511901F5805181F8E966BA
:104DE0006D1CADB2142DF6D30021554643182B444B
:104DF0001E79531803F5805383F8EE66491C89B277
:104E00000F29F3D300210320F4F7EEFE94F8A10656
:104E100020F0780048307CE28AE03EE1C4A1C1483D
:104E200006F00EFA0028C2D04A46511901F5805109
:104E300081F8A2666D1CADB2142DF6D30021534645
:104E400045181D446E79551805F5805585F8A766F7
:104E5000491C89B20F29F3D394F8A10620F07800F9
:104E6000503056E2AEA1AF4806F0EAF900289ED0D5
:104E700094F8A10620F07800583001E194F8680712
:104E800058B194F8A10620F07800603084F8A106AB
:104E9000C4F84066012084F83E06A7A1A14806F0A8
:104EA000CFF9002895D0C4F84066012184F83E1659
:104EB00050445546417900793039303841EA001084
:104EC000C117FDF719F884F868079DA1954806F009
:104ED000B7F90028A7D029184A78302A06D349788C
:104EE000285C3038303941EA001001E0285C303865
:104EF000C117FDF701F884F8690704E788A189481C
:104F000006F09EF900287DD1FDE685A1854806F0D2
:104F100097F90028F1D094F8A10620F07800AFE0CE
:104F20000BE2F9E1E4E1B4E1AAE1A1E198E19AE060
:104F300094F8A106C0F3C3000C28DED2DFE800F02D
:104F40000810323E467107939B6206A8DBE635E700
:104F500073A1744806F074F900287FF403AFD2E619
:104F600078A1704806F06CF90028C6D04B46591954
:104F700001F5805181F8E9666D1CADB2142DF6D3B0
:104F8000002155464218AF5C5A1802F5805282F84B
:104F9000EE76491C89B20F29F4D300210320F4F7DF
:104FA00023FE9CE05EA15F4806F04AF90028A4D0E9
:104FB000C4F84066012084F83E06EEE062A159483C
:104FC00006F03EF900287FF4E1AE9CE658A1554872
:104FD00006F036F9002890D04A46511901F5805163
:104FE00081F8A2666D1CADB2142DF6D30021554692
:104FF00043182B445F79531803F5805383F8A77641
:10500000491C00E00AE189B20F29F1D3C4F84066D7
:10501000012084F83E0694F8A10620F0780028309C
:1050200077E145A13F4806F00BF900288ED094F8AF
:10503000681731B194F8A11621F07801303184F865
:10504000A116C4F84066012184F83E165044417907
:1050500000793039303841EA0010C117FCF74CFFB5
:1050600084F868074FE62EA12E4806F0E9F80028DC
:105070007FF46DAF47E694F8A10620F07800483041
:1050800084F8A106C4F84066012084F83E063AE69A
:1050900094F8A10620F078003BE194F8A106C0F353
:1050A000C300052891D2DFE800F00314257EC2007A
:1050B0001BA11C4806F0C4F8002886D0C4F840663E
:1050C000012084F83E0694F8A10620F0780008300C
:1050D0001FE113A1134806F0B3F80028C2D0C4F8AA
:1050E0004066012084F83E0694F8A10620F078007E
:1050F00010300EE116A10B4806F0A2F80028B1D03E
:10510000C4F84066012184F83E1650445546817922
:10511000407921E0107AFF1FBD290020647A002029
:105120004F4B000094720020494D45493A00000061
:1051300049434349443A00004353513A00000000B8
:105140002C0000002200000052454144590000009C
:10515000617475733A0000003038303941EA00104C
:10516000C117FCF7C9FE84F86807AFF22C0181482B
:1051700006F066F888B129184A78302A06D34978AB
:10518000285C3038303941EA001001E0285C3038C2
:10519000C117FCF7B1FE84F8690794F8A10620F066
:1051A00078001830B5E0AFF28801724806F048F890
:1051B000002893D0C4F84066012084F83E06DBF84E
:1051C000000038606C48006878606B48001D00681B
:1051D000B8604846411901F5805181F8E9666D1CB7
:1051E000ADB2142DF6D3387A04ADFB7ABA7A797A57
:1051F00085E80F003879FB79BA7979798DE80F0065
:10520000BB783A785DA1089804F060FA0021032089
:10521000F4F7EAFC10B16448C0F8886294F8A1067B
:1052200040F0800084F8A106C4F844866BE5AFF234
:105230001011504806F004F80028F7D094F8A106A1
:1052400020F0800084F8A10694F8A10620F07800F0
:1052500084F8A106049880F8A662C0F8A86252E516
:1052600052A1444805F0ECFF00287FF481AD4AE5E7
:105270004FA1404805F0E4FF00287FF47FAD42E5F0
:10528000AFF264113B4805F0DBFF00287FF484ADEA
:1052900039E548A1374805F0D3FF0028C6D0C4F847
:1052A0004066012184F83E1653464F464119194481
:1052B0000A79791901F5805181F86A276D1CADB220
:1052C000142DF3D33CA13D4805F0BAFF50B10021A5
:1052D0000A183A4402F5805282F86967491C89B27B
:1052E0000229F5D394F8A10620F07800303010E0C0
:1052F000AFF2D4111F4805F0A3FF002896D0C4F8E0
:105300004066012084F83E0694F8A10620F078005B
:10531000383084F8A106F6E429A1164805F090FF7C
:1053200000289CD0C4F84066012084F83E0694F81A
:10533000A10620F078004030EBE7AFF21C210D48C9
:1053400005F07EFF00288AD0DBF8000038600A48AC
:10535000006878600848001D0068B8604846411938
:1053600001F5805181F8E9666D1CADB2142DF6D3BC
:1053700039E7000094720020147AFF1F253032783C
:105380002530327825303278253032782530327821
:105390002530327825303278253032782530327811
:1053A00025303278250000000000424261000000F4
:1053B0006F6B0000444843502C0000003E2A002040
:1053C000434F4E4E45435445440000002DE9F74FEE
:1053D00086B00020019081460090FD4D00212954A7
:1053E000401C80B26428F8D3FA4890F8A612A0F5C1
:1053F000405419B3002180F8A61294F8A10620F0B9
:10540000800084F8A10694F8640728B101280ED022
:10541000022806D0032811D194F8A10620F07800C4
:105420000AE094F8A10620F07800203004E094F817
:10543000A10620F07800583084F8A10694F8A1065F
:10544000E54E00067ED594F8660601287BD194F8D7
:105450006207012877D10020DFF88083824600EBC5
:10546000400101EB0A1108EB0110039000F5805098
:10547000002702905EE0039800EB071505F58055C4
:1054800095F8B60B000653D595F8B60B40F004001E
:1054900085F8B60B95F8B60B000749D595F8B60B0D
:1054A00020F0080085F8B60B0020C1F835000AEBA3
:1054B0000A1101EB0A2108EBC10007EB071100EB11
:1054C000C10BC64842F26D0159441022253005F641
:1054D000B435F2F7BAFE0BF50050414650F8652F8F
:1054E00041F8192F42684A602A7888F81820D0F8C5
:1054F0001B10C8F82110BA4940468A6A40F8392F73
:10550000898D81806968C8F83F10D8F8540081B24D
:105510000220F3F75FFD00210620F4F765FBD8F8C1
:105520005400401CC8F8540000210520F4F75CFB2F
:105530007F1CBFB20298414690F88B0BB8429AD8B4
:10554000514601E0FEE31AE00220F4F74DFB0AF1B8
:10555000010080B28246042881D394F864070328AE
:1055600003D094F86407012803D19E490020C1F8B4
:105570008802002084F862070B2084F86607944FA5
:1055800000203A3F387000980DE001F047FCC4F865
:10559000B003D4F8B003C0F300400190D4F8B003D6
:1055A000C0F3420000900028EFD094F8640702286E
:1055B0000ED1874855214FF007090170FD21417038
:1055C000AA2181700021C170017161224271817133
:1055D0007F49F52201F809200020D4F8B013C0F16A
:1055E0000302D200D1407A4A09EB00031A44D17079
:1055F000401C80B20428F0D394F8630720B17948A6
:10560000D0F80802B0B906E07148089A4844C2715F
:1056100009F1080533E07148007858B194F864073F
:10562000032807D094F86407012803D0012084F8E8
:105630006606F8E36949664A00200B1803F58053B3
:1056400093F8E93609EB00051544EB71401C80B274
:105650001428F2D300200B1803F5805393F8A857B1
:1056600009EB00031344DD76401C80B20A28F2D314
:1056700002EB0900089980F8251009F12605002D94
:10568000D7D0089884F8270608981021FF221128FF
:105690007ED008DCA0F10B00062816D2DFE800F06F
:1056A0001515FE08FD16A2280FDA12280DD13AE2D0
:1056B00084F866174C49464A00202F180B5CD355D6
:1056C000401C80B20A28F8D30A3537E394F89C01CD
:1056D000C0077CD0012080F31388BFF34F8F43486D
:1056E0000168434A01F4E06111430160BFF34F8F49
:1056F000FEE700EB400101EB0B10384901EB001015
:10570000039000F58050804690F88A0B032816D04D
:1057100098F88A0B012812D098F88A0B02280ED02C
:1057200098F88A0B04280AD098F88A0B8A4605282C
:105730007ED098F88A0B0A4606287AD06EE1244A71
:1057400001205055ED1CA8B2022304901354401CB4
:1057500080B21D231354401C85B20020B9E0039988
:1057600001EB0A1202F5805292F8B40B1849485521
:105770006D1CA8B292F8B65B0D54401C85B292F82D
:10578000B60B400709D492F8B60B000705D400E029
:105790006EE192F8B60B80077ED500201F46D2F846
:1057A000B83BC0F1030C4FEACC0C23FA0CF300EB2E
:1057B000050C01F80C30401C80B20428EFD32D1DDD
:1057C000ABB20BEB0B15002005EB0B2212E028E12E
:1057D000520A0020D4520020BC640240D41200209F
:1057E000542600200000404250B301080CED00E0B8
:1057F0000400FA0507EBC2050AEB0A1205EBC20228
:10580000029202F50052D2F86550C0F10307FF0082
:10581000FD40C718CD55401C80B20428F3D31B1D92
:105820009BB20020D2F86950C0F10307FF0001E0ED
:1058300060E098E0FD40C718CD55401C80B20428B8
:10584000F0D31B1D9BB20020D2F88050C0F102079C
:10585000FF00FD40C718CD55401C80B20328F3D38C
:10586000DB1C9FB20025029901F50050D0F86D00B5
:1058700001F50051D1F87110C5F10502D200F2F71F
:10588000D2FCFF49EA1988546D1CADB2062DEAD34B
:10589000BF1DBFB2002502E018E07DE1C8E002991B
:1058A00001F50050D0F8750001F50051D1F87910DC
:1058B000C5F10502D200F2F7B6FCF149EA198854A5
:1058C0006D1CADB2062DE6D3BF1DBDB20AF10100BD
:1058D00080B2EC4B98F88B1B824651453FF63FAFA8
:1058E0000498E749049A281A1144030A01F8023D72
:1058F000487093E0E24802214155ED1CADB2A84644
:105900000021864623E0481C03460EF805000AEBFA
:10591000010707F580576D1C97F84575A8B20EF87A
:105920000070401C82B200200AEB011175460F186E
:1059300007F5805797F8517500EB020C05F80C70CD
:10594000401C80B21028F2D3103295B299B294F86C
:1059500044058842D7D80EEB0800002100F8021D4C
:10596000A5EB080159E0C64F03207855ED1CA8B2FD
:10597000022182463954401C80B20E213954401C09
:1059800085B2002196463DE0039800EB0110A0F29D
:105990004C4000F5005002787A556D1CAAB285780B
:1059A000BD54521C807895B2400729D50BEB0B1CD7
:1059B0000CEB0B220EEBC20201EB0113002002EBF9
:1059C000C302131803F5005393F88B3000EB050C5A
:1059D00007F80C30401C80B20A28F2D30A35ABB26B
:1059E0000020151805F5005595F8A45000EB030CA0
:1059F00007F80C50401C80B20228F2D39B1C9DB2C9
:105A0000491C89B298F88B0B8842BDD807EB0A0075
:105A1000002100F8021DA5EB0A0141700BF1010005
:105A200080B294F8E01A834659453FF662AE85E1AC
:105A30007878401C78707878052803D294F89C0117
:105A4000C00706D084F8661794F89C01C00704D0FC
:105A500005E00D2084F8660701E084F8A02178882D
:105A6000010A87484155798828444170AD1C65E199
:105A700084F8661794F8A101DFF8048208F805009D
:105A80000022DFF800C26D1C3EE094F8A10102EB99
:105A9000021700EB001101EB00200CEBC00000EB43
:105AA000C70000F5805090F83C0801282AD194F8EE
:105AB000A10100EB400101EB00100CEB001000EB2A
:105AC000021000F5805090F8840A08F805006D1C5B
:105AD000ABB2002094F8A11101EB011505EB0121F7
:105AE0000CEBC10101EBC701014401F5805191F8B4
:105AF0003D181D1808F80510401C80B20A28E9D38B
:105B00000A339DB2521C92B294F8A10100EB4001FD
:105B100001EB00100CEB001000F5805090F85B0AD0
:105B20009042B2D80AE17878401C787078780528DD
:105B30000ED294F8A10100EB400303EB001351488F
:105B400000EB031000F5805090F86C0AC00711D0EC
:105B500084F8661794F8A10100EB400101EB0011F5
:105B6000484800EB011000F5805090F86C0AC0071F
:105B700004D005E0122084F8660701E084F8A02133
:105B800094F8A1113E48415579882844090A41708A
:105B900079888170ED1CD1E0DFF8E8A001218AF856
:105BA0000610DAF854100A22B1FBF2F234494A55D1
:105BB000DAF854006D1C0A2801D90A2201E0DAF84B
:105BC00054200020029093464A5522206D1C4855CF
:105BD00000276D1CABE0DAF85400D04638B1D8F895
:105BE0005400C01B401E81B20220F3F787F998F8D9
:105BF00018004346DFF888C00CF805006D1CA9B2F8
:105C00000020D3F81920C0F10305ED00EA40451843
:105C10000CF80520401C80B20428F2D3091D89B27B
:105C20000020D3F81D20C0F10305ED00EA4045181F
:105C30000CF80520401C80B20428F2D3091D89B25B
:105C40000020D3F82120C0F10205ED00EA404518FC
:105C50000CF80520401C80B20328F2D3C91C1FFA9F
:105C600081F800259A46514651F8250F4968C5F13B
:105C70000502D200F2F7D7FA05EB0802004903E06B
:105C8000520A0020D412002088546D1CADB2062D9B
:105C9000E9D308F106001FFA80F80025514651F8B3
:105CA0002D0F4968C5F10502D200F2F7BCFAFA4996
:105CB00005EB080288546D1CADB2062DEED308F139
:105CC00006009AF83E3080B25146F34A1354401C05
:105CD0009AF83D3080B21354401C9AF83C3080B2A0
:105CE0001354401C9AF83B3080B21354401C91F876
:105CF0003A3080B21354401C91F8393080B21354BA
:105D0000401C83B20020D1F83F50C0F1030C4FEA91
:105D1000CC0C25FA0CF500EB030C02F80C50401CDF
:105D200080B20428EFD31B1D7F1C9DB2BFB2029A24
:105D30000020B7EB0B019041FFF64DAFA5EB090733
:105D40003A0A00E044E0D44901EB0900824642707F
:105D5000877000238B460CE009EB03015944884609
:105D6000C879DDE90021F3F7BBFE88F807005B1C6A
:105D70009BB29F42F0DC94F8A70328B1B9B2504619
:105D800000230422F4F728FEB9B25F465046F3F729
:105D900095FC010A79556D1CA9B27854491C94F8F8
:105DA00064078DB202280AD1681F010AF9703871A0
:105DB00081B2781D01F079F978556D1CADB235606E
:105DC0000121B648F3F7D0FC09B02846BDE8F08FB2
:105DD00094F86407B34BDFF8C8E2DFF8CCA242F2D4
:105DE000107BA3F18107A3F1830CA3F10B08A3F1AE
:105DF000720930B1012878D0022877D0032812D157
:105E000018E394F8A106C0F3C3000E280BD2DFE814
:105E100000F0071623313F4E5D6E7D8C9BD9E8FC68
:105E20000027984605E0ABE218F80700E8557F1C0C
:105E3000BFB29C48F2F727FAB842F5D815E3002420
:105E400003E0385D2855641CA4B296488138F2F707
:105E50001AFAA042F5D8AFE30024674603E0385DA4
:105E60002855641CA4B28F488338F2F70CFAA0427C
:105E7000F5D8A1E3002404E018F804002855641CB8
:105E8000A4B288480B38F2F7FEF9A042F4D893E3A5
:105E9000844F00241C3F03E0385D2855641CA4B2E5
:105EA00080481C38F2F7EFF9A042F5D884E37D4F23
:105EB00000242D3F03E0385D2855641CA4B27948C6
:105EC0002D38F2F7E0F9A042F5D875E3724F0024BF
:105ED000323F03E0385D2855641CA4B26E48323866
:105EE000F2F7D1F9A042F5D866E39CE0C6E16D4F28
:105EF00000243C3F03E0385D2855641CA4B2694887
:105F00003C38F2F7C0F9A042F5D855E3654F0024BC
:105F1000163703E0385D2855641CA4B2614816307A
:105F2000F2F7B1F9A042F5D846E35E4F00240A37F4
:105F300003E0385D2855641CA4B25A480A30F2F7D1
:105F4000A2F9A042F5D837E3DEF81802554C643CBC
:105F500088B10020215C2954401C80B20D28F9D35F
:105F60005046F2F790F900231A4650EA02011FD07A
:105F700000214E4C17E0002703E0E05DE8557F1C50
:105F8000BFB248486438F2F77EF9B842F5D821E14B
:105F9000671807F5805797F8B77605EB010C8CF872
:105FA0000D70491C89B20F1A73EB0207F0DB36E162
:105FB0003948F2F768F987B20CE101213748F3F765
:105FC000D3FB0BE3374F0024213703E0385D28551E
:105FD000641CA4B233482130F2F755F9A042F5D839
:105FE000EAE2DFF8C0800027A8F1790805E00CE0BC
:105FF00018F80700E8557F1CBFB22A487938F2F735
:1060000042F9B842F4D83760E2E2002704E019F818
:106010000710E9557F1CBFB222487238F2F733F9F6
:10602000B842F4D8EFE794F8A106C0F3C3000C28F7
:10603000C7D2DFE800F006213D4A5968778695A46B
:10604000FBF9DFF860800027A8F16B0804E018F87E
:106050000700E8557F1CBFB212486B38F2F713F9FE
:10606000B842F4D8376001210C48F3F77DFB4FF4B8
:106070007A70C4F84406B1E20A4F0024D73703E02F
:10608000385D2855641CA4B20648D730F2F7FBF8F7
:10609000A042F5D890E20000520A0020B864024005
:1060A0000000434273B901088B290020D41200205C
:1060B0000024FA4F03E0385D2855641CA4B2F74869
:1060C000F2F7E1F8A042F6D876E2F44F0024A53FBB
:1060D00003E0385D2855641CA4B2F048A538F2F7F7
:1060E000D2F8A042F5D867E2EC4F00249A3F03E0D3
:1060F000385D2855641CA4B2E8489A38F2F7C3F812
:10610000A042F5D858E2E54F00248F3F03E0385D08
:106110002855641CA4B2E1488F38F2F7B4F8A042C5
:10612000F5D849E2DD4F0024863F03E0385D28556D
:10613000641CA4B2D9488638F2F7A5F8A042F5D875
:106140003AE2D64F0024773F03E0385D2855641CBF
:10615000A4B2D2487738F2F796F8A042F5D82BE2ED
:10616000CE4F0024593F03E0385D2855641CA4B28B
:10617000CA485938F2F787F8A042F5D81CE2DEF891
:106180001802C64C4C3CC8B10020215C2954401C6C
:1061900080B21428F9D35046F2F775F80446002768
:1061A000BFA1504605F04CF8014654EA07003FF401
:1061B000FFAE0020A1F1010CBA4B18E0002703E06C
:1061C000E05DE8557F1CBFB2B4484C38F2F75BF88D
:1061D000B842F5D83760F0E61A1802F5805292F806
:1061E000B72605EB000888F81420401C80B26045F3
:1061F000F2DB22206A18D074641C47F100000AE028
:106200005A1802F5805292F8B62605EB010C8CF86C
:106210001420491C89B20A1B77EB0002F0DBA2A113
:10622000A248F2F724F8C3E60FE0FFE79B4F0024F3
:106230001C3F03E0385D2855641CA4B297481C3805
:10624000F2F721F8A042F5D8B6E1DFF85082002736
:10625000A8F10B0804E018F80700E8557F1CBFB24E
:106260008E480B38F2F70FF8B842F4D837600121A6
:106270008F48F3F779FA43F69820FAE694F8A106E6
:10628000C0F3C30005287BD2DFE800F003135D7B79
:10629000BB00002084F86507074604E018F80700F3
:1062A000E8557F1CBFB28348F1F7EDFFB842F5D83F
:1062B000A9E6002184F8651708462954401C80B2DD
:1062C0006428FAD384F865177A49002087310A5C7C
:1062D0002A54401C80B20828F9D3DFF8C88141F263
:1062E0002570002408EB000709E008EB040000F526
:1062F000805090F8250729190872641CA4B238460A
:10630000F1F7C1FFA042F0D82C20291908720934F6
:10631000A7B241F24D70002408EB000909E008EB38
:10632000040000F5805090F84D173A19A954641CE8
:10633000A4B24846F1F7A7FFA042F0D85AA15B48A3
:10634000F1F795FF58E0DFF854810027A8F1C40861
:1063500004E018F80700E8557F1CBFB24F48C43866
:10636000F1F791FFB842F4D8376001215048F3F7B4
:10637000FBF994F8A10620F07800183084F8A10603
:106380002CE194F863074B4FA43702284FF000002C
:1063900017D000212954401C80B26428FAD384F815
:1063A00065170020395C2954401C80B20E28F9D3AF
:1063B0005046F1F768FF0104090C1DD00020394A4E
:1063C00017E084F86507002403E0385D2855641C55
:1063D000A4B23848A430F1F756FFA042F5D8EBE05C
:1063E000131803F5805393F8B7362C18A373401C89
:1063F00080B28842F4D3A1E72C48F1F744FF306023
:10640000DBE5DFF898800027A8F1B80804E018F869
:106410000700E8557F1CBFB22048B838F1F733FFBA
:10642000B842F4D8376001212148F3F79DF941F2D1
:1064300088301EE694F8A106C0F3C300092874D280
:10644000DFE800F0051E3A47556474ACBC00002735
:10645000984604E018F80700E8557F1CBFB21548BD
:106460000B30F1F710FFB842F4D837600121104823
:10647000F3F77AF994F8A10620F0780008307DE768
:10648000002403E0385D2855641CA4B2094876381E
:10649000F1F7F9FEA042F5D88EE00000F9BA010844
:1064A0002C000000D41200200D0A0000520A002027
:1064B000B864024068B901080024674603E0385D0B
:1064C0002855641CA4B24748F1F7DDFEA042F6D877
:1064D00072E0002404E018F804002855641CA4B2FB
:1064E00040487830F1F7CFFEA042F4D864E03D4F49
:1064F0000024D83703E0385D2855641CA4B239481D
:10650000D830F1F7C0FEA042F5D855E0354F002451
:10651000E73703E0385D2855641CA4B23148E73002
:10652000F1F7B1FEA042F5D846E057E094F86307D2
:106530002C4FAE3702280FD00020395C2954401C64
:1065400080B20F28F9D35046F1F79DFE0104090CE3
:106550001FD00020244A15E0002403E0385D2855B0
:10656000641CA4B21F48AE30F1F78DFEA042F5D8EE
:1065700022E0131803F5805393F8B7362C18E37311
:10658000401C80B28842F4D3AFF2E4011748F1F71F
:106590006EFE1648F1F777FE84B20DE0114F00242D
:1065A000F13703E0385D2855641CA4B20D48F13082
:1065B000F1F769FEA042F5D83460FEE4002019F836
:1065C00000102954401C80B20728F8D3401E3060C8
:1065D00001210748F3F7C8F858464AE509B00020FA
:1065E000BDE8F08FF0B80108D4120020520A002054
:1065F000B864024070B5164C40F224452946204646
:1066000002F0C5FF002821D02946204602F05CFF99
:10661000104D00212846F3F7A7F861102846F3F73C
:106620008DF80D49012081F865072088A088281D74
:106630000268C2F5FA62A1F82A264FF4FA610160F5
:106640002846BDE870400121F3F78EB870BD000008
:106650000010014088640240D422002010B5074C8D
:1066600005492046F3F76AF800212046F3F77CF845
:1066700003490120087010BD00800028B864024062
:10668000180A00202DE9F04301218FB0880500F0A1
:106690001BFBDFF894904846F3F770F840200501A3
:1066A00003900024CDE90545C60207940894CDE97E
:1066B00009464FF000681E480B940C940D941B4F34
:1066C000CDF800800E94CDE9017069464846F3F795
:1066D000FDF8012210214846F3F7E2F8DFF8489070
:1066E000A9F130094846F3F749F84FF4FA60CDE9CB
:1066F0000340CDE9054507940894CDE909460D48C6
:106700000B940C940D94CDF800800E94CDE901709B
:1067100069464846F3F7DAF801214846F3F724F8CA
:106720000FB0BDE8F0830000B864024004100140DF
:10673000520A0020947200201CB50121032000F0B1
:10674000C3FA0E4C072206212046F3F769FE072202
:1067500011462046F3F764FEC020022100908DF818
:10676000051000228DF8062001208DF807008DF815
:10677000041069462046F3F717FE1CBD00040240D2
:106780002DE9F0410024FFF7D7FFFFF77BFF4FF41F
:10679000E13000F0ADF800F08DF80121402000F06C
:1067A000ABFA012000F02CFB4FF47A75284604F078
:1067B000A7FB3C490B2081F82A01002381F82631F0
:1067C0000B768B764B76CB760D6281F828300126DE
:1067D00081F82A6081F8296081F82B60E80008635D
:1067E0000B708E704E70CE708D600B738E734E7307
:1067F000CE73001148612C4A137093705670D67096
:106800004EF660259560294F42F6F82CA1F23C61C6
:10681000A2F5297204EB440007EB8000A0F5196093
:1068200000F50050037083704670C370C0F808C054
:10683000641C042CEED391F86107000706D091F890
:10684000610700F00F00401E81F8630791F86107AF
:10685000000906D091F86107FF2404EB101081F8BD
:10686000640781F8683791F8640770B1104C01280B
:106870000ED0022809D0032805D147F23050C2F8C3
:10688000AC02C4F88832BDE8F081C2F8AC52FAE735
:10689000C2F8AC52C4F8883242F21070C1F8440613
:1068A000F1E700001029002078550020D4120020C4
:1068B0000000404238B546208DF8000002208DF8D7
:1068C000010001248DF802408DF803406846FCF772
:1068D000E9F925208DF800008DF8014000208DF8A1
:1068E00002008DF803406846FCF7DCF938BD000073
:1068F0001FB504460121102000F022FA0020ADF857
:1069000004000094ADF80600ADF80800ADF80C00E6
:106910000C200D4CADF80A006946204602F06EFED0
:106920000121204602F0D3FD012240F224412046FD
:1069300002F04CFE1021204602F0C6FD0122C021CB
:10694000204602F0CEFD1FBD001001402DE9F04FA2
:106950008DB034225E496846F1F777FC5D4F002622
:1069600097F8630700287DD0DFF86CB10121CBF8E0
:1069700088124FF0000987F86597584D584C02E08F
:10698000A85DA055761C5548F1F77DFCB042F7D8BC
:10699000DFF85081C8F800600121A8F10400F2F787
:1069A000E3FE4FF4FA7004F0ABFA87F86597DFF86E
:1069B0002CA100260AF1830A03E01AF80600A0556C
:1069C000761C46488330F1F75EFCB042F5D8C8F833
:1069D000006044480121001FF2F7C6FE4FF47A70B0
:1069E00004F08EFA87F86597DFF8F0A000260AF128
:1069F000020A03E01AF80600A055761C3748801CEE
:106A0000F1F741FCB042F5D8C246C8F800603548FD
:106A10000121001FF2F7A8FE4FF47A7004F070FA1B
:106A2000C84687F86597002602E0A85DA055761C49
:106A30002A48F1F728FCB042F7D85546CAF800605A
:106A4000DFF8A0A00121AAF1040A5046F2F78CFE5B
:106A50004FF47A7004F054FA23496846F1F707FCC2
:106A60001E4900E030E0891D6846F1F700FC87F818
:106A700065870026E94603E019F80600A055761C54
:106A80006846F1F700FCB042F6D82E60012150466E
:106A9000F2F76AFE4FF47A7004F032FA464687F84D
:106AA00065870E4900200A310A5C2254401C0728E1
:106AB000FAD3401E286001215046F2F755FE6420AB
:106AC00004F01EFACBF888620DB0BDE8F08F00002C
:106AD00010BD0108D422002000004242F0B8010895
:106AE000520A0020BC640240D12900202DE9FC5F3D
:106AF0000121592000F0E8F80024DFF89CB04FF4A1
:106B00007C578DF80440022600978DF8076069468F
:106B10005846F3F749FCFC20DFF880A000908DF880
:106B2000044001258DF8075069465046F3F73CFCB8
:106B3000DFF86C904FF440488DF80440CDF80080A9
:106B40008DF8075069464846F3F72EFC8DF804404F
:106B50008DF807600720134E009069463046F3F722
:106B600023FC07213046F3F772FC41464846F3F711
:106B700070FC39465846F3F76CFCFC215046F3F79D
:106B800068FC0948D0F828120848012902D004708E
:106B9000BDE8FC9F0570FBE70010024000180240B2
:106BA000000C02400000024000004242D4120020CB
:106BB00070B5FFF79BFF642004F0A2F91548D0F8E8
:106BC0003C3201221449154800243BB180F8634748
:106BD000D1F814121248D1B1047570BDD1F8183231
:106BE0008BB180F86327D1F80832D1F80C5243EA10
:106BF0004503DB4380F8643790F8643703F0030300
:106C000080F86437E4E7022380F86337EBE7027526
:106C100070BD00000080414200004342D4220020A9
:106C2000D41200202DE9FC410121112000F04CF884
:106C300001248DF8044000254CF204008DF8065024
:106C40000326184F00908DF805608DF807406946BF
:106C50003846F3F7A9FB04213846F3F7F8FB12484E
:106C600090F86417032903D090F86407012812D123
:106C70008DF804408DF8065004200C4D00908DF8DE
:106C800005608DF8074069462846F3F78DFB04211F
:106C90002846F3F7DCFB0648C0F8B842C0F8BC420F
:106CA000BDE8FC8100100240D42200200000024018
:106CB00000004242FFF7B6BF4FF400610148F3F70E
:106CC000BFBB000000040240044A0029116801D043
:106CD000014300E0814311607047000030380240FA
:106CE000044A0029116801D0014300E0814311608A
:106CF0007047000010380240044A0029116801D092
:106D0000014300E0814311607047000034380240C5
:106D1000044A0029116801D0014300E08143116059
:106D20007047000040380240044A0029116801D031
:106D3000014300E0814311607047000020380240A9
:106D4000044A0029116801D0014300E08143116029
:106D50007047000044380240044A0029116801D0FD
:106D6000014300E081431160704700002438024075
:106D700070B5204B1968204C11F00C0104D066103E
:106D8000042903D0082903D004601BE0066019E041
:106D9000184A121F1168C1F38055116801F03F01B4
:106DA00015B1B6FBF1F101E0B4FBF1F11468126822
:106DB000C4F388146143C2F30142521C5200B1FB78
:106DC000F2F1016019680F2202EA11110B4A545CBA
:106DD0000168E14041601C68072505EA9424145DC0
:106DE00021FA04F484601B6805EA5333D25CD14075
:106DF000C16070BD083802400024F400000000208B
:106E000005490028086802D040F0040001E020F0A5
:106E10000400086070470000000806500148006840
:106E2000704700000808065070B5012080F31088F4
:106E30000C4D10212846F3F70AFB08212846F3F7EA
:106E400008FBD720F2F77EF9FF20F2F77BF9044622
:106E500010212846F3F7FDFA002181F3108820461F
:106E600070BD00000000024070B5012080F3108862
:106E7000194C0020A080FFF7D7FF000609D401209D
:106E800004F03EF8A088401C80B2A080C828F2D34D
:106E90001EE0A088C8281BD2104D10212846F3F709
:106EA000D6FA08212846F3F7D4FA9F20F2F74AF9D8
:106EB000FF20F2F747F9FF20F2F744F96070102144
:106EC0002846F3F7C6FA002080F31088607870BD7A
:106ED000002080F3108870BD2212002000000240C4
:106EE00070B5012188B08803FFF712FF012102204D
:106EF000FFF7EAFE00244FF400602F4E8DF80440A7
:106F000000908DF8074069463046F3F74DFA0121AD
:106F10008DF8041002258DF8055008038DF8064001
:106F20008DF80710009069463046F3F73DFA0522C8
:106F30000D213046F3F774FA05220E213046F3F79F
:106F40006FFA05220F213046F3F76AFA4FF46040DA
:106F500000908DF8045003208DF805008DF8064050
:106F60008DF8074069463046F3F71EFA134D284660
:106F700000F04AF8ADF810406815ADF8120018207E
:106F8000ADF814000720ADF81800ADF808404FF434
:106F90008270ADF80C40ADF80A00ADF80E40ADF8C7
:106FA000164002A9284600F064F80121284600F0A6
:106FB00021F808B070BD0000000402400038004015
:106FC00070B50B4C05460221204600F047F800281A
:106FD000F9D02946204600F04AF80121204600F069
:106FE0003DF80028F9D0204600F03FF8C0B270BD4F
:106FF000003800400029018802D041F0400101E042
:1070000021F0400101807047114910B588420AD132
:10701000841401212046FFF79FFE2046BDE8104062
:107020000021FFF799BE0B49884202D101210414C7
:1070300004E0094988420AD10121C4132046FFF720
:1070400073FE2046BDE810400021FFF76DBE10BD65
:107050000030014000380040003C00400246002063
:1070600012890A4200D001207047808970478181CF
:10707000704730B502884C8802F441530A88CD88A5
:1070800022438C882C4322430C8922434C8922437F
:107090008C892243CC8922431A430280828B22F4BA
:1070A00000628283098A018230BD0246002003E02B
:1070B00012F8013B1844C0B2491E89B2F8D2704799
:1070C0002DE9F04101218D070024284601F082FEC0
:1070D000F0B3F3F771FC284E002006F580533DE035
:1070E00006EB840101F58051D1F8B4271278012A0A
:1070F000D1F8B42703D05278012A08D02CE01070C0
:10710000D1F8B4275070D1F8B427907030E0D1F89E
:10711000B427927802BBD1F8B42757687F1C576018
:10712000D1F8B4275268D1F8B477BF68BA4213D304
:10713000D1F8B4770122BA70D1F8B427D278012AF5
:1071400016D0D1F8B4275070D1F8B427506000E0C1
:1071500008E0D1F8B417C870641CE4B293F8B21711
:10716000A142BDD82846BDE8F041012101F07CBD17
:10717000D1F8B4174860EFE7D41200200CB5002214
:10718000254900920192086840F4803008604FF46D
:10719000A063086800F4003001900098401C009043
:1071A000019810B900989842F3D10868800330D54F
:1071B0000120019018484030026842F0805202607D
:1071C0001648026842F480420260134808300268A0
:1071D00002600268026002680260031F104A1A60BF
:1071E0000A6842F080720A600A689201FCD50D4A72
:1071F00040F205611160016821F00301016001683E
:1072000041F0020101600168C1F381010229FAD154
:107210000CBD01920CBD000000380240007000401F
:1072200008544007003C02407CB500229FED170A3D
:1072300000928DED010A6D4601AC16E0835CA3F16E
:107240003006102E05D2009B1B010093865C303E59
:1072500007E0413B062B0CD2009B1B010093865C90
:10726000373E1E43521CD2B200968A42E6D300201B
:1072700006E0BFEE000A7CBD2A5C2254401CC0B26E
:10728000B0EB510FF8D39DED010A7CBD000000006A
:1072900030B505460022104611E0AB5CA3F1300486
:1072A000102C02D244EA001007E0A3F14104062C9E
:1072B00008D20401A3F137002043521CD2B28A4203
:1072C000EBD330BD4FF0FF3030BD00002DE9FE4361
:1072D000534C4FF03809A07800263146FAF70CFEDF
:1072E000012508270096CDE90175024618200023E4
:1072F0004946FBF727FF00F1040808EB4800400669
:10730000000E08232D2249460095FBF7ADFE60785C
:1073100008F101080021FAF7EFFD0246009608EB9C
:107320004800CDE901754006000E00234946FBF7F1
:1073300009FF804408EB48004006000E08232D2278
:1073400049460095FBF790FE207808F101080021DE
:10735000FAF7D2FD0246009608EB4800CDE9017528
:107360004006000E00234946FBF7ECFE804408EB84
:1073700048004006000E0823202249460095FBF7EE
:1073800073FE607908F101080021FAF7B5FD0246A5
:10739000009608EB4800CDE901754006000E002379
:1073A0004946FBF7CFFE804408EB48004006000E3C
:1073B00008232D2249460095FBF756FE207908F157
:1073C00001080021FAF798FD0246009608EB4800F4
:1073D000CDE901754006000E00234946FBF7B2FED9
:1073E000804408EB48004006000E08232D22494641
:1073F0000095FBF739FEE07808F101080021FAF763
:107400007BFD0246009608EB4800CDE90175400679
:10741000000E00234946FBF795FEBDE8FE83000001
:107420007C2600200249C870012088717047000046
:10743000D41200202DE9FE4F00252F46F2F706FE5C
:10744000F74EB07900287CD0A94686F80690FBF765
:1074500065FCF0784FF0080A4FF001084FF0100B70
:1074600006F58054102881F05F83DFE810F01000EB
:107470008C00FD004802B403F80306057106970767
:10748000E4073A08E308DD09240AC50A360BF3F7D6
:1074900083FA01280AD0022808D0042806D0082838
:1074A00004D10220FFF7BEFF84F8A091CDE900B817
:1074B000002145461523DBA20846FBF706FF94F89A
:1074C000A10128B3CDE900A557460523DAA214216E
:1074D0000020FBF7FAFECDF80090CDE9017594F895
:1074E000A121002314211E20FBF72CFECDE90075FD
:1074F00094F8A1010A2300EB400101EB001006EB18
:10750000001041F66221421814212820FBF7DDFE0D
:1075100094F8A001FF2829D094F8A001CDE9000536
:107520000A2364221E211846FBF71CFDCDF80090AB
:10753000CDE901A594F8A0214E4600232D2132204B
:1075400000E0F3E3FBF7FEFD00EB4000322101EB2E
:107550004000C0B2082325222D210095FBF784FDB1
:1075600094F8A001642808D001F0DEBACDE900A5A6
:1075700015232D21B2A21420FCE384F8A06102207F
:10758000FFF750FFF0E7F3F707FA01280BD00228C6
:1075900009D0042802D0082805D101E0092000E024
:1075A0000420FFF73FFF94F8620738B194F86307AF
:1075B00038B1012808D0022811D108E01523A4A26F
:1075C00007E01523A5A204E01523A8A201E01523D6
:1075D000A9A2CDE900A800210846FBF776FEB07805
:1075E000012802D0022811D106E0A7480923CDE9DD
:1075F00000081A460A2106E0A34909231231CDE901
:1076000000181A460A210020FBF712FE9E48182394
:107610004838CDE9000844461A4600216820FBF7A7
:1076200007FECDE900A45546152398A21A21002093
:10763000FBF74BFECDE9005415239AA2242100202C
:10764000FBF743FECDF80090CDE90154726D0023A5
:1076500024215420FBF776FD706D10B90220FFF74E
:10766000E1FEFFF733FE7FE7F3F796F9042802D037
:10767000082811D107E094F89C0120F0800084F8DC
:107680009C01092006E094F89C0120F0800084F819
:107690009C010420FFF7C6FE94F8620738B194F805
:1076A000630768B101280ED0022814D118E0CDE993
:1076B00000A8002115237FA20846FBF706FE15E06F
:1076C000152366A201E0152368A2CDE900A80021D8
:1076D0000846FBF7FAFD94F827060F2803D005E0CB
:1076E000152365A2F1E70120FFF79CFEB078012881
:1076F00002D002280CD101E0634901E06249123155
:10770000CDE9001809231A460A210020FBF790FD55
:1077100094F8A00110B10020FFF784FE94F864678C
:1077200059495C31A1F10E00A0F10E05A0F11C0237
:10773000A0F12A03022E07D094F86467012E51D0DD
:1077400094F86467F6B320E05C4ED6F80062D6B3D6
:1077500094F86837322B04D2CDE9001808230E22A2
:107760000FE094F868173C2948D394F86807462836
:1077700052D2CDE9005808230E220021592002E000
:107780000E2200215920FBF753FD3F4818234838AB
:10779000CDE9000845461A4600216820FBF748FD60
:1077A000CDE900B55E46102345A214212820FBF741
:1077B0008CFDCDE900A5152343A224211220FBF75F
:1077C00084FD01E00EE095E094F89C0100067FF551
:1077D00048AFCDE90065102340A22E210020FBF721
:1077E00074FD3EE794F86867202ECED294F868675F
:1077F0001A2EB1D894F86817172905D9CDE90008D1
:1078000008230E220021BDE794F868071428B0D899
:1078100094F8680712286ED9CDE900280823AFE74D
:10782000D41200204669726D77617265446F776E7D
:107830006C6F616400000000506F72743A000000C9
:10784000446F776E6C6F6164204661696C21000043
:107850004E6F205369676E616C000000547970654B
:107860003A53746174696F6E00000000547970655A
:107870003A436C6F75640000547970653A436C6FDD
:1078800075642D546573740098D901084F66666C51
:10789000696E65205265636F72642055706C6F610C
:1078A000640000005265636F7264206E756D6265DE
:1078B000723A00004F66666C696E650000004042D7
:1078C000424C5545534B5900454E4552475920545B
:1078D0004543484E4F4C4F47590000005570677262
:1078E0006164652045525220436865636B2047758B
:1078F0006E000000FFE7CDE90038082340E7F3F70A
:107900004BF8012806D002281CD004283AD00828B9
:1079100038D132E03F210FE0307918B13079401E84
:10792000307100E03171307900EB8002C2EB8010E1
:10793000304490F85C00F8B930796D1CADB2402D40
:1079400020D8E9E7494614E06D1CADB2402D19D8A6
:1079500030793F2803D23079401C307100E031711A
:10796000307900EB8002C2EB8010304490F85C006C
:1079700010B930794028E7D304E00220FFF752FD28
:1079800086F80490F078344603287CD10122002147
:10799000FE4801F007F9207900EB8001C1EB80106F
:1079A000204490F85C004E460021FAF7A5FA0096B4
:1079B000CDE901B80246002345465F4619465820E6
:1079C000FBF7C0FBCDE900751023F1A2194600209A
:1079D000FBF77BFC207900EB8001C1EB8010204499
:1079E000D0F85D000021FAF787FA4FF00208CDF8D1
:1079F0000080CDE901750246002310211820FBF715
:107A0000A1FBCDE900751023E6A220210020FBF7A1
:107A10005CFC207900EB8001C1EB80102044D0F8A1
:107A200061000021FAF768FACDF80080CDE9017510
:107A30000246002320211820FBF784FB207900EB6D
:107A40008001C1EB8010204490F87F000021FAF7FC
:107A500053FA0096CDE901A5024657463821182071
:107A60000023FBF76FFB00F1040808EB4800400619
:107A70003821000E08232D220095FBF7F5FA08F1B6
:107A80000108207900E090E200EB8001C1EB80105A
:107A9000204490F87E000021FAF72EFA0246009664
:107AA00008EB4800CDE9017540063821000E00239F
:107AB000FBF748FB804408EB480040063821000EE5
:107AC00008232D220095FBF7CFFA207908F1010851
:107AD00000EB8001C1EB8010204490F87D00002174
:107AE000FAF70AFA0246009608EB4800CDE901755C
:107AF00040063821000E0023FBF724FB804408EBEE
:107B0000480040063821000E082320220095FBF78C
:107B1000ABFA207908F1010800EB8001C1EB80107D
:107B2000204490F882000021FAF7E6F90246009618
:107B300008EB4800CDE9017540063821000E00230E
:107B4000FBF700FB804408EB480040063821000E9C
:107B500008232D220095FBF787FA207908F1010808
:107B600000EB8001C1EB8010204490F881000021DF
:107B7000FAF7C2F90246009608EB4800CDE9017514
:107B800040063821000E0023FBF7DCFA804408EBA6
:107B9000480040063821000E08232D220095FBF7EF
:107BA00063FA207908F1010800EB8001C1EB801035
:107BB000204490F880000021FAF79EF902460096D2
:107BC00008EB4800CDE9017540063821000E00237E
:107BD000FBF7B8FAC8E4F2F7DFFE012806D0022866
:107BE00009D004280ED008281ED121E03079D8B160
:107BF0003079401E04E03079032815D23079401CDA
:107C0000307111E0307930B1012806D0022806D059
:107C1000032809D105E0052004E0062002E0072042
:107C200000E00820FFF7FEFBF078042805D09BE475
:107C30000220FFF7F7FB4846E2E754480422002100
:107C4000803800F0AFFFCDE900B930794F49803975
:107C500001EB001230790007010E1023F6E3F2F772
:107C60009BFE082802D10420FFF7DCFBF078B14628
:107C70000528AFD1454804220021403800F092FF8A
:107C800094F8630720B101280AD0022823D134E0F8
:107C90001023AFF23842CDE900A81946002018E0C1
:107CA000474656461023AFF23C42CDE900A819469C
:107CB0000020FBF70AFB10233FA238210020CDE96A
:107CC0000067FBF702FB11233D4A38211E20CDE956
:107CD0000067FBF7FAFA94F8640740B394F8640776
:107CE000012825D094F86407354E253602287BD02C
:107CF00094F86407032878D036E4CDE900A810236F
:107D0000464657462FA219460020FBF7DEFACDE97A
:107D10000076102328A238210020FBF7D6FACDE9FF
:107D20000076112338212B4A1E20D2E7F0E3FFE72B
:107D30004C46601900F5805090F8A20618B96D1CE9
:107D4000ADB2152DF5D3CDE900A846465746102310
:107D500021A21A210020FBF7B8FA601941F2A261B2
:107D60004218CDE9007610231A212020FBF7ADFA46
:107D7000102300E0B4E3CDE9007619A2242100200D
:107D8000FBF7A3FA0E4A102339322FE082DA0108FA
:107D90004C3A20202020202020202020202020209D
:107DA00000000000503A2020202020202020202009
:107DB000202020200000000055524C3A0000000016
:107DC00098290020547970653A436C6F75642D547E
:107DD000617374001CB90108494343494400000021
:107DE00041504E203A00000015E024E0CDE9007635
:107DF00024210846FBF769FACDE900761023FDA29D
:107E00002E210020FBF761FACDE900760F232E2109
:107E1000FA4A242064E3CDE900A8444655461023DD
:107E2000F7A21A210020FBF750FAF44A1023373248
:107E30001A211E200EE0CDE900A844465546102325
:107E4000F1A21A210020FBF740FAEC4A10237C3201
:107E50001A211220CDE90054FBF737FACDE900547E
:107E60001023E4A224210020FBF72FFA142332462A
:107E70002E21CDE90054002032E3F2F78DFD0128D8
:107E800004D0022807D008280FD10BE0307960B168
:107E90003079401E04E03079032806D23079401C46
:107EA000307102E00420FFF7BDFAF07806287CD19B
:107EB00004220021D54800F075FECDF80090CDE9F0
:107EC00001B844463279B346B046012300213E2032
:107ED000521CFBF737F9CDE900A456461023CCA27B
:107EE00000214820FBF7F1F9DFF830A3CDE900A429
:107EF00008231A4600217820FBF79AF9CDE900649F
:107F00001023C7A208214820FBF7DFF90823CDE999
:107F100000A91A4619467820FBF78AF9CDE90064D2
:107F20001023C2A219460020FBF7CFF998F80400ED
:107F300000EB400101EB001108EB011000F580504F
:107F400090F8910B4FF01003012844D0B9A2CDE96D
:107F5000006410211E20FBF7B8F9CDE90064A046AB
:107F60001023B6A218210020FBF7AFF99BF80400FC
:107F700000EB400101EB00100BEB001000F580500E
:107F800090F88A0BCDE9006805289BF8040000EB07
:107F9000400101EB00100BEB001000F580501CD0ED
:107FA00090F88A0B9949403100E043E201EB00125E
:107FB0000C2318213620FBF788F90120CDE9006059
:107FC000B0461023A0A220210020FBF77EF909264D
:107FD0004FF0200BACE09FA2B9E790F8900B8B49D3
:107FE000B031E1E706EB46014FF07A0ABAEB410FF8
:107FF00002D27F1CBFB20026207900EB400101EBCA
:10800000001004EB001000EB051000F5805090F814
:10801000B60BCDF80090C009CDE90180207900EBC6
:10802000400101EB001004EB001000EB051000F51F
:10803000805090F8B42B0BEBC700C1B206EB4600A2
:108040004006000E0023FBF77DF8304486B206EBB5
:108050004601BAEB410F02D27F1CBFB20026207945
:1080600000EB400101EB001004EB001000EB0510E9
:1080700000F5805090F8B60B0823C00900900BEB78
:10808000C700C1B206EB46004006000E2D22FAF7EB
:10809000EBFF761CB6B206EB4601BAEB410F02D2FB
:1080A0007F1CBFB20026207900EB400101EB0010DD
:1080B00004EB001000EB051000F5805090F8B60BB3
:1080C000CDF80090C009CDE90180207900EB400196
:1080D00001EB001004EB001000EB051000F58050E0
:1080E00090F8B52B0BEBC700C1B206EB460040067B
:1080F0005C46000E0023FBF725F8304486B206EB01
:108100004601BAEB410F02D27F1CBFB2002601200C
:10811000009004EBC700C1B206EB46004006000E1B
:1081200008233B22FAF7A0FF761C6D1CB6B2ADB255
:108130004A4C207900EB400101EB001004EB0010E9
:1081400000F5805090F88B0BA8423FF64BAF71E1E1
:10815000F2F722FC012804D0022807D008280FD10A
:108160000BE0307960B13079401E04E030790328AB
:1081700006D23079401C307102E00420FFF752F93A
:10818000F0780728E3D10124B471204804220021AB
:10819000E03000F007FD0021CDE9001B02943279A8
:1081A00001234020521CFAF7CDFFCDE900A4D346AD
:1081B00010232BA214210020FBF787F80924DDE00F
:1081C00004EB44014FF07A08B8EB410F02D27F1C58
:1081D000BFB200240020CDE9000B4FF00109CDF81B
:1081E0000890307900EB400101EB001006EB001025
:1081F0003CE00000494D45493A000000C2290020FA
:10820000535349443A00000049503A00C2DA010889
:108210004F6E4C696E65203A2000000048D9010875
:108220004F66664C696E653A2000000054797065AF
:108230003A000000525334383500000050726F7419
:108240006F636F6C3A00000047756E2D4164647275
:108250003A0000004C4F524100000000D4120020B0
:1082600047756E2D525353493A00000000EB05103C
:1082700000F5805090F8B42B4FF0140A0AEBC700B9
:10828000C1B204EB44004006000E0023FAF75AFF87
:10829000204484B204EB4401B8EB410F02D27F1CAE
:1082A000BFB200240AEBC700C1B204EB4400400691
:1082B000000E08232D22CDF80090FAF7D5FE641C9D
:1082C000A4B204EB4401B8EB410F02D27F1CBFB251
:1082D00000240021CDE9001BCDF80890307900EB97
:1082E000001101EB002006EBC00005EB051100EBCF
:1082F000C10000F5005090F88800642110FB01F0E7
:10830000020A0AEBC700C1B204EB4400400656461D
:10831000000E0023FAF716FF204484B204EB440158
:10832000B8EB410F02D27F1CBFB2002406EBC7009E
:10833000C1B204EB44004006000E08232522CDF80C
:108340000090FAF791FE641CA4B204EB4401B8EB70
:10835000410F02D27F1CBFB2002406EBC700C1B29E
:1083600004EB44004006000E08233B22CDF80090A9
:10837000FAF77AFE641C6D1CA4B2ADB2FC4E3079E3
:1083800000EB400101EB001006EB001000F58050FF
:1083900090F88B0BA8423FF613AFC5E3F2F7FCFA57
:1083A000082802D10420FFF73DF8F0780828F4D11E
:1083B00004220021EF4800F0F5FBCDE900A8474674
:1083C00054461023EC4A14210020FAF77EFFB246EF
:1083D00005EB450000EB05110AEB011841F69C3056
:1083E00010F80800C00721D005EB8501142000EB30
:1083F0004106CDE90047F1B20523E0A20020FAF7DB
:1084000064FFCDF80090CDE90147F1B201236A1C69
:108410001E20FAF797FE41F69231CDE9004708EBAE
:108420000102F1B20A232A20FAF74FFF6D1CADB208
:10843000042DCDD378E3F2F7AFFA012807D0022854
:108440000CD0042812D0082831D134E047E030792C
:1084500010B13079401E25E0052023E03079052851
:1084600002D23079401C1DE048461BE030790628D6
:108470001DD2DFE800F00305070911190A2014E0F6
:108480000B2012E00C2010E00D20FEF7CBFF94F83B
:10849000610700F00F0005E00E20FEF7C3FF94F81F
:1084A00061070009307102E00F20FEF7BBFFF07892
:1084B000092804D038E30220FEF7B4FFD4E730796E
:1084C000AC4C0422403404EB0010002100F06AFBA5
:1084D000CDE900B93079102304EB0012002100200F
:1084E00087E2F2F759FA012806D0022809D00428B9
:1084F0000FD0082851D154E0307918B33079401E9C
:1085000004E03079032848D23079401C307144E0CF
:108510000EE3307900EB400101EB001006EB001098
:1085200000F5805090F8910B01280CD0307900EBC9
:10853000400101EB001006EB001000F5805090F8B0
:10854000910BA0B129E030794C4600EB400101EBE2
:10855000001006EB001000F5805080F8919B3179F7
:108560000220F1F741FB8748C0F8884215E03079D6
:10857000444600EB400101EB001006EB001000F553
:10858000805080F8918B3079FAF78CF97D48C0F8EB
:10859000884231790220F1F727FBF0780A2805D0CC
:1085A000C2E20920FEF73EFF4846AFE771480422C9
:1085B0000021D03000F0F6FACDE900A84446554637
:1085C000152371A214212820FAF77FFECDF8009020
:1085D000CDE901543279012314214620521CFAF7C7
:1085E000B1FD307900EB400101EB001006EB00100B
:1085F00000F5805090F8910B01280CD0307900EBF9
:10860000400101EB001006EB001000F5805090F8DF
:10861000910B18B10AE015235DA201E015235FA2BA
:10862000CDE900541E210020FAF74FFE15235EA26B
:1086300032211EE4F2F7B0F9604C012806D002287E
:108640000FD004281AD0082830D11CE0307968B344
:1086500094F8BD0210B13079FAF724F93079401E50
:108660000AE03079032821D294F8BD0210B13079A4
:10867000FAF718F93079401C307117E084F8BD82A0
:1086800084F8B18212E00920FEF7CCFE484686F855
:10869000049084F8B08294F8BD1239B13949C1F818
:1086A000880284F8BD023079FAF7FCF8F0780B28DC
:1086B00031D104220021424800F074FACDE900A82B
:1086C00045465746152330A212212820FAF7FDFD12
:1086D000CDF80090CDE901753279012312214620B1
:1086E000521CFAF72FFDCDE90075152335A21C2188
:1086F0000020FAF7EAFDCDE90075152337A22621FF
:108700000020FAF7E2FDCDE90075152339A23021EA
:108710000020FAF7DAFD94F8BD02012827D145467A
:1087200086F8068094F8B20280B11649C1F88892A2
:1087300084F8B29230790121FAF7D8F9CDE900A591
:10874000152331A238210020FAF7BFFD94F8BC02AE
:1087500000280CD084F8BC92CDE900A515232EA2E8
:1087600038210020FAF7B1FD0648C0F88852DBE155
:10877000D4120020E2DB010850B30108506F72747C
:108780002D00000000004242504F52543A000000B9
:10879000545950453A4C4F524100000054595045ED
:1087A0003A525334383500005061737320456E746B
:1087B0006572204368616E6765000000D452002036
:1087C000F2DC0108313A4469702073776974636898
:1087D0002031616E6432204F4E000000323A496E03
:1087E0007365727420736C617665206D6F64756C4F
:1087F00065000000333A5061737320456E746572F2
:10880000205374617274000053746174653A536547
:108810006E64696E6700000053746174653A436F5B
:108820006D706C6574650000F2F7B6F8012813D01E
:10883000022811D0042802D008280DD109E0F0F751
:10884000FDFD142803D0484684F8A70304E0404601
:10885000FAE70920FEF7E6FDF0780C287ED1042225
:108860000021B44800F09EF9CDE900A845465646DF
:108870001523B1A21A210020FAF727FDCDE90065E2
:108880001523B2A224210020FAF71FFDCDE90065CF
:108890001523B2A22E210020FAF717FD94F8A703A2
:1088A0004FF0150308B1B3A200E0B8A2CDE900650E
:1088B000382100209DE0F2F76FF8012806D0022849
:1088C0000BD0042812D0082857D165E0307910B1B8
:1088D0003079401E08E0032006E03079032802D2F8
:1088E0003079401C00E04846307146E0317994F818
:1088F000610761F3030084F8610700210320F1F7A9
:1089000073F960B394F86157022004F5CE74FEF752
:1089100089FDF1F7BFF984F8C55500210320F1F76F
:1089200063F9207820F001002070207840F00600E4
:108930002070A4F8029000210120F1F755F994F875
:10894000050520F0800084F8050594F8C805A4F515
:10895000CE74B0B1012819D0022801E0E4E00CE0A7
:1089600002D0032807D10CE094F8A10620F078008B
:10897000203084F8A106FDF703FFF0780D280FD012
:10898000D2E094F8A10620F07800F2E794F8A1066E
:1089900020F078005830ECE70920FEF743FDA2E70D
:1089A000644804220021403000F0FCF8CDE900B812
:1089B00094F861075D465F4F00F00F00C03707EB8A
:1089C0000012102319460020FAF77FFC94F8610783
:1089D000317900F00F00884202D0CDE9005901E062
:1089E000CDE9005830790C2307EB0012202100203C
:1089F000121DFAF76AFC97E0F1F7CEFF012806D0C6
:108A000002280BD0042812D0082848D143E030793E
:108A100010B13079401E08E0042006E030790428C7
:108A200002D23079401C00E04846307137E031799D
:108A300094F8610761F3071084F8610700210320AF
:108A4000F1F7D2F858B30220FEF7ECFC94F8A10637
:108A500020F0800084F8A10694F8640780B1012812
:108A600013D0022802D0032807D109E094F8A10608
:108A700020F07800203084F8A106FDF781FED3E7CE
:108A800094F8A10620F07800F5E794F8A10620F00C
:108A900078005830EFE70920FEF7C4FCC4E7F0780F
:108AA0000E2841D1234804220021803000F07AF8BA
:108AB000CDE900B894F861075D46374F20F00F000C
:108AC000C219102319460020FAF7FFFB307994F8F9
:108AD0006117B0EB111F83D07FE7F1F75DFF01282D
:108AE00019D0022817D0042802D0082813D10FE08B
:108AF000F1F7D0F888F31388BFF34F8F2749086840
:108B0000274A00F4E06010430860BFF34F8FFEE790
:108B10000920FEF787FCF0780F2805D11E480422B3
:108B20000021503000F03EF8BDE8FE4FFAF760BA81
:108B3000BDE8FE8F32DD0108496E73657274205501
:108B40002D4469736B204669727374005468616EBA
:108B5000205061737320456E74657200466F726DAC
:108B600061743A46415433323B4D41583A333247AF
:108B70000000000046696E6420552D4469736B2C1B
:108B80004F7574707574696E67000000537461747A
:108B9000653A49646C65000032DE01080CED00E0C6
:108BA0000400FA052DE9F84F0025924688468146D3
:108BB000012715E000242E0109EB040101EB081048
:108BC00000EB051000970278E006F1B2000E1023CA
:108BD000FAF74AFA641CE4B2102CEDD36D1CEDB226
:108BE0005545E7D3BDE8F88F064800210172817230
:108BF00001214172C1726422026181710220FEF77B
:108C000011BC0000D4120020124810B5016841F4D4
:108C1000700101601048016841F0010101600E4AD5
:108C200000210832116002680C4B1A400260031DDB
:108C30000B4A1A60026822F48022026006480C3057
:108C40000160FEF79BFA03494FF00060803908602D
:108C500010BD000088ED00E000380240FFFFF6FE86
:108C600010300024FEF72CBAC94301827047002956
:108C7000018802D041F0010101E021F001010180F1
:108C800070470000464910B5884206D101210846C8
:108C9000FEF762F8002101205BE0B0F1804F09D0BF
:108CA000404988420DD101210220FEF73DF8002104
:108CB000022070E001210846FEF736F8002101206D
:108CC00069E03949884206D101210420FEF72CF8D9
:108CD000002104205FE03549884206D101210820A7
:108CE000FEF722F80021082055E03149884206D1DC
:108CF00001211020FEF718F8002110204BE02D492B
:108D0000884206D101212020FEF70EF80021202004
:108D100041E02949884206D101210220FEF71CF8D2
:108D20000021022015E02549884202D101210C04CE
:108D30000AE02349884202D101214C0404E0214980
:108D400088420AD101218C042046FEF705F8002153
:108D50002046BDE81040FDF7FFBF1B49884206D101
:108D600001214020FDF7E0FF0021402013E01749DA
:108D7000884206D101218020FDF7D6FF0021802006
:108D800009E0134988420AD1841501212046FDF7E4
:108D9000CBFF00212046BDE81040FDF7C5BF10BD48
:108DA000000001400004004000080040000C0040AA
:108DB0000010004000140040000401400040014049
:108DC000004401400048014000180040001C0040E1
:108DD0000020004002460020138A92890B4202EADA
:108DE000010202D0002A00D001207047002A8289A7
:108DF00001D00A4300E08A438281704730B502887F
:108E0000164C174DA0420DD0A8420BD0B0F1804FA8
:108E100008D0144B984205D0134B984202D0134B04
:108E2000984203D122F070034A881A43104B9842AB
:108E300006D0104B984203D022F440730A891A439B
:108E400002804A68C2620A880285A04201D0A84214
:108E500001D1897A01860121818230BD0000014063
:108E6000000401400004004000080040000C0040E5
:108E7000001000400014004010B5FDF799FE00F00E
:108E8000D9F9F0F7BDFF1448017821F00101017014
:108E9000017841F006010170002141800120F0F7C6
:108EA000A3FEF1F7CBFCF0F7D5F8F0F739FDF1F7B9
:108EB0008BFDF9F7A9FFFFF797FEF1F70BF9F9F72B
:108EC00071FBFDF75DFCFDF7F5FE04484FF4FA6118
:108ED000C1820121417510BD70240020D4120020F0
:108EE0002DE9F0470024F1F7B7FAD14D95F8320695
:108EF0000026A5F58057012808D185F83266F0F7DD
:108F000059FDF878022801D80120B87165E104EB19
:108F1000440007EB800000F5805090F8721601299C
:108F200001D180F8726690F8711600297DD190F811
:108F3000161B0129FAD104EB440101EB041107EBE4
:108F4000011909F5805292F88A1B00296DD080F82A
:108F5000166B92F88A0B072868D2DFE800F06704E6
:108F60003D73A5FCFC0004EB041000EB042007EBB0
:108F7000C00101F5005090F84730012B0BD090F85C
:108F8000463003EB031301EBC30303F5005393F8DF
:108F90004C30002B4AD190F846305B1C80F84630AC
:108FA00090F844302BB190F8443080F8463080F887
:108FB000446090F8463003EB031301EBC30303F561
:108FC000005393F84C30052B30D090F8460000EB5E
:108FD000001001EBC000C1E004EB041000EB042022
:108FE00007EBC00101F5005090F84730012B0BD082
:108FF00090F8463003EB031301EBC30303F5005372
:1090000093F84C30002B11D190F846305B1C80F85F
:10901000463090F844302BB190F8443080F8463018
:1090200080F8446090F8463001E0D4E056E003EB6D
:10903000031301EBC30303F5005393F84C300F2BDC
:10904000C3D19CE004EB041000EB042007EBC0014B
:1090500001F5005090F84730012B0AD090F84630C7
:1090600003EB031301EBC30303F5005393F84C30F8
:10907000A3BB90F846305B1C80F8463090F8443033
:109080002BB190F8443080F8463080F8446090F876
:10909000463003EB031301EBC30303F5005393F8CE
:1090A0004C30072B91D16AE004EB041000EB042054
:1090B00007EBC00303F5005090F8471001290AD0D0
:1090C00090F8461001EB011103EBC10101F50051CD
:1090D00091F84C1011B990F846101EE042E090F85B
:1090E000468009EB081C0CF5805C9CF8B58B09EBFD
:1090F000011C0CF5805C9CF8C5CBE04505D090F8D0
:109100004610491C80F846100BE090F846C00CF160
:10911000010C80F846C0491CC9B292F88BCB8C4533
:10912000DDD890F8441029B190F8441080F846102A
:1091300080F8446090F8461001EB011103EBC10187
:1091400001F5005191F84C10052918D090F846000F
:1091500000EB001000E006E003EBC00000F500505B
:1091600080F84C600BE004EB041000EB042007EBEC
:10917000C000463000F500500178491C017004EB36
:10918000041000EB042007EBC00303F5005090F837
:10919000461092F88B2B914201D380F8466090F8EC
:1091A000451051B190F8461080F8441090F84510E1
:1091B000491E80F8461080F8456010F8461F01EB04
:1091C000011103EBC10101F5005191F85120017823
:1091D0002046F7F71DFD641CE4B295F8E00AA042B2
:1091E0003FF695AE95F8630720B195F83E06012845
:1091F00007D010E095F84A0601280CD185F84A6698
:1092000001E085F83E6695F8662795F8621795F8AF
:109210006307FCF7DBF8F1F7BDFC95F8650718B1BB
:1092200085F86567FAF7A0F8BDE8F047FEF702B9E0
:10923000D42200202DE9FE4F012100240846FDF72D
:1092400067FDA720ADF80000002540F2E73001904F
:109250004FF0804BADF80250ADF8085069465846C3
:10926000FFF7CCFD864880F8B25741F2706C41F6AA
:10927000143841F6E42944F2742AA0F5805642F2EB
:10928000580704EB440106EB810190F8B22701EB8B
:109290000C0306EB820202F58052C2F8B43790F854
:1092A000B227521C80F8B22790F8B22701EB0803CE
:1092B00006EB820202F58052C2F8B43790F8B2276A
:1092C000521C80F8B22790F8B22701EB090306EB95
:1092D000820202F58052C2F8B43790F8B227521CCD
:1092E00080F8B22701EB0A0290F8B21706EB810171
:1092F00001F58051C1F8B42790F8B217491C80F8E5
:10930000B21704EB041202EB0422002106EBC205A3
:1093100001EB011205EBC20290F8B2373A4406EBBA
:10932000830303F58053C3F8B42790F8B227521C87
:1093300080F8B227491CC9B21029E9D3641CE4B2F1
:10934000042C9ED34F4A90F8B21706EB810101F529
:109350008051C1F8B42790F8B217491C80F8B217B1
:1093600090F8B217283A06EB810101F58051C1F857
:10937000B42790F8B217491C80F8B21790F8B217CA
:109380000C3206EB810101F58051C1F8B42790F849
:10939000B217491C80F8B21790F8B2170C3206EBDE
:1093A000810101F58051C1F8B42790F8B217491C2A
:1093B00080F8B21790F8B21702F5A47206EB81019B
:1093C00001F58051C1F8B42790F8B217491C80F814
:1093D000B21790F8B21702F54E7206EB810101F553
:1093E0008051C1F8B42790F8B217491C80F8B21721
:1093F00090F8B217A2F2A44206EB810101F5805168
:10940000C1F8B42790F8B217491C80F8B21790F849
:10941000B21702F5325206EB810101F58051C1F815
:10942000B42790F8B217491C80F8B217164990F883
:10943000B22706EB820202F58052C2F8B41790F808
:10944000B217491C80F8B217104A90F8B21706EB11
:10945000810101F58051C1F8B42790F8B217491C79
:1094600080F8B21701215C465846FFF700FC012244
:1094700011462046FFF7BAFC00F00AF8BDE8FE8F5F
:10948000D422002038290020DC120020785500204A
:1094900008B51C208DF8000001208DF80100022184
:1094A0008DF802108DF803006846F9F7FBFB08BD44
:1094B000F8F790BDF8F7AEBDFDF79CB8F8F764BDBE
:1094C000F8F7C8BDF1F7D6B8C94301807047002945
:1094D000818902D041F4005101E021F400518181E1
:1094E0007047002A828A01D00A4300E08A438282C0
:1094F000704700001C4910B5884206D10121102098
:10950000FDF72AFC0021102028E01849884202D1EA
:1095100001214C0410E01649884202D101218C043B
:109520000AE01449884202D10121CC0404E0124926
:1095300088420AD101210C052046FDF7F5FB2046A3
:10954000BDE810400021FDF7EFBB0C49884209D16E
:1095500001212020FDF700FC00212020BDE8104063
:10956000FDF7FABB10BD00000010014000440040B0
:1095700000480040004C00400050004000140140F2
:109580000246002012880A4200D00120704770B5C0
:1095900001F01F0501260024C1F3421306FA05F26B
:1095A000012B0FD0022B0FD0838A4FEA11210088A4
:1095B000134206FA01F600EA060001D000B10124C8
:1095C000204670BD8389F0E7038AEEE710B5C1F34A
:1095D000421301F01F040121A140012B07D0022BEF
:1095E00007D01430002A026805D00A4304E00C308A
:1095F000F8E71030F6E78A43026010BD7FB50446F5
:10960000008A0D46C98820F4405001432182A08978
:1096100041F20C618843A9882A8911436A8902436F
:109620001143A181A08A20F44071A8890843A08237
:109630006846FDF79DFB1A48844202D019488442CF
:1096400001D1039800E00298A189090400EBC00150
:1096500001EB0010296801D5490000E08900B0FB4A
:10966000F1F06422B0FBF2F109010B096FF018056B
:109670006B4300EB8300A3891D044FF0320306D532
:1096800003EBC000B0FBF2F000F0070005E003EBD5
:109690000010B0FBF2F000F00F00084320817FBD06
:1096A000001001400014014070B50024064DFDF784
:1096B00003FB20B1641CAC42F9D3FA2070BDBDE8B5
:1096C0007040EFF7E9BE0000404B4C000FB4084B70
:1096D00010B504A902AA039801F0E2F9044602A910
:1096E000002001F008FC204610BC5DF814FB0000CF
:1096F000F7AE010803B401984100009850EAC12078
:1097000018BF04204A0D18BF40F0010040F2FF725C
:10971000B2EB515F08BF40F00200012808BF0520EE
:1097200002B070470000000030B583B0044601F07D
:1097300093F99FED090B05468DED000B00222146A4
:109740006846EFF73CF8284601F09CF99DED000BC8
:1097500003B030BD00000000000000000000000069
:1097600070B5D94B00242DED020B2DED108BDDE9EA
:109770001010984205DA20F000429A4201D809D12F
:1097800041B19DED100BBDEC108B02B0BDE87040F7
:1097900001F01EB9B0F5801F26DA11430BD0002866
:1097A00013DA012001F06EF9BDEC108B02B0BDE8B8
:1097B000704001F021B9022001F064F901F0F0F8E5
:1097C00051EC100B81F000419EE06FF035049FEDED
:1097D000C00B53EC102B9DED100B51EC100BEEF762
:1097E0000FFECDE91001084604EB2051C0F313042D
:1097F000B948A1F2FF31204400F4801080F07F626C
:1098000082F04052224301EB20559FEDB50B11929F
:1098100053EC102B9DED100B51EC100BEEF7EAFD05
:1098200041EC180BA01CC0F313009FEDAFDB9FEDC4
:10983000B0EBB14E7E4403286CD296ED000B51EC98
:10984000180B53EC102BEFF7EBFA1DD1002D01BFD5
:1098500096ED000BBDEC108B02B070BD2846EEF704
:10986000B0FE41EC180B53EC1D2BEEF7C9FD41EC9B
:10987000190B53EC1E2B51EC180BEEF7C1FD53ECFA
:10988000192BEEF716FD3FE09FED9D0B51EC180BE9
:1098900053EC102BEEF7B4FD9FED9B1B53EC112BFB
:1098A000EEF7ABFD41EC190B53EC182B51EC180BF8
:1098B000EEF7A6FD53EC192BEEF7A2FD41EC190BC8
:1098C000002D04BF53EC192B51EC180B1AD028466D
:1098D000EEF777FE41EC1A0B53EC1D2BEEF790FDE3
:1098E00053EC192BEEF789FD53EC182BEEF782FDA4
:1098F00041EC180B53EC1E2B51EC1A0BEEF780FDCC
:1099000053EC182BEEF776FDBDEC108B02B041EC5A
:10991000100B70BD9FED7E0B51EC180B53EC102B10
:10992000EEF7C7FC41EC100B51EC180B53EC102B6D
:10993000EEF7D8FD41EC190B2846EEF742FE41EC5C
:109940001B0B53EC192B51EC190BEEF759FD41ECA5
:109950001A0B714853EC1A2B261851EC1A0BEEF720
:109960004FFD41EC1F0B6D48C4F1510404F5D724A1
:10997000B0EE4F0AF0EE6F0A0321784400F094FF36
:1099800053EC1F2B51EC100BEEF73AFD41EC1C0B86
:109990006348B0EE4F0AF0EE6F0A0421784400F0FD
:1099A00083FF53EC1A2B51EC100BEEF729FD3443D7
:1099B00053EC1C2BEEF77DFC41EC1C0B002C4CDD1A
:1099C0009FED510B51EC180B53EC102BEEF718FDDB
:1099D00053EC182BEEF714FD41EC1A0B55B353EC76
:1099E0001D2B51EC1B0BEEF70BFD41EC1D0B53EC4B
:1099F0001C2B51EC1A0BEEF75CFC53EC192BEEF719
:109A0000FFFC53EC1D2BEEF754FC53EC1A2BEEF736
:109A1000F4FC53EC182BEEF7EDFC41EC180B53EC77
:109A20001E2B51EC1B0BEEF7EBFC53EC182BEEF757
:109A3000E1FC69E753EC1C2B51EC1A0BEEF739FCF7
:109A400053EC192BEEF7DCFC53EC1A2BEEF7D5FC9C
:109A500053EC182BEEF7D1FC56E735B353EC1D2B26
:109A600051EC1B0BEEF7CCFC41EC1A0B53EC1C2B0E
:109A700051EC180BEEF7BEFC53EC192BEEF7C0FCC3
:109A800053EC1A2BEEF7B6FC53EC182BEEF7B2FCA6
:109A900041EC180B53EC1E2B51EC1B0BEEF7B0FCFA
:109AA00053EC182BEEF7A6FC2EE753EC1C2B51ECD5
:109AB000180BEEF79FFC53EC192BEEF7A1FC53ECBF
:109AC000182BEEF79AFC1FE70000F07F0000000063
:109AD0000000000000005043645F09000000000027
:109AE000000000000000F03F763C7935EF39EA3D98
:109AF0000000E0FE422EE63F50470000000000005C
:109B0000555555555555D53F000000000000E03F24
:109B1000000000000000004086EBF9FFD245000085
:109B2000C84500000000000070B5414A00252DED39
:109B3000020B2DED048BDDE90404944205DA24F0D8
:109B40000041914201D809D140B19DED040BBDEC1B
:109B5000048B02B0BDE8704000F03ABFB4F5801F3E
:109B600026DA08430BD0002C13DA012000F08AFF1C
:109B7000BDEC048B02B0BDE8704000F03DBF022098
:109B800000F080FF00F00CFF51EC100B81F0004161
:109B900046E09FED290B6FF0350553EC102B9DED42
:109BA000040B51EC100BEEF72BFCCDE904010C4635
:109BB00005EB2450A0F2FF30C10F40F2FF32521AE1
:109BC00062F31F540844EEF7FCFC05949DED040B72
:109BD00041EC180B51EC100B01F0C6FA9FED181B6D
:109BE00053EC112BEEF70CFC9FED170B41EC190B0E
:109BF00053EC102B51EC180BEEF702FC53EC192B25
